:020000040800F2
:1000000000040020A51F0008F71F0008F71F0008C4
:10001000F71F0008F71F0008F71F00080000000086
:10002000000000000000000000000000F71F0008B2
:10003000F71F000800000000F71F000851FE01082C
:10004000DDFF0108DFFF0108E1FF0108E5FF01080E
:100050000500020807000208090002082D00020836
:10006000510002087500020899000208BD0002084C
:10007000BF000208C1000208C3000208C500020850
:10008000C7000208C9000208CB000208F71F0008D9
:10009000F71F0008F71F0008F71F0008CD0002082F
:1000A000190102081B0102081D0102081F010208B4
:1000B000210102082501020851010208C1010208BC
:1000C000C3010208C5010208C7010208C9010208EC
:1000D000CD0102083D03020865020208010402087E
:1000E000C5040208890502088B0502088D0502086F
:1000F00091050208F9050208FB050208FD05020842
:10010000FF050208010602080306020805060208A8
:1001100009060208DD060208DF060208E1060208F9
:10012000ED070208EF070208F1070208F3070208CB
:1001300000000000000000000000000000000000BF
:1001400000000000000000000000000000000000AF
:10015000000000000000000000000000000000009F
:10016000000000000000000000000000000000008F
:10017000000000000000000000000000000000007F
:10018000000000000000000000000000000000006F
:10019000000000000000000000000000000000005F
:1001A000000000000000000000000000000000004F
:1001B000000000000000000000000000000000003F
:1001C000000000000000000000000000000000002F
:1001D000000000000000000000000000000000001F
:0401E0005FF8E0F1F3
:1001E800032A70B404460D4626D941EA000313F0E9
:1001F800030F13D020782B78984208BF294606D0E1
:100208001EE014F8010F11F8013F984218D1012A95
:1002180002F1FF32F5D1002070BC70470B4604464E
:1002280051F8045B50F8046BAE4204D1043A04461A
:10023800032A0B46F2D81D461046002ADAD1EBE70E
:10024800C01AE9E7032A2DE9F00109D82AB10023E9
:10025800CC5CC45401339342FAD1BDE8F001704735
:100268000B468218014603E02478013301F8014B5C
:1002780011F0030F1C46F7D113F003055DD06E4251
:10028800C5F1040CED009B594FEACC0C08E004348E
:10029800A7593B4607FA0CF748EA070741F8047BD9
:1002A800571A23FA05F8032FF1DC03E014F8013B91
:1002B80001F8013B8A42F9D8CFE753F8404C41F89E
:1002C800404C53F83C4C41F83C4C53F8384C41F8FE
:1002D800384C53F8344C41F8344C53F8304C41F80E
:1002E800304C53F82C4C41F82C4C53F8284C41F81E
:1002F800284C53F8244C41F8244C53F8204C41F82E
:10030800204C53F81C4C41F81C4C53F8184C41F83D
:10031800184C53F8144C41F8144C53F8104C41F84D
:10032800104C53F80C4C41F80C4C53F8084C41F85D
:10033800084C53F8044C41F8044C561A1D460C4618
:10034800403340313F2EB8DC2B460FE053F8101CE9
:1003580044F8101C53F80C1C44F80C1C53F8081CE7
:1003680044F8081C53F8041C44F8041C161B2146C6
:100378001D46103410330F2EE8DC2B4602E02468AB
:1003880041F8044B551A1C46032D03F10403F6DC0F
:1003980090E700BF032AC9B270B408D82AB103464F
:1003A800121803F8011B9342FBD170BC70478218E6
:1003B800044601E004F8011B14F0030FFAD14FF0D2
:1003C800013303FB01F31FE044F8403C44F83C3C94
:1003D80044F8383C44F8343C44F8303C44F82C3C6D
:1003E80044F8283C44F8243C44F8203C44F81C3C9D
:1003F80044F8183C44F8143C44F8103C44F80C3CCD
:1004080044F8083C44F8043C161B254640343F2E6B
:10041800DADC2C4607E044F8103C44F80C3C44F87D
:10042800083C44F8043C161B254610340F2EF2DC19
:1004380001E045F8043B541B032CFADC01E005F805
:10044800011B9542FBD3B0E710F0030F38B5044603
:1004580012D10368A3F1013222EA030313F0803FAB
:100468000AD1031D184653F8042BA2F1013525EAD9
:10047800020212F0803FF5D003782BB1431C1846D6
:1004880013F8012B002AFAD100F076F9204638BD7E
:10049800C9B2F0B4002950D010F0030F10D003787F
:1004A800002B79D0994246D0431C05E013F8012B64
:1004B800002A3FD091423ED013F0030F1846F5D1E1
:1004C800036841EA01270646A3F1013247EA0747D4
:1004D80022EA030212F0803F1DD187EA0303A3F149
:1004E800013222EA030313F0803F14D1043002E002
:1004F80012F0803F0FD1064650F8043BA3F10135B6
:1005080087EA030225EA0303A2F1013413F0803FCE
:1005180024EA0202ECD033783046002B3CD09942D2
:1005280009D0731C01E0914205D0184613F8012B3D
:10053800002AF8D11046F0BC704710F0030F0CD019
:100548000378002BF7D0431C03E013F8012B002A93
:10055800F1D013F0030F1846F7D102680346A2F151
:10056800013121EA020212F0803F0AD10430034629
:1005780050F8042BA2F1013121EA020212F0803F67
:10058800F5D01A781846002AD5D00133184613F842
:10059800012B002AFAD1CEE71846CCE780EA0102FF
:1005A80012F0030F3AD110F0030220F0030021F0FB
:1005B800030150F804CB08BF51F8043B0DD082F07A
:1005C80003024FEAC2026FF07F4323FA02F251F8A6
:1005D800043B4CEA020C43EA020300BFACF10132CF
:1005E8009C4501BF22EA0C0212F0803F50F804CB70
:1005F80051F8043BF2D04FEA0C604FEA1C2C01285A
:1006080028BFB0EB036F08BF1B0AF4D003F0FF0349
:100618004FEA1060A0EB0300704700BF10F0030F13
:100628000AD010F8012B11F8013B012A28BF9A4281
:10063800F4D0A2EB030070474DF8045D4DF8044D6B
:100648004FF0010242EA022242EA024201F0030CA0
:1006580021F0030150F8044B51F8045BBCF1020F80
:1006680026D04BD824F07F4CBCEB152FA4EB02030B
:1006780023EA04030DD113EAC21308BF51F8045B3F
:100688000AD18CEA040CBCEB056F0CD150F8044B72
:10069800E8E74FEA15255CE033F07F4352D10D7847
:1006A8004FEA146C55E04FEA146C05F0FF0550E072
:1006B8004FEA044CA4EB02034FEA1C4C23EA040360
:1006C800BCEB154F17D113EAC21308BF51F8045BEE
:1006D80007D18CEA040CBCEB054F08D150F8044B49
:1006E800E6E71B042ED10D884FEA144C31E04FEA9F
:1006F80005454FEA144C4FEA15452AE004F0FF0C73
:10070800BCEB156FA4EB020323EA04030DD113EA33
:10071800C21308BF51F8045B0AD18CEA040CBCEB85
:10072800052F0AD150F8044BE8E74FEA156510E0A9
:1007380014F0FF0F06D051F8045B4FEA142C25F093
:100748007F4506E04FF000005DF8044B5DF8045B60
:1007580070470CF0FF0205F0FF00012828BF904207
:1007680004BF4FEA1C2C2D0AF3D0A2EB00005DF861
:10077800044B5DF8045B704780EA0102844612F07E
:10078800030F4FD111F0030F32D14DF8044D11F082
:10079800040F51F8043B0BD0A3F101329A4312F035
:1007A800803F04BF4CF8043B51F8043B16D100BF0E
:1007B80051F8044BA3F101329A4312F0803FA4F19F
:1007C80001320BD14CF8043BA24312F0803F04BF26
:1007D80051F8043B4CF8044BEAD023460CF8013B93
:1007E80013F0FF0F4FEA3323F8D15DF8044B70473D
:1007F80011F0010F06D011F8012B0CF8012B002A7B
:1008080008BF704711F0020FBFD031F8022B12F069
:10081800FF0F16BF2CF8022B8CF8002012F47F4F24
:10082800B3D1704711F8012B0CF8012B002AF9D12C
:10083800704700BF20F0030110F00300C0F1000072
:1008480051F8043B00F1040C4FEACC0C6FF00002A5
:100858001CBF22FA0CF213434FF0010C4CEA0C2C8B
:100868004CEA0C4CA3EB0C0222EA030212EACC126B
:1008780004BF51F8043B0430F4D013F0FF0F1FBF3E
:10088800013013F47F4F013013F47F0F18BF01308C
:10089800704700BFF0B4002A46D041EA000313F0C5
:1008A80003032CD1032A07460E4643D904680D6872
:1008B800AC423FD1043A37D0A4F1013525EA04040B
:1008C80014F0803F18BF18462CD1041D0D1D0EE0F2
:1008D80054F8043B55F8041BA3F101308B4220EA7D
:1008E800030027D1043A1FD010F0803F1ED1032AFD
:1008F80027462E46ECD820462946002A1DD00478E3
:10090800013A0D78AC420CD172B18CB1002302E0EF
:1009180093420BD064B1013310F8014FCD5CAC4267
:10092800F6D0601BF0BC70471046FBE70020F9E7E3
:100938002046F7E738463146E1E724782D78F0E796
:1009480041EA000313F0030F0B4670B414BF0024F0
:100958000124032A94BF002404F001040546D4B9F5
:10096800BAB10E782B46013A03F8016B56B1AC1CAC
:100978007AB111F8015F2346013A04F8015C0134A9
:10098800002DF5D12AB19A18002103F8011B9342D2
:10099800FBD170BC7047194653F8044BA4F10136DB
:1009A80026EA040616F0803FDAD1043A45F8044BEB
:1009B800032A1946EFD8D3E701232DE9F0071D468E
:1009C80000264FF0FF37AC1900EB070C8C420DD214
:1009D8001CF805C010F80480E0452ED201252646F3
:1009E800E31BAC198C4200EB070CF1D34FF0010963
:1009F80000264D464FF0FF3C1360AC1900EB0C0885
:100A0800A1420ED918F8058010F804A0C2451AD9D9
:100A180001252646CCEB0409AC19A14200EB0C08D1
:100A2800F0D80CF101000137B8423CBF994638466E
:100A3800C2F80090BDE8F00770470BD00123374695
:100A48001D46F618BFE709D04FF00109B4464D46D8
:100A58004E44D2E79D4205D00135B4E74D4505D057
:100A68000135CAE72B4626460125ACE7A9462646A6
:100A78000125C2E72DE9F04FADF5826D81B014462E
:100A8800074610460DF580628B460C3219461D4606
:100A9800FFF792FF03AE04A901F57E72331F0090A1
:100AA80043F8045F9342FBD14DB1681E0023E25C1A
:100AB800C11A013303AEAB4246F82210F7D1DDF874
:100AC8000C142046009A6118FFF78AFB002877D19A
:100AD8000099814605F1FF380646C1F101020192ED
:100AE8005A46AB4609EB0B0501F1FF3AB81800214D
:100AF800AA1A00F0E5F900284FD1002D00F0C080B7
:100B08007B1903A913F8013C51F82330002B4CD171
:100B1800009B9E4228BF334698450FD903EB090135
:100B2800E05C7A18795C884205D038E012F8011F39
:100B3800E05C884233D101339845F7D8009A964251
:100B480080F0A48007EB090214F80A10534612F843
:100B58000A20914204BF0AEB0901791807D095E0F1
:100B680014F802C011F8010D844503D113465A1E2A
:100B7800B342F5D101369E4200F28D80DDF80C6457
:100B88002A46B144C6EB0B0609EB0B05B818002141
:100B9800AA1A00F095F90028AFD0002071E0019A58
:100BA8000026914499442A46EEE7002EFAD0DDF853
:100BB8000C2493423CBFC2EB0B0306469944F2E770
:100BC800009E4FF000080099AB1BB34238BF334674
:100BD800C1F101026E1E019201F1FF3A5A4689469F
:100BE800AB460133CDF80C3408EB0B05B8180021DF
:100BF800AA1A00F065F90028CFD1002D40D07B1942
:100C080003A913F8013C51F82330002B30D1B1452A
:100C180013D208EB090314F80910FA18FB5C99427F
:100C280018BF4B4627D14B4604E012F8011FE05C81
:100C3800884220D10133B342F7D3BAF1FF3F53467C
:100C48002CD007EB080C14F80A101CF80A20914263
:100C58000CD10AEB0802BA1804E0E05C12F8011D96
:100C6800884203D1013BF8D260460AE0DDF80C3433
:100C780098442A46B8E701992A4688449844B3E735
:100C8800284605B00DF5806DBDE8F08F009B013654
:100C98009E427FF673AF07EB0900F2E707EB080CFB
:100CA8006046EEE72DE9F04F8346037885B00C46A1
:100CB800002B00F0F9800A78A2B106460131012024
:100CC80002E011F8012B8AB1934214BF002000F012
:100CD800010016F8013F0D46002BF2D12B782BB1FD
:100CE8004FF0000B584605B0BDE8F08F0028F9D149
:100CF8000BF101002178FFF7CBFB2D1BA5F10102B9
:100D0800534243EB0203002808BF43F001030746A0
:100D180083B90BEB0508404594BFC0EB08084FF0BA
:100D280001081F2D08D9414622462B46FFF7A2FE8F
:100D38008346D7E78346D5E7294603AA2046FFF727
:100D48003BFE03996118814620464A46FFF748FA58
:100D580000284FD109F1FF33C9F10102064601927B
:100D680082464246C84699460AEB050BB818002148
:100D7800C2EB0B0200F0A4F80028B1D1BBF1000FC0
:100D8800B0D046452CBF334643469D420FD903EBAE
:100D98000A01E05C7A18795C884205D075E012F89F
:100DA800011FE05C884270D101339D42F7D1B04504
:100DB8007DD907EB0A0214F809104B4612F80920EE
:100DC800914202BF09EB0A01AC46791806D06EE0E1
:100DD800A55C11F8010D854203D113465A1EB34292
:100DE800F6D1654601369E4267D8039E5A46B244FC
:100DF800AE1BB9E7C9F10101C9EB0503424600265C
:100E080009F1FF3A88464B4538BF4B4601330393F7
:100E180006EB050BB8180021C2EB0B0200F050F8E6
:100E280000287FF45DAFBBF1000F3FF45BAF4D4589
:100E380012D906EB090314F80910FA18FB5C994259
:100E480008BF4B4605D026E012F8011FE05C884237
:100E580022D101339D42F7D1BAF1FF3F534628D042
:100E680007EB060C14F80A101CF80A20914217D157
:100E78000AEB0602BA1804E0E05C12F8011D884289
:100E88000ED1013BF8D2E3462CE7019A00269244A2
:100E98005A469A4468E74B4646445A46F618B7E716
:100EA800039B5A46F618B3E70D46012016E743465A
:100EB80098E707EB060CE34614E707EB0A0B11E784
:100EC80010F0030F034670B4C9B211D0002A22D023
:100ED80003788B421DD0013A013005E0DAB110F8F1
:100EE800014B013A8C4218D010F0030F0346F5D19C
:100EF800032A14D87AB1187888420ED0541E5D1C83
:100F080003E015F8016B8E4203D0013C2846F8D265
:100F1800002070BC70471046FBE71846F9E741EA25
:100F2800012646EA0646184653F8044B86EA0404A6
:100F3800A4F1013525EA040414F0803F03D1043AF2
:100F48001846032AEFD80346D4E700BF0000000084
:100F5800C1F30A5C0246ACF57E7C2DE9F84FACF192
:100F68000704132C0B4606460F468946804627DCA5
:100F7800002C52DB4FF6FF7CC0F20F0C4CFA04FA3F
:100F88000AEA0105054317D037A3D3E9002300F087
:100F980075F80022002300F0B3FC002856D0002F7B
:100FA80005DD4FF4801353FA04F407EB040929EA2A
:100FB8000A0900264B46324610461946BDE8F88F06
:100FC800332C07DDB4F5806FF6D100F057F80246F0
:100FD8000B46F1E74FF0FF3BACF11B0C2BFA0CFB77
:100FE8001BEA000FE8D020A3D3E9002300F046F85D
:100FF8000022002300F084FC40B3002F0ADD142CEB
:1010080006D00126C4F13404A64016EB080601D325
:1010180007F1010926EA0B0619E013A3D3E9002317
:1010280000F02CF80022002300F06AFC78B1002FB1
:1010380013DB46EA07054FF000094D45C3F6F07982
:101048000CBF2E46002608BFA94600E0B9464B460D
:10105800324610461946BDE8F88F00264FF0004981
:10106800F5E700BFAFF300809C7500883CE4377E4D
:1010780081F0004102E000BF83F0004330B54FEA41
:1010880041044FEA430594EA050F08BF90EA020FAE
:101098001FBF54EA000C55EA020C7FEA645C7FEA41
:1010A800655C00F0E2804FEA5454D4EB5555B8BF64
:1010B8006D420CDD2C4480EA020281EA030382EAD5
:1010C800000083EA010180EA020281EA0303362D67
:1010D80088BF30BD11F0004F4FEA01314FF4801C3A
:1010E8004CEA113102D0404261EB410113F0004F4C
:1010F8004FEA03334CEA133302D0524263EB430303
:1011080094EA050F00F0A780A4F10104D5F1200EA0
:101118000DDB02FA0EFC22FA05F2801841F10001FB
:1011280003FA0EF2801843FA05F359410EE0A5F1CF
:1011380020050EF1200E012A03FA0EFC28BF4CF000
:10114800020C43FA05F3C01851EBE37101F00045B6
:1011580007D54FF0000EDCF1000C7EEB00006EEBC3
:101168000101B1F5801F1BD3B1F5001F0CD349084D
:101178005FEA30004FEA3C0C04F101044FEA4452A4
:1011880012F5800F80F09A80BCF1004F08BF5FEA2B
:10119800500C50F1000041EB045141EA050130BD0B
:1011A8005FEA4C0C404141EB010111F4801FA4F1AE
:1011B8000104E9D191F0000F04BF01460020B1FA03
:1011C80081F308BF2033A3F10B03B3F120020CDA3B
:1011D8000C3208DD02F1140CC2F10C0201FA0CF019
:1011E80021FA02F10CE002F11402D8BFC2F1200C7E
:1011F80001FA02F120FA0CFCDCBF41EA0C01904034
:10120800E41AA2BF01EB0451294330BD6FEA04047C
:101218001F3C1CDA0C340EDC04F11404C4F1200267
:1012280020FA04F001FA02F340EA030021FA04F379
:1012380045EA030130BDC4F10C04C4F1200220FAD0
:1012480002F001FA04F340EA0300294630BD21FA0E
:1012580004F0294630BD94F0000F83F4801306BFD4
:1012680081F480110134013D4EE77FEA645C18BFC8
:101278007FEA655C29D094EA050F08BF90EA020F5F
:1012880005D054EA000C04BF1946104630BD91EA57
:10129800030F1EBF0021002030BD5FEA545C05D15A
:1012A8004000494128BF41F0004130BD14F5800499
:1012B8003CBF01F5801130BD01F0004545F0FE410D
:1012C80041F470014FF0000030BD7FEA645C1ABF42
:1012D800194610467FEA655C1CBF0B46024650EA79
:1012E800013406BF52EA033591EA030F41F40021A5
:1012F80030BD00BF90F0000F04BF0021704730B52B
:101308004FF4806404F132044FF000054FF00001FF
:1013180050E700BF90F0000F04BF0021704730B5C0
:101328004FF4806404F1320410F0004548BF404295
:101338004FF000013EE700BF42004FEAE2014FEAEA
:1013480031014FEA02701FBF12F07F4393F07F4FC5
:1013580081F06051704792F0000F14BF93F07F4FF7
:10136800704730B54FF4607401F0004521F000413A
:1013780020E700BF50EA010208BF704730B54FF0C0
:1013880000050AE050EA010208BF704730B511F0C5
:10139800004502D5404261EB41014FF4806404F1FD
:1013A80032045FEA915C3FF4DCAE4FF003025FEA7F
:1013B800DC0C18BF03325FEADC0C18BF033202EB07
:1013C800DC02C2F1200300FA03FC20FA02F001FA61
:1013D80003FE40EA0E0021FA02F11444C1E600BF00
:1013E80070B54FF0FF0C4CF4E06C1CEA11541DBFB3
:1013F8001CEA135594EA0C0F95EA0C0F00F0DEF87E
:101408002C4481EA030621EA4C5123EA4C5350EA62
:10141800013518BF52EA033541F4801143F48013B3
:1014280038D0A0FB02CE4FF00005E1FB02E506F044
:101438000042E0FB03E54FF00006E1FB03569CF099
:10144800000F18BF4EF0010EA4F1FF04B6F5007F9F
:1014580064F5407404D25FEA4E0E6D4146EB060611
:1014680042EAC62141EA55514FEAC52040EA5E509A
:101478004FEACE2EB4F1FD0C88BFBCF5E06F1ED844
:10148800BEF1004F08BF5FEA500E50F1000041EB7B
:10149800045170BD06F0004646EA010140EA020028
:1014A80081EA0301B4EB5C04C2BFD4EB0C0541EA4A
:1014B800045170BD41F480114FF0000E013C00F35F
:1014C800AB8014F1360FDEBF002001F0004170BD83
:1014D800C4F10004203C35DA0C341BDC04F114049C
:1014E800C4F1200500FA05F320FA04F001FA05F228
:1014F80040EA020001F0004221F0004110EBD370F5
:1015080021FA04F642EB06015EEA430E08BF20EA20
:10151800D37070BDC4F10C04C4F1200500FA04F3C3
:1015280020FA05F001FA04F240EA020001F0004155
:1015380010EBD37041F100015EEA430E08BF20EAC8
:10154800D37070BDC4F1200500FA05F24EEA020E10
:1015580020FA04F301FA05F243EA020321FA04F03F
:1015680001F0004121FA04F220EA020000EBD370F6
:101578005EEA430E08BF20EAD37070BD94F0000FF6
:101588000FD101F00046400041EB010111F4801F2A
:1015980008BF013CF7D041EA060195F0000F18BFDB
:1015A800704703F00046520043EB030313F4801F17
:1015B80008BF013DF7D043EA0603704794EA0C0FD1
:1015C8000CEA135518BF95EA0C0F0CD050EA4106E7
:1015D80018BF52EA4306D1D181EA030101F0004164
:1015E8004FF0000070BD50EA410606BF104619468C
:1015F80052EA430619D094EA0C0F02D150EA013698
:1016080013D195EA0C0F05D152EA03361CBF1046D8
:1016180019460AD181EA030101F0004141F0FE4177
:1016280041F470014FF0000070BD41F0FE4141F4FB
:10163800780170BD70B54FF0FF0C4CF4E06C1CEAFB
:1016480011541DBF1CEA135594EA0C0F95EA0C0FB0
:1016580000F0A7F8A4EB050481EA030E52EA03356B
:101668004FEA013100F088804FEA03334FF080558C
:1016780045EA131343EA12634FEA022245EA1115B9
:1016880045EA10654FEA00260EF000419D4208BF6A
:10169800964244F1FD0404F5407402D25B084FEA17
:1016A8003202B61A65EB03055B084FEA32024FF4C3
:1016B80080104FF4002CB6EB020E75EB030E22BF20
:1016C800B61A754640EA0C005B084FEA3202B6EBE0
:1016D800020E75EB030E22BFB61A754640EA5C008F
:1016E8005B084FEA3202B6EB020E75EB030E22BF1F
:1016F800B61A754640EA9C005B084FEA3202B6EB20
:10170800020E75EB030E22BFB61A754640EADC00DE
:1017180055EA060E18D04FEA051545EA16754FEA40
:1017280006164FEAC30343EA52734FEAC2025FEA5E
:101738001C1CC0D111F4801F0BD141EA00014FF0ED
:1017480000004FF0004CB6E711F4801F04BF0143BE
:101758000020B4F1FD0C88BFBCF5E06F3FF6AFAEDA
:10176800B5EB030C04BFB6EB020C5FEA500C50F16A
:10177800000041EB045170BD0EF0004E4EEA1131ED
:1017880014EB5C04C2BFD4EB0C0541EA045170BDF4
:1017980041F480114FF0000E013C90E645EA060E38
:1017A8008DE60CEA135594EA0C0F08BF95EA0C0F66
:1017B8003FF43BAF94EA0C0F0AD150EA01347FF4AE
:1017C80034AF95EA0C0F7FF425AF104619462CE785
:1017D80095EA0C0F06D152EA03353FF4FDAE1046E8
:1017E800194622E750EA410618BF52EA43067FF439
:1017F800C5AE50EA41047FF40DAF52EA43057FF4C9
:10180800EBAE12E74FF0FF3C06E000BF4FF0010CD3
:1018180002E000BF4FF0010C4DF804CD4FEA410C37
:101828007FEA6C5C4FEA430C18BF7FEA6C5C1BD004
:1018380001B050EA410C0CBF52EA430C91EA030F85
:1018480002BF90EA020F0020704710F1000F91EAE2
:10185800030F58BF994208BF90422CBFD8176FEAB0
:10186800E37040F0010070474FEA410C7FEA6C5C7E
:1018780002D150EA013C07D14FEA430C7FEA6C5C85
:10188800D6D152EA033CD3D05DF8040B704700BFB1
:101898008446104662468C461946634600E000BFFF
:1018A80001B5FFF7B7FF002848BF10F1000F01BDD1
:1018B8004DF808EDFFF7F4FF0CBF012000205DF89C
:1018C80008FB00BF4DF808EDFFF7EAFF34BF012021
:1018D80000205DF808FB00BF4DF808EDFFF7E0FFBA
:1018E80094BF012000205DF808FB00BF4DF808ED0B
:1018F800FFF7CEFF94BF012000205DF808FB00BF72
:101908004DF808EDFFF7C4FF34BF012000205DF853
:1019180008FB00BF4FEA4102B2F1E04324BFB3F530
:10192800001CDCF1FE5C0DD901F0004C4FEAC0024E
:101938004CEA5070B2F1004F40EB830008BF20F032
:101948000100704711F0804F21D113F13872BCBFEC
:1019580001F00040704741F480114FEA5252C2F141
:101968001802C2F1200C10FA0CF320FA02F018BF8A
:1019780040F001004FEAC1234FEAD32303FA0CFCDD
:1019880040EA0C0023FA02F34FEA4303CCE77FEA6C
:10199800625307D150EA01331EBF4FF0FE4040F4B6
:1019A8004000704701F0004040F0FE4040F4000065
:1019B800704700BF80F0004002E000BF81F00041A6
:1019C80042001FBF5FEA410392EA030F7FEA226CDD
:1019D8007FEA236C6AD04FEA1262D2EB1363C1BF6D
:1019E800D218414048404140B8BF5B42192B88BFDC
:1019F800704710F0004F40F4000020F07F4018BFFF
:101A0800404211F0004F41F4000121F07F4118BF1E
:101A1800494292EA030F3FD0A2F1010241FA03FCC6
:101A280010EB0C00C3F1200301FA03F100F00043AE
:101A380002D5494260EB4000B0F5000F13D3B0F176
:101A4800807F06D340084FEA310102F10102FE2AE5
:101A580051D2B1F1004F40EBC25008BF20F0010055
:101A680040EA03007047490040EB000010F4000F03
:101A7800A2F10102EDD1B0FA80FCACF1080CB2EB96
:101A88000C0200FA0CF0AABF00EBC25052421843F5
:101A9800BCBFD0401843704792F0000F81F400019A
:101AA80006BF80F400000132013BB5E74FEA41036D
:101AB8007FEA226C18BF7FEA236C21D092EA030FD9
:101AC80004D092F0000F08BF0846704790EA010F53
:101AD8001CBF0020704712F07F4F04D1400028BF80
:101AE80040F00040704712F100723CBF00F5000062
:101AF800704700F0004343F0FE4040F40000704798
:101B08007FEA226216BF08467FEA23630146420243
:101B180006BF5FEA412390EA010F40F48000704756
:101B28004FF0000304E000BF10F0004348BF4042FC
:101B38005FEA000C08BF704743F0964301464FF038
:101B480000001CE050EA010208BF70474FF0000394
:101B58000AE000BF50EA010208BF704711F00043D5
:101B680002D5404261EB41015FEA010C02BF8446A5
:101B78000146002043F0B64308BFA3F18053A3F504
:101B88000003BCFA8CF2083AA3EBC25310DB01FA4B
:101B980002FC634400FA02FCC2F12002BCF1004FCF
:101BA80020FA02F243EB020008BF20F00100704760
:101BB80002F1200201FA02FCC2F1200250EA4C00B4
:101BC80021FA02F243EB020008BF20EADC707047FA
:101BD8004FF0FF0C1CEAD0521EBF1CEAD15392EA08
:101BE8000C0F93EA0C0F6FD01A4480EA010C4002E4
:101BF80018BF5FEA41211ED04FF0006343EA50103E
:101C080043EA5111A0FB01310CF00040B1F5000F7F
:101C18003EBF490041EAD3715B0040EA010062F12E
:101C28007F02FD2A1DD8B3F1004F40EBC25008BF18
:101C380020F00100704790F0000F0CF0004C08BF36
:101C480049024CEA502040EA51207F3AC2BFD2F103
:101C5800FF0340EAC250704740F400004FF0000311
:101C6800013A5DDC12F1190FDCBF00F0004070474B
:101C7800C2F10002410021FA02F1C2F1200200FA89
:101C880002FC5FEA310040F1000053EA4C0308BF50
:101C980020EADC70704792F0000F00F0004C02BFA1
:101CA800400010F4000F013AF9D040EA0C0093F01C
:101CB800000F01F0004C02BF490011F4000F013B76
:101CC800F9D041EA0C018FE70CEAD15392EA0C0FE4
:101CD80018BF93EA0C0F0AD030F0004C18BF31F04F
:101CE800004CD8D180EA010000F00040704790F025
:101CF800000F17BF90F0004F084691F0000F91F0C9
:101D0800004F14D092EA0C0F01D142020FD193EA8E
:101D18000C0F03D14B0218BF084608D180EA010016
:101D280000F0004040F0FE4040F40000704740F0F2
:101D3800FE4040F4400070474FF0FF0C1CEAD052C0
:101D48001EBF1CEAD15392EA0C0F93EA0C0F69D01C
:101D5800A2EB030280EA010C49024FEA402037D087
:101D68004FF0805343EA111143EA10130CF000407E
:101D78008B4238BF5B0042F17D024FF4000C8B426E
:101D880024BF5B1A40EA0C00B3EB510F24BFA3EB4E
:101D9800510340EA5C00B3EB910F24BFA3EB91031E
:101DA80040EA9C00B3EBD10F24BFA3EBD10340EA78
:101DB800DC001B0118BF5FEA1C1CE0D1FD2A3FF6BE
:101DC80050AF8B4240EBC25008BF20F00100704773
:101DD8000CF0004C4CEA50207F32C2BFD2F1FF0316
:101DE80040EAC250704740F400004FF00003013A47
:101DF80037E792F0000F00F0004C02BF400010F4EB
:101E0800000F013AF9D040EA0C0093F0000F01F0FE
:101E1800004C02BF490011F4000F013BF9D041EA20
:101E28000C0195E70CEAD15392EA0C0F08D1420253
:101E38007FF47DAF93EA0C0F7FF470AF084676E726
:101E480093EA0C0F04D14B023FF44CAF08466EE7FF
:101E580030F0004C18BF31F0004CCAD130F00042CD
:101E68007FF45CAF31F000437FF43CAF5FE700BF25
:101E78004FF0FF3C06E000BF4FF0010C02E000BF4E
:101E88004FF0010C4DF804CD4FEA40024FEA4103F0
:101E98007FEA226C18BF7FEA236C11D001B052EAA6
:101EA800530C18BF90EA010F58BFB2EB030088BF6C
:101EB800C81738BF6FEAE17018BF40F001007047DB
:101EC8007FEA226C02D15FEA402C05D17FEA236CBD
:101ED800E4D15FEA412CE1D05DF8040B704700BF04
:101EE800844608466146FFE70FB5FFF7C9FF00289B
:101EF80048BF10F1000F0FBD4DF808EDFFF7F4FFD4
:101F08000CBF012000205DF808FB00BF4DF808ED6C
:101F1800FFF7EAFF34BF012000205DF808FB00BF8F
:101F28004DF808EDFFF7E0FF94BF012000205DF8B1
:101F380008FB00BF4DF808EDFFF7D2FF94BF012062
:101F480000205DF808FB00BF4DF808EDFFF7C8FF5B
:101F580034BF012000205DF808FB00BF42000ED20C
:101F6800B2F1FE4F0BD34FF09E03B3EB126209D4CC
:101F78004FEA002343F0004323FA02F070474FF082
:101F88000000704712F1610F01D1420202D14FF0F7
:101F9800FF3070474FF00000704700BF00F026F890
:101FA8000C4880F30888002103E00B4B5B58435032
:101FB80004310A480A4B42189A42F6D3094A02E009
:101FC800002342F8043B084B9A42F9D317F084FBEC
:101FD8007047000000C00020EC3603080000002015
:101FE800280E0020280E0020C84400207047FEE775
:101FF80010B586B0002301244FF46022114801A9CE
:1020080001938DF80930039204938DF808408DF8F8
:10201800144021F0DDF90B48214621F0FFF9094869
:1020280021F006FA074821F008FA0028FAD10548F5
:1020380021F007FA034821F009FA0028FAD106B07E
:1020480010BD00BF00240140014610B50D48012213
:10205800032321F009FA0B48012121F0FBF97F2025
:1020680022F038F80748022121F048FA0028F6D073
:102078000448022121F048FA0248BDE8104021F046
:102088003ABA00BF002401400C4A0C2303FB012389
:1020980010B59C880CB9588010BD5B8803F11304F7
:1020A800844204DA142B07D9133B834204DC0C2343
:1020B80003FB012102238B8010BD00BF3C260020BA
:1020C8000A4B10B500241C7021464FF4E0720848F2
:1020D800FEF760F9074B4FF474501C70064B1C70E8
:1020E8000EF09EFE054B187010BD00BFF4100020C6
:1020F800C01200200B150020881400208A1400202C
:10210800074B1978013101F01F011970054B1A7836
:102118008A4203D1013202F01F021A70704700BFD1
:10212800881400200B15002010B50E4A0E2303FB5F
:1021380000200D4A014614780C4A03FB042300F1E1
:102148000C0251F8044B914243F8044BF9D10A8828
:1021580000211A800E22FEF71DF9BDE81040FFF796
:10216800CFBF00BFF810002088140020C012002044
:10217800084B1A5C002352FA03F111F0010FD8B290
:1021880002D00130C0B270470133082BF3D10120CF
:10219800704700BFC915002000F07F0000F574509B
:1021A8002DE9F84305300C46154698460EF038FEE2
:1021B80000284ED043F63837002638460EF030FE59
:1021C800C0B25FFA86F988B120280FD04FEA5909C2
:1021D8004AF20B5048440EF023FEC0B208B1022860
:1021E80004D10123B34022781343237011370136F9
:1021F800B7F56F5FE1D14AF2B2300EF011FEC0B20E
:1022080080B120280ED02B784AF2A13043F0010388
:102218002B700EF005FEC0B220B1202802D0012399
:1022280088F800304AF2E3300EF0FAFDC0B280B10F
:1022380020280ED02B784AF2A13043F002032B70ED
:102248000EF0EEFDC0B220B1202802D0012388F89C
:102258000030BDE8F8830000034610465A1E10B54A
:10226800032A1CD8DFE802F00E0E0207114A527842
:1022780002F0100203E00F4A527802F00802D2B2CC
:1022880072B10BE00C4A927802F04002D2B23AB135
:102298000A4A127802F003029A4200D140B10022A1
:1022A8000748105C984203D00132052AF8D1002172
:1022B800084610BDD842002040320020D336002006
:1022C800B8120020F8B5064643F6383500242846EB
:1022D8000EF0A6FDC0B2E7B268B120280BD07F0887
:1022E8004AF20B5038180EF09BFD012803D1A0408C
:1022F80033781843307001341135082CE7D1F8BD14
:1023080003780E2202FB0313084AD3189978002396
:1023180051FA03F010F00100DAB202D0501CC0B23A
:1023280070470133082BF3D1704700BFC01200205B
:102338002DE9F04101248C40284A29490346E4B29A
:10234800107891F800C019E0264F0E2606FB00769B
:10235800F178A9B996F80680B8F1000F10D196F86F
:102368000580B8F1000F0BD196F80480B8F1000F82
:1023780006D1F67926B9013000F01F00054626E09F
:10238800FBB1012B05D0022B06D10E2101FB0077F2
:1023980039790C4218D014E0042B04D10E2101FB2A
:1023A8000077B9790CE0032B04D10E2101FB0077EB
:1023B800797905E0052B07D10E2101FB0077F97922
:1023C80011B11570BDE8F081013000F01F006045C3
:1023D800BAD11570FF20BDE8F08100BF0B150020B1
:1023E80088140020C01200202DE9F043434D444BCF
:1023F8002A780E2101FB0232917A85B0044698466C
:1024080031B101390523594301F56F5189B201E012
:102418004FF46F51204604220EF013FD2B780E2541
:1024280005FB038393F80B80354E344FB8F1000F4A
:1024380025D131232371073363713B7801A86B439E
:102448000422F15E06F084FA3B7802A805FB0363D8
:102458000222997A06F07CFA3B780DF10A0005FB16
:1024680003650322697A06F073FAA01D01A90922FF
:10247800FEF766FA4FF00F0984F8108012E0B8F101
:10248800010F0FD132232371053363713B784FF06D
:10249800080905FB036393F90130E3713B785D4359
:1024A800735BA371002320461A4612E010F8011B43
:1024B800A1F13005EDB2092D04D8EB183029DBB2B3
:1024C80003D004E037395B1800E00A33DBB201328D
:1024D800D2B24A45EAD10F21B3FBF1F10801411A02
:1024E8005B1AC3F10F03DBB2092BA35401D83033B5
:1024F80000E03733A35405B0BDE8F083BE120020D6
:10250800C0120020024B1A7842F001021A7070477C
:102518005518002008B50C4B0C4A1B780E2101FBFE
:102528000323D97A21B101290CBF0921002100E038
:10253800102140221346064806F02EF8054B1A785B
:1025480042F002021A7008BDBE120020C01200201C
:102558008B14002055180020034B1A7802F0F8025B
:102568006FF3C3021A70704755180020024B1A788F
:1025780042F004021A70704755180020024B1A786E
:1025880042F008021A7070475518002038B5114BF0
:102598001C7814F0010502D1FFF7B4FF05E004F040
:1025A8000405EDB21DB9FFF7E1FF284638BD04F078
:1025B8000805EDB215B9FFF7E1FFF6E704F00204EC
:1025C800E4B21CB9FFF7A6FF204638BDFFF7C4FFE9
:1025D800012038BD55180020014B1878704700BFFE
:1025E800F410002030B51E4B85B01B780446002B34
:1025F80034D11C4D2B78034113F0010F2ED01A4B08
:102608001A4A1B780E2101FB0323DA78024112F0E3
:10261800010F1CD11B79034113F0010317D110F0EE
:10262800010001F1F1014FEA540206D00132009194
:10263800019302926D20FE3905E00132009101906C
:1026480002923C20012103220B460EF067FC012375
:1026580013FA04F42B7823EA04042C7005B030BD77
:102668008A140020811400200B150020C0120020BD
:10267800037830B513F0010F144A4FF00E0419D146
:1026880004FB01210133012212FA03F3CD7825EA74
:102698000303CB7004780D79A41812FA04F425EA20
:1026A80004040C7103789B189A408B7823EA020281
:1026B8008A7030BD04FB0121013B012212FA03F3A9
:1026C8008A7822EA03038B7030BD00BFC012002055
:1026D80010B500230278590052FA01F404F00304FB
:1026E800022C05D1013414FA01F122EA0102027028
:1026F8000133042BEED110BD2DE9F04F85B00192C6
:10270800BDF838201C46734B0092DA78054612F063
:1027180020028B4640F0D8808DF80E208DF80F20CF
:102728008DF80D20DCB99B7803F04003DBB21BB1B8
:1027380001238DF80F3020E0674B5B7803F002032C
:10274800DBB21BB101238DF80E3016E00DF10F013D
:102758000DF10E020DF10D03FFF71EFD0DE0012C2A
:102768000BD19B7803F04003DBB223B90DF10F00C6
:10277800FFF7A8FD01E08DF80F409DF80F3023B951
:102788009DF80E00002800F0A28044B905F07F01F2
:10279800490001F574510DF10A00623109E0012C7C
:1027A8000AD1E90101F50C413C310DF10A0001EBB8
:1027B8004B0102220EF045FBBDF90A3013B9002C7B
:1027C80000F08480009B33B9444B454F93F8008058
:1027D800FFF796FC08E0434B434F93F8008008F15D
:1027E800010202F01F021A700DF10F00FFF770FFCF
:1027F800002C44D1BDF80A3069B240F6B83212EA6A
:10280800210238BF4FF47A72D2180E2303FB08F363
:10281800ADF80A20FA529DF80F9022464946012049
:10282800FE18FFF719FD4946F07022460220FFF70F
:1028380013FD86F8029030719DF80E9022464946A5
:102848000420FFF709FD4946B0718246224603205D
:10285800FFF702FD05F07F0570713572BAF1000FC0
:1028680000D128B1214B1B7813B99DF80D3000E039
:102878000023F37186F809B0019AB2721CE0012CAA
:102888001AD10E2303FB08F3BDF80A202046FA529A
:102898009DF80F6000223146FD18FFF7DDFC314638
:1028A800E87000220220FFF7D7FC00232871AE70E1
:1028B800AB716B71EB71AB720E2303FB0877FC7283
:1028C800009B0120BB8102E0002000E0204605B00B
:1028D800BDE8F08F40320020D84200208814002044
:1028E800C0120020F3100020F81000203A18002031
:1028F80073B5154B04461B780E46D3B113482146D1
:102908001FF00DFF0546A0B9012E04F1010606D1FE
:102918002046FFF72DFC00950246812005E0204661
:10292800FFF726FC00950246982031462B46FFF714
:10293800E3FE214605481FF0DCFE0548214602B0AB
:10294800BDE870401FF0E0BE891400200417002085
:10295800181500202DE9F7437B4B04461B7843B13B
:102968007A4B1B7803F02403042B02D1002900F0D2
:10297800E880774B774F1B78002B00F0C7807648AC
:1029880021461FF0CCFE002840F0C08007F5C47037
:1029980021461FF0C4FE8046002840F0B7803B194E
:1029A80093F880302D2B01D0532B3AD16B4E3578CC
:1029B80045B30EF0ADFD04F10108054650B12046BF
:1029C800FFF7D6FB337802461E3300939320414627
:1029D800002307E02046FFF7CBFB0095024641465F
:1029E80093202B46FFF788FE0EF092FD014628B192
:1029F800337803201E330093002101E00090032068
:102A08000A4680E02046FFF7B3FB611C02462B46CE
:102A180093200095FFF770FE0095032029462A466B
:102A280071E0542B09D12046FFF7A2FBCDF80080B6
:102A38000246611C9420434666E0462B474D20D150
:102A48002E78BEB10EF064FD04F10109064648B1C6
:102A58002046FFF78DFB2B7802461E3300939A2001
:102A6800494622E02046FFF783FB00960246494686
:102A78009A2025E02046FFF77BFB009602469A2025
:102A880039E02E78002E2CD00EF042FD04F11C09FE
:102A9800064660B12046FFF76BFB2B7802461E33D3
:102AA80069F07F000093C0B2611C434609E02046EC
:102AB800FFF75EFB024669F07F000096C0B2611C1A
:102AC8003346FFF719FE0EF023FD21B2024628B166
:102AD8002B7803201E330093002214E0009003207B
:102AE80011E02046FFF744FB024604F11C0060F0A9
:102AF8007F000096C0B2611C3346FFF7FDFD0096CB
:102B08000320214632460123FFF7F6FD12482146ED
:102B18003F191FF0EEFD97F880302D2B0AD0532B6C
:102B280008D0542B06D0462B04D00D4821461FF060
:102B3800F6FD30B10B48214603B0BDE8F0431FF065
:102B4800E3BD03B0BDE8F083F6100020F2160020C4
:102B58008914002068240020041700205C17002036
:102B6800F0250020FC160020002302780E2101FB2E
:102B78000232044901338A180021062B9170F4D1DE
:102B8800704700BFC0120020064B00201870064B8B
:102B98001A78064B1B789A4202D00146FFF7C8BB49
:102BA800FF207047F4100020881400200B15002027
:102BB8000121814038B5114BC9431A78104BC9B26D
:102BC80002F0030203F5E074012A04D1DD7801EA7A
:102BD8000505DD7005E0022A03D11D7901EA050526
:102BE8001D710E33A342EFD1FFF7FCFC4FF4745074
:102BF8000EF016F9034B187038BD00BFD33600200D
:102C0800C01200208A1400202DE9F743A34D8DF847
:102C180007002B78A24C1BB12378C2B29A4204D089
:102C28004FF474500EF0FCF828709DF807302370AC
:102C38009C4C2278072A00F22D81DFE812F0080068
:102C48002400360054005D0072008D00BA00964AD8
:102C58003C211170954A1946107800F00300FFF7DF
:102C680067FB934BFF28187000F036811EF058FA66
:102C7800904B002093F8742042F0010283F87420EE
:102C88008D4B187064E0884B1B78002B00F0248172
:102C98001EF00EFC012840F04D81237814220133E8
:102CA8002370864B01381A7047E17F4B1B78002B45
:102CB80000F01281814E307808B901234AE01EF0F5
:102CC800F7FB022804D01EF0F3FB032840F0328102
:102CD8001EF026FA23780422013323701D23337053
:102CE800774B1A7026E1704B3C221A707548FFF733
:102CF8007BFB2378013323706B4B1B78002B00F090
:102D0800EB806E4B1D78002D40F014811020FFF7EA
:102D18003DFC002800F011812378284601332370F8
:102D28000BE1614B1B78002B00F0D68005F09EFC70
:102D3800002800F00281614B7D221A705E4B002052
:102D480018705C4B93F8742042F0010283F87420E9
:102D5800237801332370F0E0534B1B78002B00F0ED
:102D6800BB801EF0A5FB0128544E03D01EF0A0FB2B
:102D780003280FD19DF80720012111FA02F2524BC6
:102D8800197821EA02021A70642333702378013318
:102D98002370CFE03078002840F0CC80484A0323E5
:102DA80023701378013BDBB21370002B00F0948082
:102DB800C3E0404A414E92F86A201AB13278002A9C
:102DC80040F0B88000223270013212FA03F3DFF8C3
:102DD800E0803E4F98F800104FF00E0909FB017291
:102DE800DB4392F803E0DBB203EA0E0E907882F838
:102DF80003E092F804E003EA0E0E0340937082F8B1
:102E080004E00DF10700FFF733FC98F8003009FBE8
:102E18000372D278DFF894902AB999F8002002F06A
:102E28000302012A0AD00E2202FB03721279B2B9F8
:102E380099F8002002F00302022A10D10E2202FBA8
:102E48000377BA785AB9224F3A789A4207D1184884
:102E5800FFF78AFE3B78013303F01F033B7099F8B4
:102E680000009DF8071000F00300FFF761FA144B0B
:102E78000422FF281A7088F80000164B42D0987870
:102E880000F04000C0B200283CD1032323701A335D
:102E9800337052E0002020704FE000BF8A140020F9
:102EA800F7100020F410002082140020D3360020F0
:102EB800BE12002058360020F5100020F210002025
:102EC800801400208B14002081140020C0120020E0
:102ED8000B15002040320020FFF73EFB0023237033
:102EE8001EF01EF92B78013BDBB22B702BB1144B73
:102EF8009B7803F04003DBB2F3B19DF80700FFF7BE
:102F080057FE19E09B780E4A03F04003DBB22BB161
:102F1800136843F400031360FFF7D2F8FFF71CFBB4
:102F28001EF0FEF8002323704FF474500DF078FF64
:102F3800287001E0002000E0FF20BDE8FE8300BF0C
:102F480040320020044B1A780AB1013A1A701B78F3
:102F58000BB9FFF72DBE70478A140020044A054BB1
:102F680010781B7803EA501000F00100704700BF8A
:102F780040320020CB160020044B054A1B781078FD
:102F8800C3F3400303EA1010704700BFCB160020BC
:102F980040320020034B044A1B78D078C3F38003E7
:102FA80018407047CB16002040320020044B054AD9
:102FB8001B78D078C3F3C00303EA5000704700BF02
:102FC800CB16002040320020044B054A1B78D078ED
:102FD800C3F3001303EA9000704700BFCB1600202C
:102FE80040320020044B1878044BDB785B005BB25E
:102FF800DB1103EAD0107047CB16002040320020C6
:103008002DE9F041154E0024B04620E0204629461F
:103018001BF000F890B1F35DFF2B0FD04FF4A073B5
:1030280063430A2202FB053318F80330DB0905D095
:103038000B4B1878C0F30010BDE8F08101350A3752
:10304800202DE3D10134022C06F5A07602D000270A
:103058003D46DBE70020BDE8F08100BFA537002032
:10306800CB16002008B51AF0D7FB034B1B7800EAF3
:10307800931000F0010008BDCB160020044B054A50
:103088001B78D078C3F3401303EAD000704700BF21
:10309800CB160020403200202DE9F84FFFF75EFFE5
:1030A8008146FFF769FF8246FFF774FF8346FFF703
:1030B8007DFF8046FFF788FF0446FFF7A1FF05461E
:1030C800FFF7DCFF0746FFF7CDFF0646FFF78AFF4D
:1030D8004FEA8B0343EA4A0343EA090343EAC80376
:1030E80043EA471343EA861345EA040443EAC01354
:1030F800E0B243EA0010BDE8F88F0000044B98786E
:1031080000F00F00A0F10203584240EB03007047A3
:1031180069150020044B987800F00F00A0F1010217
:10312800504240EB0200704769150020044B987824
:1031380000F00F00A0F10301484240EB0100704786
:1031480069150020054B987800F00F00A0F1060CD7
:10315800DCF1000040EB0C00704700BF691500204F
:10316800514AF0B513781446012B29D003D3022B0A
:1031780040F098805EE04D484D4B047819786FF325
:10318800C304047001F0F80158786FF3C301197093
:1031980000F08001C9B2002900F08480012111707B
:1031A8009C78062204F00F04544302464148005D0F
:1031B80060F306025A701A7861F302021A70F0BDC1
:1031C8003B494D780B4625F07F00002838D00A7817
:1031D80002F00802D2B222B9344A117841F008014B
:1031E80011709A7802F00F02012A04D12F4A11783F
:1031F80041F00101117015F07F0F53D119789E78B5
:1032080001F00700062206F00F0602FB0606294F0A
:103218005D78BE5D013066F3060500F007005D705D
:1032280090FBF2F502FB150262F30201197002230A
:103238002370F0BD1E494D780B4625F07F0028B954
:103248008B7860F303038B701070F0BD174A117808
:103258006FF3C3011170997801F00F01012903D1AF
:1032680011786FF30001117015F07F0F1AD11978DA
:103278009E7801F00700062206F00F0602FB0606FC
:103288000C4F5D78BE5D013066F3060500F007005F
:103298005D7090FBF2F502FB150262F302011970F2
:1032A80001232370F0BD00BFB815002017150020BA
:1032B800691500207C41020810B51F4A1F4B92F97E
:1032C800031009B1002231E008B1032119701978FF
:1032D800032930D8DFE801F00209192C11780029F8
:1032E80029D0154881700121197092F902001249FC
:1032F80020B1134B1A786FF3861217E0487808B993
:10330800032213E088700221197092F902100A480A
:1033180089B90B4A147861F386141470026861F352
:103328000F22D1B261F31742026001221A7010BD58
:1033380000211160197010BD6017002015150020BC
:103348003835002038B5044643F6EF2343F6F0201D
:10335800012A08BF18460D460DF062FD2378C0B259
:103368001842104C09D043F6EE200DF059FD2368A1
:1033780060F307036FF30F230CE02B7818420AD091
:1033880043F6EE200DF04CFD2368C0B260F307034E
:1033980060F30F23236094F9003013B1014B0F221F
:1033A800DA7038BD6017002008B543F6F7200DF035
:1033B80037FD014B187008BD16150020014B187019
:1033C800704700BFD4160020024B1A5C6FF303024B
:1033D8001A5470471216002070B50C46C10001F54A
:1033E800CE411B488B3108220DF02BFD00251848D3
:1033F8002946EEB21FF093F908B9237823BB154B81
:103408002278EB5C1A421FD13046FFF7DDFFF60841
:103418004AF2B34030180DF003FD05F00703C0B2BF
:10342800184110F0010F0FD10B4829461FF077F90A
:1034380050B1294608481FF067F9074B06F5CC40FC
:10344800CA30995D0DF0E2FC0135402DCFD170BD39
:10345800D6160020C91500206C15002038B546F294
:10346800127540242046FFF7AFFFA5F5CC43094A63
:10347800D23BD15C11F0100F06D06FF30411D15478
:10348800284600210DF0C2FC0134E4B20135B92C04
:10349800E8D138BD121600203F287FB5054607D869
:1034A80000F5E2400D300DF0BBFCC3B22BB930E1A2
:1034B8009C4A1478002C00F031819B4E725D02F01A
:1034C8000F014C1C04F00F0464F303023F2D7255E6
:1034D80033D8002C00F0228101339C4240F01B813C
:1034E800924B5A1992F88020522A725D03D161F3E7
:1034F800030272550FE16FF30302EC081B197255B2
:1035080093F8902105F0070352FA03F313F0010F23
:1035180040F00381294686481FF0EBF8844B04F5F8
:10352800CC40195DCA3001240DF070FC2D1902231E
:1035380000930194029518209EE0002C00F0EE8084
:10354800784B1B7801339C4240F0E580735D05F5AC
:10355800CC406FF30303D230012173550DF056FCB4
:10356800735D43F010037355A5F14003DBB2072BDD
:1035780007D80422009201330232019202931920E3
:10358800B3E0A5F14803DBB2072B07D80422009269
:1035980001330332019202931A2061E0A5F150032E
:1035A800DBB2062B07D804220092013303320192C2
:1035B80002931B2054E0A5F15703DBB2032B07D875
:1035C800042200920133033201920293212047E042
:1035D800A5F15B03DBB2012B07D80422009201336B
:1035E80002320192029322207FE05D2D06D104234E
:1035F80000930193043B0293284684E05E2D07D193
:103608000423009301330193053B02935E207AE083
:10361800A5F15F03DBB23F2B09D8042200920133E6
:1036280092180192029333200121053A6DE005F1C9
:103638006103DBB2072B07D804220092013303325F
:10364800019202935F200BE005F15903DBB2012BD5
:1036580009D80422009201330332019202936020B8
:103668000121043A51E0AA2D0CD10423009301242E
:10367800043B0194029361202146032223460DF066
:103688004DFC4BE0A92D07D104230093023B019385
:10369800023B0293622036E0AD2D08D1042300934B
:1036A8000322043B01920293632001212DE0AB2DFC
:1036B80006D104230093043B01930293642022E083
:1036C800AC2D06D104230093043B01930293702090
:1036D80019E005F15203DBB2032B09D8042200924A
:1036E800013302320192029368200121033A0CE06F
:1036F8004E35EDB2062D10D8042300930135023360
:10370800019302956A20012103220B460DF006FC65
:1037180003E01C4602E0002400E00124204604B037
:1037280070BD00BF00000020121600206824002091
:103738006C150020024B185CC0F30010704700BFE6
:1037480012160020F8B508220E4600210746FCF79D
:1037580021FE46F28B7500243378234113F0010FC4
:1037680008D02946064808220DF06BFB3846044964
:103778001EF08DFF01340835082CEDD1F8BD00BFCF
:10378800E0160020024846F2CA6108220DF059BB33
:103798006C15002070B5044600F56A5044300DF0F1
:1037A8003FFB0B4D06462B7813F0010F02D1CC20BE
:1037B8001FF0A2FD2B8843F001032B80054B1E55FB
:1037C800054B13F8242042F0010203F8242070BDB1
:1037D800F21600204915002028150020024B185C1D
:1037E800084100F001007047C915002070B5054672
:1037F8000024094BE0B2E618E35C4BB12946FFF719
:10380800EDFF28B100233370044821461EF07CFFE9
:103818000134402CEDD170BD14170020591500203B
:1038280038B5054600242846E1B2FFF7D7FF10B1A6
:10383800044BE35C23B90134082CF4D1002038BDD3
:10384800012038BD4915002038B505460DF060FE49
:10385800A0B100242846E1B2FFF7C0FF40B1084BF1
:1038680013F8243013F0010F02D0064BE35C23B1A8
:103878000134082CEED1002038BD012038BD00BF2E
:103888002815002049150020F8B5114800214022CC
:10389800FCF780FD46F28B75002401270D48294668
:1038A8000822A7400DF0CDFAFFB20026094831469C
:1038B8001EF035FF20B1064BF25C47EA0202F254D3
:1038C8000136402EF2D101340835082CE5D1F8BD77
:1038D800C9150020E01600202DE9FF4100263446D6
:1038E800B0461A4B1B78234113F00102184B23D022
:1038F800184F1D5D17F82430A84538BFA84613F0A7
:10390800010F1AD0CDB965F3000307F8243023B2AC
:103918000122F71902935B2029462B460092019554
:103928000DF0FCFA7B78B878F9781843621C2B46BE
:103938000095FEF7E1FE00E01A5501340436082C24
:10394800CFD1054B83F80080BDE8FF811615002014
:1039580049150020281500201415002010B50C4B1F
:103968001B78A3B10B4B1B788BB100240A48214666
:103978001EF0D5FE40B1094821461EF0D0FE18B908
:1039880020460121FEF7E6FF0134402CEED110BDA0
:1039980089140020F6100020FC160020CE1E0020FE
:1039A8002DE9F043324C334A238800266FF38613FF
:1039B8006FF3C4032380304B304F85B016701E70F0
:1039C8009146984617F8013B5BB32278D20052B271
:1039D80043EAA2122388402E62F3C40343F0400353
:1039E80023801ED000253046E9B2FFF7F7FEA8B1C4
:1039F80017F8013C13F0010F06D00122AA4099F8EC
:103A080000100A4389F8002013F0020F06D00123A2
:103A1800AB4098F80020134388F800300135082D92
:103A2800E1D10136F6B2412ECCD1237803F040051E
:103A3800EDB2D5B903F02403042B0BD1FFF78EFFA9
:103A4800FF2300934020294601222B460195029529
:103A58000DF064FA238800226FF345136FF3820395
:103A68006FF3C4032380064B1A7005B0BDE8F083DA
:103A7800F21600208C340020BC340020771500207A
:103A8800D516002010B50024054821461EF047FE33
:103A980008B9044BE0540134402CF5D110BD00BFE7
:103AA800CC1600207715002010B5127804469DF832
:103AB8000810DAB1D3B111B10D491EF0DDFDACB17A
:103AC800082246F2CA610B480DF0BBF921460948A5
:103AD8001EF0DDFD0749082246F2CA600DF0ABF979
:103AE80005480449BDE810401EF0E7BD10BD00BF01
:103AF800002600200C1500206C15002030B5064B60
:103B080004781D7824EA05040C7001781B7823EAF0
:103B18000103137030BD00BF1615002038B50A4DDB
:103B2800002415F8013F2D2B09D0532B07D0542B17
:103B380005D0462B03D0054821461EF0E5FD01348B
:103B4800402CEED138BD00BFE7240020FC16002031
:103B580010B50F481EF088FD00240E4821461EF0BF
:103B6800DEFD80B10C4BE31893F88030482B06D06B
:103B780003D82D2B03D0462B00E0542B03D1044847
:103B880021461EF0B6FD0134402CE6D110BD00BF21
:103B9800B9150020FC16002068240020094A0A4BA9
:103BA800117831B1997801F00F01814201D00021DB
:103BB80011709A7860F303029A705A7842F0800282
:103BC8005A707047B8150020691500207FB55F4B03
:103BD800154604461A780E4600235D4911F823104D
:103BE80011F0010F03D00121994022EA01020133AB
:103BF800082BF2D1574B1A70002C6FD014F0010F1C
:103C08000AD0FF2301210093FF3B01930293522026
:103C18000A460B460DF082F914F0020F0AD0FF2372
:103C280001210093FF3B0193029353200A460B4660
:103C38000DF074F914F0040F0AD0FF23012100934A
:103C4800FF3B0193029354200A460B460DF066F998
:103C580014F0080F0AD0FF2301210093FF3B0193C2
:103C6800029355200A460B460DF058F914F0100F30
:103C78000AD0FF2301210093FF3B019302935620B2
:103C88000A460B460DF04AF914F0200F0AD0FF231C
:103C980001210093FF3B0193029357200A460B46EC
:103CA8000DF03CF914F0400F0AD0FF2301210093D6
:103CB800FF3B0193029358200A460B460DF02EF95C
:103CC80014F0800F0AD0FF2301210093FF3B0193DA
:103CD800029359200A460B460DF020F9CEB1002474
:103CE800284621461EF01BFD60B1FF230093FF3BD1
:103CF8000193631C1BB2012102935A200A460B460A
:103D08000DF00CF92146284601341EF0FDFC402C2C
:103D1800E6D110481049114AFFF7F0FE104B002277
:103D28001A700132009206320192F83202920A4960
:103D38000A4A08480AF00CFC0A4B3C2251201A7027
:103D480004B0BDE870400DF0C9BC00BF16150020D6
:103D580028150020C0180020961900208A19002074
:103D6800851800204815002010B5FFF795F904467E
:103D780007481EF0A7FCD0F1010138BF002104B9A3
:103D880029B1034A2046BDE81040FFF71FBF10BD08
:103D98000A160020054B03EBD00393F8903100F08E
:103DA800070053FA00F000F0010070476824002073
:103DB80010B50F4B04461B7813F0010315D0FFF71D
:103DC8002FFD28B90B4B1B1993F88030462B0DD1CA
:103DD8000DF09EFB18B92046FFF7DCFF30B106480E
:103DE80021461EF086FC012010BD184610BD00BFFC
:103DF800F2160020682400200A160020024B1878CA
:103E0800003818BF012070474815002010B5034C32
:103E180004EB830358709970DA7010BD28150020E0
:103E280010B500240948002100190E220E34FCF7B1
:103E3800B1FAB4F5E07FF5D1054A00231370054ABD
:103E4800002199520233AA2BF9D110BDF810002095
:103E5800F31000200A1A00207FB5474B04461B7850
:103E68000E46AA2B78D0454821461EF058FC054638
:103E7800002871D12046FFF79BFF00286DD14048EC
:103E880021461EF04CFC50B93E4821461EF047FC26
:103E9800054620B92046FFF7FFFA00285DD13A4BC6
:103EA8001B7823B9394B1B7813F0010F09D1384B14
:103EB800DB7803F02003DBB21BB9364B032283F80F
:103EC8004020012E05D82E4821461EF028FC40B17E
:103ED80042E0022E07D12B4821461EF020FC10B1EB
:103EE8003AE0274800E0274821461EF002FC2A480D
:103EF80021461EF009FC022E15D101252946032270
:103F08002B4600964A206619019502960DF006F890
:103F18002046FEF72DF9002302463146182000936B
:103F2800FEF7EAFB19E0012E09D102230093631C76
:103F380002930196122031460322334609E07EB9E6
:103F48000121022300936318029301911120032297
:103F58000B460CF0E3FF03E00025284604B070BDD3
:103F68002046FEF705F90246012000232118009398
:103F78000125FEF7C1FBF0E7D41600206C150020E0
:103F8800181500205417002016150020061A0020C6
:103F98004032002077150020041700202DE9FF4744
:103FA80004460D46754821461EF0B9FB8146002897
:103FB80040F0DF80214671481EF09BFB7048214687
:103FC8001EF0A2FB6F4E0DBB01274FF00208E3194C
:103FD80002934246032039463B46CDF800800197BC
:103FE8000CF09CFF327862B10DF092FA024630B1C3
:103FF800337840461E33009321462A4604E0009059
:1040080000E00092404621463B4628E0012D2BD196
:104018005D4B04F5E2400D301F5D0CF001FF07F029
:104028000F07874209DA631C022202930E202946F1
:104038002B46009201950CF071FF327892B10DF089
:1040480067FA024638B14F4B0D201B7821461E33C4
:104058000093002202E000900D2021460123FEF784
:104068004BFB5EE00092F7E7022D0BD10123019391
:10407800E3180293142049462A464B4600950CF053
:104088004DFF4EE0032D4CD101272A464FF0020880
:1040980004EB070A4D2039463B46CDF800800197CE
:1040A800CDF808A00CF03AFF35783DB30DF030FAA2
:1040B800024630B1337840461E33009321464A46C3
:1040C80002E00090214640463B46FEF715FB0DF006
:1040D8001FFA671C054648B12046FEF749F83378B1
:1040E80002461E3300931A2039462CE02046FEF77C
:1040F8003FF80095024639461A202DE021462A4607
:104108003B4640460095FEF7F7FA2046FEF730F8A2
:10411800514602462B461A200095FEF7EDFA38461E
:1041280028E03578EDB10DF0F3F904F11C060546E9
:1041380058B12046FEF71CF8124B02461B78304651
:104148001E330093611C002307E02046FEF710F899
:10415800009502463046611C2B46FEF7CDFA012039
:1041680008E02046FEF704F80095024604F11C001A
:10417800F1E7002004B0BDE8F08700BFFC1600207E
:10418800041700205C17002012160020064B1B188D
:1041980093F84001492804D0452814BF0320022081
:1041A80070470120704700BF682400202DE9F041C6
:1041B800244F00243C70244821461EF0B0FAE5B292
:1041C800224B002837D01E5D3B789E4200D303B9AE
:1041D8003E70002E30D131461C484022FCF7DAF8F8
:1041E8001B4B1C4803EBD50393F8888104F00703A5
:1041F80048FA03F8214608F001081EF090FA68B959
:10420800B8F1000F02D02846022101E028463146C5
:10421800FFF7C4FE28460DF061FA0DE0B8F1000F73
:104228000AD12846FFF7B2FF0B4BDB7803F02003D7
:10423800DBB20BB9094B18550134402CBBD1BDE892
:10424800F08100BF5C1700205915002014170020CA
:1042580068240020FC16002040320020771500203A
:104268002DE9F04F914B89B01B7813F0010F06D060
:104278008F4B1A786FF386121A7001F09BBA8D492A
:104288008D4A0B7810788D4D984218BF8C49137061
:1042980018BF0B706B7803F00803DBB24BB143F621
:1042A800CF200CF0BDFD864B18702B886FF3CB2305
:1042B8002B80844B1B78AA2B08D18349AA3B0B700F
:1042C8002B8843F080032B8000F0A8BE6A787B4BD4
:1042D80002F01002D2B27D4CA2B11A886FF30C32F0
:1042E8001A807B4B1B7823B97A4B1B7813F0010F8C
:1042F80008D1E37803F02003DBB21BB9764B032225
:1043080083F840202368754F6FF3186323603A7869
:1043180002F00202D2B232B96B494A781AB16B4A3A
:1043280043F080731360E67816F0010648D05D20EC
:10433800FFF700FA00285AD16B78DFF8808103F084
:104348000203DBB22BBB5D30FFF7A6F8064600BBC5
:10435800B8F80030012143F40073A8F800300423B2
:1043680003220093019302900B460D200CF0D6FD1A
:1043780045200DF0B3F93146012233460D20009651
:10438800FEF7BAF909203146324601230096FEF7B6
:10439800B3F96B7803F00203DBB243B34C4B1B78E1
:1043A80023B94C4B1B7813F0010F20D1E37803F0AD
:1043B8002003DBB2DBB9484B032283F8402016E028
:1043C8006B7803F00203DBB26BB13146324601234E
:1043D8000A200096FEF790F98D20314601223346D7
:1043E8000096FEF789F92B886FF349232B80236801
:1043F800354A6FF35963236093787BB1D37823B937
:104408003B7813F00C0F05D108E03B7803F00C0360
:10441800042B03D0236843F000732360E17801F094
:104428000201C9B200295BD05E20FFF783F900289A
:1044380065D16B78214F03F00403DBB2EBB95E3032
:10444800FFF72AF80646C0B93B88012143F4806388
:104458003B800423009301330322019302900B460F
:1044680017200CF05BFD45200DF038F90D20314682
:10447800012233460096FEF73FF96B7803F00403F8
:10448800DBB2002B3BD0124B1B7823B9114B1B78A6
:1044980013F0010F33D1E37803F02003DBB273BBD1
:1044A8000D4B032283F8402029E000BFC1180020EB
:1044B80038350020DE160020DF160020F216002016
:1044C8005D170020D4160020280E0020403200205E
:1044D80016150020061A00207715002066240020F3
:1044E8006B7803F00403DBB22BB18D2001220B465D
:1044F8000091FEF701F92B886FF38A232B8023683C
:10450800DFF8DCB26FF3DF7323605F2306930026C6
:10451800D94696E03046394619F07CFD002871D01E
:104528001BF80A30FF2B6DD04FF4A0727243A8F12C
:104538005E03DBB207930A2303FB072219F802E0A4
:1045480009EB02035FEADE1E50D02268404642F0C3
:10455800004222600593FFF7EDF8059B00285CD127
:104568001A7912F0040F24D14046FEF795FF059BF7
:104578008446F0B91A79322042F004021A71079978
:10458800042300930291DB180121032201930B46B7
:10459800CDF814C00CF0C2FC4A200DF09FF8DDF8ED
:1045A80014C00C20079901226346CDF800C0FEF71D
:1045B800A3F84FF4A07373430A2202FB07334B445A
:1045C8001B7913F0040F28D0804B1B7823B9804B3C
:1045D8001B7813F0010F20D1E37803F02003DBB23E
:1045E800DBB97C4B032283F8402016E01B7913F0DB
:1045F800040F07D08C20079901227346CDF800E0FC
:10460800FEF77AF84FF4A07373430A2202FB0733CC
:104618004B441A796FF382021A71013708F10108C5
:10462800202F5FFA88F80AF10A0A7FF473AF069A16
:10463800013602F12003DBB2022E0BF5A07B0693B4
:1046480005D04FF0000ADDF81880574662E7236866
:10465800614923F080636FF39E7323600B79002B0D
:1046680000F049845D4ADFF87CB106924FF09F085C
:1046780000271BF8011F3E460137002952D0236846
:10468800A8F15F0A43F080635FFA8AFA2360504614
:10469800FFF750F800285CD117237343DFF84891DF
:1046A80019F8032012F0100F23D150460593FEF796
:1046B800F3FE059B8246E0B919F80320012142F078
:1046C800100209F8032004230093023301933BB23C
:1046D800032202930F200B460CF020FC45200CF01F
:1046E800FDFF0D20514601225346CDF800A0FEF7EC
:1046F80003F81723734319F8033013F0100F28D069
:10470800324B1B7823B9324B1B7813F0010F20D1A1
:10471800E37803F02003DBB2DBB92E4B032283F8E6
:10472800402016E017237343DFF8BC9019F80330D4
:1047380013F0100F05D08D2001220B460091FDF7D4
:10474800DBFF1723734319F803206FF3041209F8EA
:104758000320069A12F8011F0692002946D0236802
:10476800404643F080432360FEF7E4FF002854D11D
:104778004FF0170909FB06F9DFF86CA01AF80930A1
:1047880013F0200F49D14046FEF786FE0646002862
:1047980043D11AF80930012143F020030AF80930FF
:1047A80004230093033301933BB2032202934B206B
:1047B8000B460CF0B3FB50200CF090FF192031464B
:1047C800012233460096FDF797FF26E016150020D4
:1047D800061A002077150020280E002094330020A8
:1047E800A5370020C0330020CF33002017237343A0
:1047F800DFF8989219F8033013F0200F05D09920AC
:1048080001220B460091FDF777FF17235E4319F845
:1048180006306FF3451309F8063008F10108082F30
:104828005FFA88F87FF425AF934ADFF864B20692FE
:104838004FF05008083F1BF8011F3E46013700297A
:1048480050D0236808F1620A43F080635FFA8AFA5D
:1048580023605046FEF76EFF002858D1DFF83492E7
:10486800330119F8032012F0400F23D15046059365
:10487800FEF712FE059B8246E0B919F803200121D4
:1048880042F0400209F80320042300930233019305
:104898003BB20322029369200B460CF03FFB4520F4
:1048A8000CF01CFF0D20514601225346CDF800A004
:1048B800FDF722FF330119F8033013F0400F26D01B
:1048C8006E4B1B7823B96E4B1B7813F0010F1ED16A
:1048D800E37803F02003DBB2CBB96A4B032283F8F9
:1048E800402014E0DFF8AC91330119F8033013F0DD
:1048F800400F05D08D2001220B460091FDF7FCFEEC
:10490800330119F803206FF3861209F80320069A79
:1049180012F8011F0692002933D02368404643F05D
:1049280080432360FEF706FF00283FD1DFF864A12B
:104938004FEA06191AF8093013F0200F36D140460D
:10494800FEF7AAFD064688BB1AF80930012143F094
:1049580020030AF8093004230093033301933BB280
:104968000322029310200B460CF0D8FA50200CF0CA
:10497800B5FE19203146012233460096FDF7BCFEEC
:1049880014E0DFF81091330119F8033013F0200F09
:1049980005D0992001220B460091FDF7ADFE3601A6
:1049A80019F806306FF3451309F8063008F10108C5
:1049B800072F5FFA88F87FF43EAF334ADFF8D8B0A4
:1049C80006924FF05708073F1BF8011F3E46013774
:1049D800002965D0236808F1570A43F080635FFA1D
:1049E8008AFA23605046FEF7A5FE00286DD1DFF84D
:1049F800AC90330119F8032012F0400F23D1504630
:104A08000593FEF749FD059B8246E0B919F8032096
:104A1800012142F0400209F80320042300930233E5
:104A280001933BB20322029367200B460CF076FAFF
:104A380045200CF053FE0D20514601225346CDF877
:104A480000A0FDF759FE330119F8033013F0400FA9
:104A58003BD00A4B1B7823B9094B1B7813F0010F85
:104A680033D1E37803F02003DBB273BB054B032299
:104A780083F8402029E000BF4332002016150020AB
:104A8800061A0020771500208F320020CF3300202F
:104A98007A3300200B33002083320020AC32002010
:104AA800DFF85893330119F8033013F0400F05D09D
:104AB8008D2001220B460091FDF71EFE330119F8E7
:104AC80003206FF3861209F80320069A12F8011FD3
:104AD8000692002933D02368404643F08043236080
:104AE800FEF728FE00283FD1DFF810A34FEA061989
:104AF8001AF8093013F0200F36D14046FEF7CCFCE7
:104B0800064688BB1AF80930012143F020030AF849
:104B1800093004230093033301933BB20322029329
:104B28001F200B460CF0FAF950200CF0D7FD192085
:104B38003146012233460096FDF7DEFD14E0DFF82A
:104B4800BC92330119F8033013F0200F05D09920D7
:104B580001220B460091FDF7CFFD360119F806300A
:104B68006FF3451309F8063008F10108042F5FFABE
:104B780088F87FF429AF4FF000094FF0A70AC8461C
:104B88004E46954B08F10108F15C00294ED0236888
:104B9800AAF14C0B43F080635FFA8BFB2360584605
:104BA800FEF7C8FD002854D1182373438B4FFA5CD5
:104BB80012F0200F22D158460593FEF76DFC059B95
:104BC8008346D8B9FA5C012142F02002FA54042342
:104BD8000093023301930FFA88F3032202932020F3
:104BE8000B460CF09BF945200CF078FD0D2059463A
:104BF80001225B46CDF800B0FDF77EFD1823734314
:104C0800FB5C13F0200F24D0754B1B7823B9754B30
:104C18001B7813F0010F1CD1E37803F02003DBB2FB
:104C2800BBB9714B032283F8402012E01823734369
:104C38006A4FFB5C13F0200F05D08D2001220B4634
:104C48000091FDF759FD18237343FA5C6FF3451281
:104C5800FA54664BF15C002936D02368504643F07D
:104C680080432360FEF766FD002842D15B4B4FF07E
:104C7800180B0BFB063B9BF8013013F0200F38D1C3
:104C88005046FEF709FC0746002832D19BF8013050
:104C9800012143F020038BF80130042300930333F0
:104CA80001930FFA88F3032202934C200B460CF071
:104CB80035F950200CF012FD1920394601223B46E7
:104CC8000097FDF719FD14E0444F182303FB067302
:104CD8005B7813F0200F05D0992001220B46009134
:104CE800FDF70AFD182303FB06777B786FF345135E
:104CF8007B703F4B1B78002B00F094803D4B374F67
:104D0800F35C1822002B7BD002FB06F3FA5C07EB5E
:104D18000901C2F3801BBBF1000F1BD142F0400216
:104D2800FA54782204234A800093DB180121019366
:104D38000FFA88F3032202932E200B460CF0EEF8AC
:104D480046200CF0CBFCCDF800B0092041460122EA
:104D58005B4665E0B1F9021029BB5FEAD21B22D19C
:104D680043F6DE2005930CF05BF8059BD8B1FA5C9E
:104D7800012142F08002FA5404230093DB180193C6
:104D88000FFA88F3032202932F200B460CF0C6F883
:104D980047200CF0A3FC0920414601225B46CDF8D0
:104DA80000B0FDF7A9FC18237343FB5CDB0939D07D
:104DB8000B4B1B7823B90B4B1B7813F0010F31D128
:104DC8000D4BDB7803F02003DBB25BBB064B032201
:104DD80083F8402026E000BF9233002054320020A0
:104DE80016150020061A00207715002083330020AE
:104DF800A03200209532002040320020AC32002042
:104E08007243B95C11F0400F0CD063F3861163F361
:104E1800C711B9544F447B80892000934146012231
:104E2800FDF76AFC01360AF1010A022E09F1180998
:104E38005FFA8AFA7FF4A5AEDFF8F8A34827023EA6
:104E48001AF8011FB0460136002937D023683846C2
:104E580043F080432360FEF76DFC002847D14FF0F4
:104E68001D0909FB08F9DFF8BCB31BF8093013F07A
:104E7800200F3CD13846FEF70FFB8046002836D17C
:104E88001BF80930012143F020030BF809300423F3
:104E980000930333019333B20322029313200B468A
:104EA8000CF03CF850200CF019FC19204146012266
:104EB8004346CDF80080FDF71FFC18E01D2303FBD7
:104EC80008F3DFF8609319F8033013F0200F05D0CA
:104ED800992001220B460091FDF70EFC1D2303FBD0
:104EE80008F819F808306FF3451309F80830013746
:104EF800082EFFB2A4D1A37803F00803DBB2002B7D
:104F080040F08C8048F6F234A4F50A47A7F5F97703
:104F1800AF4839461DF003FC28B9AE4839461DF0A4
:104F2800FEFB002874D0AC4839461DF0F8FB002879
:104F38006ED13946A8481DF0DCFB20460BF070FF07
:104F4800A64EC0B23070002862D00138C0B23070AE
:104F58000BF07EF800285BD13078A14E00F56A503E
:104F680078300BF05DFF9F4BC0B214F803803070AF
:104F780000EA0808394696481DF0D1FBDFF8B8A2C8
:104F8800DFF8649238B1934839461DF0C8FB10B970
:104F98009AF8003014E08F4839461DF0C0FB38B14C
:104FA8008B4839461DF0BBFB10B99AF8003004E075
:104FB8009AF8003018EA030F02D023EA080801E043
:104FC80048EA03088848894989F80080884AFEF732
:104FD80095FD8648874912F017F968B10CF098FAE0
:104FE80050B9844809F01EFB30B901238148824931
:104FF8007E4A0093FEF758FD002300930133019386
:105008003378794802937949794A7B4B09F0A0FAB9
:10501800013448F632439C427FF476AF774E73787A
:105028006FF3C71373702B7803F08002D2B2002A93
:1050380000F00C8172490C78002C40F0078103F0D5
:105048002403042B0BD1FEF789FCFF230093402097
:10505800214601222346019402940BF05FFF2B881E
:1050680000246FF3C7136FF3820364F3451364F3EB
:10507800410364F30003634A64F3492364F38A2316
:1050880014702B80604B1A7842F0C0021A705A785C
:1050980064F3C3025A70FEF741FD5C481DF0E4FA60
:1050A8005B481DF0E1FA5B481DF0DEFA5A482146DC
:1050B8004122FBF76FF917236343584A0134D15C47
:1050C800082C01F0DF016FF30411D154F3D1002350
:1050D80053491A01885C013300F0DF006FF3861032
:1050E800072B8854F4D14F4B1A786FF345121A7076
:1050F8005A7F6FF345125A7793F83A206FF34512A7
:1051080083F83A2093F857206FF3451283F8572015
:1051180093F874206FF3451283F8742093F8912064
:105128006FF3451283F8912093F8AE206FF3451280
:1051380083F8AE2093F8CB206FF3451283F8CB2089
:10514800394B1A7802F0DF026FF386121A701A7C54
:1051580002F0DF026FF386121A7493F8202002F02F
:10516800DF026FF3861283F8202093F8302002F0D4
:10517800DF026FF3861283F830202C4B5A786FF3D6
:1051880045125A701A7802F07F026FF345121A70AE
:105198005A7E6FF345125A761A7E02F07F026FF339
:1051A80045121A76002311E04FF4A07159430A20E2
:1051B80000FB02111E48013241180879202A6FF3BA
:1051C80082000871F0D10133022B37D00022EBE7BF
:1051D8004C240020542400205C24002009160020C0
:1051E800561900203699FF1FC01800209619002074
:1051F8008A19002020150020851800206915002034
:10520800280E0020D516002038350020541700201D
:10521800181500205915002077150020CF330020DD
:105228000B33002057350020AC32002054320020C8
:10523800A5370020023300201615002008227248E6
:105248000021FBF7A7F8714B00221A70704C2378E5
:10525800002B48D129786F4A01F00201C9B2D9B1AF
:105268006D481188477863F34D3163F3C30741F004
:10527800800147701180CA201EF03EF8C6201EF03B
:105288003BF81EF087F8654A13780BB90CF0B2FAB0
:10529800FEF7E4F8FEF7C4FD614A2B8811786FF336
:1052A80041036FF300016FF3000311705D480021A3
:1052B80040222B80FBF76EF85B481DF0D5F95B4860
:1052C8001DF0D2F95A481DF0CFF95A481DF0D0F90F
:1052D80008224D480021FBF75DF84C4A0023137063
:1052E800554A13706AE02F7807F00203DBB293B9CE
:1052F80017F001070FD14C481DF0B6F92378F8B222
:105308003B4113F0010F03D0FEF744FA0CF0F6F816
:105318000137082FF2D12B783E4F13F0010F25D01B
:10532800FEF722FD3B8843F002033B80FEF7D4FAE8
:10533800364B93F80080B8F1000F14D1CA201DF045
:10534800DBFFCD201DF0D8FF3B883C4868F3000305
:105358003B80334B1A7842F001021A701DF084F931
:10536800FEF77CF802E00120FEF718FC2B7803F02A
:105378000202D2B212B3304A12782AB113F0010FE6
:1053880002D10220FEF70AFCFEF710FF2C4927483D
:105398001DF088F9254926481DF06EF9FEF7D8FB5F
:1053A800224928481DF068F9274926481DF06FF959
:1053B800FEF768FB1F481D491DF07FF92049234867
:1053C8001DF05AF915490B780BB9FEF7E9FA73780D
:1053D80003F08003DBB2002B40D12B7803F02403C9
:1053E800042B06D143F6EC200BF01AFD08B1062079
:1053F80032E0FEF703FD08B105202DE00CF0E4FAD9
:1054080030B3032028E000BF491500201415002000
:1054180016150020F216002038350020280E00202E
:105428001715002014170020AD290020CC160020E5
:10543800591500200C1700205C1700200A160020C0
:105448006C150020FC160020B9150020511500200D
:1054580001F074F810B10420FEF7A0FB694B1B782B
:105468001BB173786FF3C7137370674A137813B15E
:10547800664B1B78CBB12B78654E03F04403402B69
:1054880013D10021BF3300933F200B460222019124
:1054980002910BF043FD338843F6CE2043F004031A
:1054A80033800BF0BDFC5B4B187057495A4E0B7894
:1054B8009BB1564B197881B92A78554B02F04002B6
:1054C800D2B252B11A8861F382021A80337823B9B2
:1054D80043F6CE200BF0A4FC30702A78DFF8308138
:1054E80002F00400C0B24D4B00287AD002F0200030
:1054F800C0B2484F90B11A78002042F0C0021A702A
:10550800FDF7DAFE3B78002B71D1B8F8002063F381
:10551800820263F34512A8F8002068E0D20052B274
:1055280019789211D2B241F0C00112F0010F19702E
:1055380003D0C9B260F3C711197012F0020F03D07B
:105548001A786FF386121A701B78344A03F04003F6
:10555800DBB24BB9537843F00803537023781BB17F
:105568002B8843F400532B800120FDF7A5FE43F65A
:10557800CD200BF055FCC0B20128307002D1264B6B
:1055880002221A703C78002C31D1FEF7E7F9FF238C
:1055980001220093402021462346019402940BF0F7
:1055A800BDFC2B8843F6CD2043F020032B800BF065
:1055B80037FC184B1A4A1870144B14701A780AB131
:1055C800013A1A70197891B90F4A13787BB1FF2301
:1055D8000093412002220B46019102910BF09EFCA0
:1055E80005E01A7842F0C0021A70FDF765FE0CF06B
:1055F8009BF90C481DF066F80B4BB8B91A7860F3A4
:10560800820216E0BE3C0020DE1600205D17002056
:10561800F2160020D5160020761500203835002017
:10562800280E0020C1150020171500201A7842F016
:1056380004021A706A78614812F001011A780CBFE6
:1056480061F3410242F002021A705D491DF035F81B
:105658005C495A481DF01BF858485B491DF017F87B
:105668003378012B40F0A6802B8800246FF3492360
:105678006FF38A232B80554B21461C7041225448D6
:10568800FAF788FE53481CF0EFFFFEF747FA4D483B
:105698001CF0EAFF4C481CF0E7FF172363434E4A0F
:1056A8000134D15C082C01F0DF016FF30411D154EF
:1056B800F3D1002349491A01885C013300F0DF0067
:1056C8006FF38610072B8854F4D1454B1A786FF383
:1056D80045121A705A7F6FF345125A7793F83A2099
:1056E8006FF3451283F83A2093F857206FF3451269
:1056F80083F8572093F874206FF3451283F87420C9
:1057080093F891206FF3451283F8912093F8AE2017
:105718006FF3451283F8AE2093F8CB206FF3451250
:1057280083F8CB202F4B1A7802F0DF026FF3861232
:105738001A701A7C02F0DF026FF386121A7493F85B
:10574800202002F0DF026FF3861283F8202093F8FE
:10575800302002F0DF026FF3861283F83020224BEC
:105768005A786FF345125A701A7802F07F026FF375
:1057780045121A705A7E6FF345125A761A7E02F055
:105788007F026FF345121A76002311E04FF4A071DF
:1057980059430A2000FB02111448013241180879C4
:1057A800202A6FF382000871F0D10133022B01D057
:1057B8000022EBE709B0BDE8F08F00BF322E0020D1
:1057C800FC1600201815002054170020761500201C
:1057D8007715002059150020CF3300200B33002007
:1057E80057350020AC32002054320020A537002065
:1057F8002DE9FF4104460D460CF0C0F8A04B1A19DC
:1058080092F880709F4A98461278AA2A0AD1A7F17E
:105818004F03DAB20B2A00F2AD819B4A5BB29A4081
:1058280040F1A881994B0C2202FB04335A7A0833C1
:10583800AA42C0F09F81FF2A00F09C81FF229A7043
:10584800934808EBD403214693F888511CF067FF6E
:105858000646002840F08E8104F007031D41502FB2
:1058680005F0010500F0268114D8462F00F0F280DB
:1058780009D8412F00F09E80452F00F01B812D2F65
:1058880040F0768134E0482F00F0C5804F2F40F07B
:105898006F810EE0542F67D006D8522F00F08A800F
:1058A800532F40F065811CE0A7F15903012B00F24A
:1058B8005F81784821461CF032FF0646002840F0F8
:1058C80059815A2F01D1744802E0592F04D17348E5
:1058D80021461CF00EFF54E121466F481CF009FFD9
:1058E800F5E76F4821461CF01AFF002800F04281B6
:1058F8006C4821461CF013FF8046002840F03A818E
:10590800214668481CF0F5FE674821461CF0FCFE5D
:105918000227012655B1A419142041463A464346A8
:105928000097019602940BF0F9FA2AE129463A46C3
:10593800334604F101080A2000970196CDF8088043
:105948000BF0ECFA2046FCF713FC414602462B46C6
:1059580013200095FCF7D0FE384629462A463346E0
:105968000095FCF7C9FE0CE14E4821461CF0D7FE15
:105978000746002840F005810126022231463346B9
:10598800A5193E200092019602950BF0C7FA204611
:10599800FCF7EEFB294602463B4614200097FCF72D
:1059A800ABFE21463F481CF0A4FE21463E481CF0B1
:1059B800ABFEE6E03A4821461CF0B1FE0646002858
:1059C80000F0DF80374821461CF0A9FE064628B9BA
:1059D8002046FDF761FD002840F0D380002D40F0FF
:1059E8008E802046FEF7E4F9002840F0C580204666
:1059F800FEF7CCFB2D4BDB7803F02003DBB20BB9B1
:105A08002B4B1855412F00F08880522F40F0B08062
:105A18002046012183E0234821461CF080FE28B956
:105A28002046FDF739FD002840F0A480002D66D1FE
:105A38002046FEF7BDF9002840F09E801B4BDB781E
:105A480003F02003DBB2002B67D1194B032283F844
:105A5800402062E0134821461CF061FE064628B942
:105A68002046FDF719FD002840F08B802046FEF700
:105A78009FF900287ED1002D41D1204603214EE018
:105A880068240020D4160020000030803C26002026
:105A98006C1500205C2400204C2400205424002095
:105AA800CC160020FC1600200417002040320020ED
:105AB80077150020354821461CF031FE064600289F
:105AC8005FD02046FDF7C0FE20B1214630481CF0CB
:105AD80010FE4FE0502F28D12E4B1B782BBB2046B1
:105AE800FDF79EFE08BB2C4821461CF018FE064612
:105AF80020B92046FDF7D0FC002842D115B1204638
:105B080002210CE02046FEF741FB244BDB7803F032
:105B18002003DBB20BB9224B185520460021FEF7B3
:105B28003DFA061E18BF01262BE02046FDF778FE39
:105B38000546F8B91B4821461CF0F1FD0646D8B9C0
:105B48002046FDF7A9FC0746D8B9164821461CF09F
:105B5800D0FD154A135D8BB910494E7806F0200622
:105B6800F6B26EB908EB040393F80031135508E058
:105B7800012606E0002604E02E4602E03E4600E04C
:105B88001E46304604B0BDE8F08100BFCC160020A8
:105B98000A1600205C170020FC1600204032002066
:105BA800771500205915002014170020032210B57E
:105BB80005490648FAF7C4FE054806490222BDE829
:105BC8001040FAF7BDBE00BFA62100200402002045
:105BD80009020020A421002070B5804C237813F01E
:105BE800010F0AD00BF09CFC38B100207C4902F070
:105BF80089FE7C4B7C48197849E07C4D2B78002B3A
:105C08004AD00BF093FC002846D0794B1B7873B927
:105C1800784B5B7813F0010F09D00BF079FC30B9A1
:105C2800237803F02403042B01D10330B6E0724C2F
:105C3800207870B10020714902F064FE21780122B9
:105C48006F4802F085FE00201021621C08F054F80D
:105C580002E06C4902F056FE6B4C644808F09CF870
:105C68002378002B00F00F810BF05AFC002800F07D
:105C78000A81664966481022FAF762FE64485B2189
:105C8800FAF706FC002800F0FE8021780130832214
:105C9800BDE8704002F05CBE5E4C237803F005035B
:105CA800012B5DD100205C4902F02CFE202110223E
:105CB8005A48FAF76FFB601D59490322FAF7EAFDC3
:105CC80040BBE01C57490222FAF7E4FD30B95648B8
:105CD800FAF7B0FD5449024650480BE0E01C53491E
:105CE8000222FAF7D7FD40B95148FAF7A3FD504907
:105CF80002464A48FAF724FE0EE0E01C4D4902220B
:105D0800FAF7C8FD30B94C48FAF794FD4A490246FB
:105D18004248EFE7FFF74AFF6278303AD3B2092BDF
:105D280000F2B1803B4B9B78303BDBB2092B00F291
:105D3800AA800A2101FB0231C9B2002900F0A38020
:105D4800334BFF220C291A7740F29D8010295A778D
:105D580040F2998013299A7740F29580DA7770BDDE
:105D6800234E3378F3B9234B5B7813F0010F19D026
:105D78000BF0CEFBB0B931481CF0A4FC68B1304C34
:105D8800304B226802EA03033BB917F045FD20B9FE
:105D9800E37803F04003DBB223B10020BDE8704094
:105DA80009F03ABC337863B90BF0B2FB48B1264B23
:105DB8001B7803F00603042B03D02B780BB90120C2
:105DC800ECE7FEF71BF810B10020204957E0204B04
:105DD8001C78002C40D01F4951E000BFF21600206B
:105DE800ADD7020814150020000200201615002067
:105DF80054190020061A0020A2180020C0AC02087E
:105E0800050200207EAC02085C1700209FAC020847
:105E1800F4010020A1210020C7B1020804020020DB
:105E2800F8330308FC3303082AB20208FF330308D7
:105E380009B2020802340308E8B10208C1150020BB
:105E4800403200203000000F1715002050BF020814
:105E58002D0E0020E1AC02080B4802F002FD0A48B2
:105E680002F0F6FC094802F0F3FC1BF0D7F8084BE7
:105E7800DB7803F02003DBB22BB106492046BDE8EE
:105E8800704002F03FBD70BD98190020CC1800206A
:105E980040320020D9AB0208054B1B78D8019B0182
:105EA8005BB2DB1140B243EAE070C0B2704700BF9A
:105EB800F216002070B50E4686B041000122054654
:105EC80001F5E97105A80AF0BCFF0021012E8DF843
:105ED80015104FF0FF0205F1010305D10092019161
:105EE80002930920FB3A04E00092019102931E20DC
:105EF80004220B460BF012F805A83D49FAF74EFBB1
:105F080050B105A83B49FAF749FB28B105A83A4919
:105F1800FAF744FB002867D105A83749FAF73EFB92
:105F2800364B0446F8B95A78214642F010025A70A6
:105F3800FF23022200930190FE3B02903D200AF0CD
:105F4800EDFF4D200BF0CAFB691C012223461220ED
:105F58000094FCF7D1FB122021462246012300942D
:105F6800FCF7CAFB03E05A786FF304125A70002456
:105F7800E0B2552114F0FCFF38B12846214615F04F
:105F880098F910B1204615F083F90134112CEFD19E
:105F98003EBB1B481B491C4AFDF7B0FD19481B496D
:105FA80011F032F968B10BF0B3FA50B9174808F09C
:105FB80039FB30B9012315481549124A0093FDF7FA
:105FC80073FD144B0F491D70002300930533019393
:105FD800114B0D4A1B780A4802930D4B08F0B8FA8A
:105FE80002E00E4B00221A7005A806B070BD00BF73
:105FF800893403080534030895360308383500202A
:10600800C0180020961900208A19002020150020A9
:10601800851800203F36002056190020481500201A
:1060280007B54100012201A801F5E9710AF009FF4D
:10603800002301A804498DF80530FAF7AFFAD0F12A
:10604800010038BF00200EBD8934030807B54100A0
:10605800012201A801F5E9710AF0F3FE002301A865
:1060680004498DF80530FAF799FAD0F1010038BFE4
:1060780000200EBD5236030870B5154B04461B1898
:1060880093F88050B1B1134821461CF048FB88B9F9
:10609800114821461CF02DFBA5F15903DBB2012B59
:1060A8000CD94F2D0AD0542D08D021460B481CF08E
:1060B80020FB07E0084821461CF026FB074821463C
:1060C8001CF022FB04480649BDE870401CF0D4BA15
:1060D800682400206C150020C115002061150020DF
:1060E8000C170020024B1878C0F38000704700BFDF
:1060F80017150020024B1A8860F308221A8070478F
:10610800F2160020034B5878C00140B2C011C0B24B
:10611800704700BFF2160020014B1878704700BF87
:106128001615002030B5457800230021C21891705B
:1061380055FA03F111F0010F08D0064959188C7C63
:10614800017804EA0101A14208BF91700133042BD0
:10615800EBD130BDA218002046F6753104220AF0B2
:1061680070BE000070B5104C054611222046002173
:10617800FAF710F9002004F8010C2A78103414F802
:10618800011FC3B291420BD152B10849013301F842
:10619800013B112246F6C553BDE8704002F0FEBA35
:1061A80001300428EBD170BDA3180020A2180020EC
:1061B8001FB520B1134B1A8842F480521A80124B33
:1061C80000245A78214642F010025A70FF23022216
:1061D80000933D20FE3B019402940AF09FFE4D205F
:1061E8000BF07CFA40210122234612200094FCF790
:1061F80083FA12202146224601230094FCF77CFAF8
:106208001FBD00BFF2160020383500202DE9F341EC
:106218002D4C0722E37848F6883702FB003348F60E
:10622800A930DBB218180AF0FBFD257964795FFA0A
:1062380080F8002648FA06F313F0010F3AD03946E1
:10624800042201A80AF0FDFD9DF804009DF8053020
:106258009DF806109DF8072000282BD0002929D08A
:10626800002B27D0002A25D0934204D19C4221D16B
:1062780085421FD30FE09A4210D99C421AD3944208
:1062880018D89C4201D994421AD39C4201D1854224
:1062980016D294420ED18D420CD811E09C4201D105
:1062A80085420DD2944201D18D4209D99C4207D82A
:1062B800944205D301360437082EBBD1002000E0F4
:1062C8000120BDE8FC8100BF2C3A002010B504462F
:1062D80048F6E13000EBD4000AF0A2FD04F0070410
:1062E800C0B2204100F0010010BD70B5C30848F6E7
:1062F800E1355D19044628460E460AF091FD04F082
:106308000704C0B2012126B9A14040EA0101C9B27F
:1063180002E0A14020EA01012846BDE870400AF0E9
:1063280075BD0000F0B57D4B95B0DD78082200EB17
:10633800C505EDB2E90001F5F04104A810310AF0F5
:1063480080FD774B774E1A78002304A9C95C312960
:1063580005D13039994041EA0202D2B205E030292C
:1063680003D12F39994022EA01020133082BECD1DD
:1063780032706C486C496D4AFDF7C0FB6A4B1B785C
:1063880013B96A4B1B78F3B16748694910F03CFFB1
:1063980068B10BF0BDF850B9654808F043F930B959
:1063A800012363486349604A0093FDF77DFB00239E
:1063B800009302330193FD3302935A485A495B4ACA
:1063C8005C4B08F0C5F805EB0511002401F5F24116
:1063D800347004A8D03111220AF033FD2646E0B209
:1063E800542114F0C5FD002838D004AB1B5D312BB7
:1063F80003D1204614F052FE38B104AB1B5D302B9C
:106408002CD1204614F04AFE40B34EB9FF23009326
:106418003420314604223346019602960AF07EFD66
:1064280004AE305D2146303814F046FE335D012657
:10643800312B4FF0030306D10093A3191BB2019629
:106448000293352005E00093631C1BB2019602936A
:106458003620002104220B460AF060FD0134112C7D
:10646800BDD1A90101F5FA4104A8883140220AF0FA
:10647800E8FC113C04AD274615F8013BE6B20134AF
:10648800302B03D13046FFF721FF38B115F8013C16
:10649800312B2CD13046FFF719FF40B34FB9FF23FA
:1064A80000933420394604223B46019702970AF0AC
:1064B80035FD15F8011C30463039C9B2FFF715FF14
:1064C80015F8013C0021302B4FF0FF0305D1009354
:1064D80023B201910293372004E0009323B2019183
:1064E8000293382004220B460AF018FD0127402C9D
:1064F800C2D1114D6B7803F00403DBB263B1403CA9
:106508002046FFF7E3FE38B90134E4B2402CF7D156
:106518006B7860F382036B7015B0F0BD2C3A0020E5
:1065280016150020C0180020961900208A1900208E
:10653800201500208518002038350020014B1878D8
:10654800704700BF2D0E00202DE9F04F4E4B002262
:106558001A704E4A85B01678002E40F091804C4B48
:106568004FF4B468DA78997808FB02F24FF03C08E7
:1065780008FB01285A78474F90441FFA88F8BA4612
:106588006CE03AF815303C24DAB2544304EB132497
:106598004C44A4B2042CEEB207D842F25A73984580
:1065A80003D904F51C546034A4B2444511D948F603
:1065B800A8300AF035FCC8EB0403834209DC364BEB
:1065C8001A787B1993F87030934302D02E4901232F
:1065D8000B702F4AD378B34232D142F26073B4FBC6
:1065E800F3F203FB12439BB2434523D12B4B9B7819
:1065F80013F0090F44D12A4B5B7803F08003DBB218
:10660800002B3DD1274B5B7803F00203DBB2002B54
:1066180036D1254B1A781BEA020F11D1019900983F
:1066280041EA02021A70FFF7F1FD48B90098FFF736
:1066380079FE05E01C4B02991A7801EA02021A70E9
:10664800013509F5B469072D1FFA89F999D1039E17
:1066580007370136082E0AF10E0A11D04FF0010B48
:106668000BFA06FB5FFA8BF301936FEA0B03F2B2A6
:10667800DBB24FF00009009202934D46039680E783
:1066880005B0BDE8F08F00BF2D0E00206517002073
:106698002C3A0020661700201615002040320020F2
:1066A800473500202A2C00206417002073B50C46BB
:1066B80001EBC001C9B2C90001F5F0410546082245
:1066C800684610310AF0BDFB104B002003EBC402F2
:1066D800121B521982F870001DF80020312A0AD1C5
:1066E8000121814003EBC402121B521992F8706019
:1066F800314382F8701001300828EDD16946312203
:1067080030231CF014F8C0B27CBD00BF661700200F
:1067180000B501EBC001C9B2890191B001F5FA4198
:106728008831402268460AF08CFB402069463122B5
:1067380030231BF0FCFFC0B211B000BD7FB501EBE8
:10674800C001C9B201EB011101F5F241D0311122AA
:1067580001A80AF076FB112001A9312230231BF091
:10676800E6FFC0B207B000BD2DE9F8430026344665
:106778002BE021462846FFF799FF21468146284607
:10678800FFF7C6FF214640EA09092846FFF7D6FF6A
:106798005FFA89F949EA000010F0FF0F05D040467A
:1067A800394602220AF04DFB03E04FF0FF33A8F808
:1067B80000300135EDB20237072D08F10208D8D1B3
:1067C8000134E4B20E3E082C07D0054BC6F5EE475F
:1067D800C6EB0308A0370025CBE7BDE8F88300BF68
:1067E8006617002010B51DF009F84FF480301DF031
:1067F80025F81DF03DF90128044628D110201CF089
:106808001FFF02201CF010FF00201DF057F8002089
:106818001DF068F84FF480601DF05AF84FF44040BE
:106828001DF06AF84FF480304FF4E0111DF022F8A3
:1068380020461DF02BF839201DF006F90028FAD063
:1068480002201DF029F81DF031F80828FBD17C2022
:1068580001211DF0C3F846F6012001211DF0BEF804
:106868000C4801211DF0C6F80B4801211DF0C2F8A3
:10687800042001211DF0BEF87E201DF0E5F838B196
:106888001DF00CF9054B04211A7861F344021A70C3
:1068980010BD00BF0340060020080818A13C0020D6
:1068A80010B50C46014620B110220C48FAF748F8FA
:1068B80004E00A4820211022F9F76CFD34B1084899
:1068C80021461022BDE81040FAF73AB804482021C2
:1068D8001022BDE81040F9F75DBD00BFF4010020AB
:1068E8000402002010B5FF2B1446029A03D0421868
:1068F80002F8013C08E06FF07F439A4204D0131479
:10690800437013128370C27019F088FA02E07F2076
:106918001DF0E0FB19F06EFA0028F8D1ACB10B4875
:1069280090F82010163001F00F0119F077FA02E004
:106938007F201DF0CFFB19F05DFA0028F8D1044B39
:1069480093F8693013F0010FE9D110BD580C0020FD
:10695800BC3B002010B50A4B002203EBC003013BEF
:106968001046084951184C7813F8011F8C4205D17C
:106978000130C0B20C320828F3D1F73010BD00BF87
:10698800A64102083C26002070B50D4C05460E466F
:106998004FF4007200212046F9F7FCFC2A463146E4
:1069A80004F50070F9F74EFC642024F8035C1AF033
:1069B80007FE0023A4F82D33024B64221A6070BD31
:1069C800253D0020AC21002010B5054C00212046B3
:1069D8004FF40072F9F7DEFC0023A4F82D3310BD44
:1069E800253D0020164B2DE9F0415D8A07462846D3
:1069F800FBF796F81349FBF79FF9134B134E1860F2
:106A0800D723B5FBF3F5EDB2822229460446F019E7
:106A180001F09EFF2846FBF787F801462046FAF763
:106A2800CDFF0B49FBF7D4F8FBF798FA0337BE19EB
:106A3800C1B281223046BDE8F04101F089BF00BFF4
:106A4800782900200000574310180020F401002086
:106A5800000020410000000070B54B4D2868FAF78F
:106A68006BFC45A3D3E90023FAF706FBFAF752FFBC
:106A7800FAF762FC42A3D3E90023FAF7B1FC3EA37C
:106A8800D3E90023FAF7D6FDFAF744FFFAF754FCE6
:106A9800FAF75EFAFAF73EFF3C4906462860FBF72C
:106AA8003FFA20B13046FBF759FAC4B25EE03046EF
:106AB8003649FBF749FA50B130463549FBF730FA09
:106AC80028B13046FBF74AFAC0B2441C4EE03046C3
:106AD8002F49FBF739FA50B130462E49FBF720FA17
:106AE80028B13046FBF73AFAC0B2841C3EE0304683
:106AF8002849FBF729FA50B130462749FBF710FA25
:106B080028B13046FBF72AFAC0B2C41C2EE0304642
:106B18002149FBF719FA50B130462049FBF700FA32
:106B280028B13046FBF71AFAC0B2041D1EE0304601
:106B38001A49FBF709FA50B130461949FBF7F0F941
:106B480028B13046FBF70AFAC0B2441D0EE03046C1
:106B58001349FBF7F9F948B130461249FBF7E0F958
:106B680020B13046FBF7FAF9C0B2841D0A2021464D
:106B7800BDE870400AF04AB9736891ED7CFF7F4028
:106B88000000000080842E411418002000001041ED
:106B98000000F0410000484200008E420000B84268
:106BA8000000E0420000F2422DE9F04F9DB019F0DC
:106BB800CBF809201AF0A0FE1AF086FC4FF46140C9
:106BC8001AF0D6FE09201AF053FF0022A3484FF40A
:106BD80080411CF09AFDA24800211DF063F9A149EB
:106BE80004224B78DFF8A0E26FF300034B709E4B52
:106BF8009E4C1A705A715A709A70DA701A719A719A
:106C0800DA719B4B033A1A709A4B00201F328EF8A8
:106C1800000020705A7105900546069006467F20B0
:106C28001DF058FA23780E2B01F2B681DFE813F035
:106C38000F004F009500E0007902DE033004850460
:106C4800EA06DC07EF075808B108D00882098A4E1F
:106C58008A48317801F00F01013149014118FFF7E5
:106C68001FFE337813F00F0308D1854A92F80123E9
:106C7800012A41F09181834A138024E0012B03D13A
:106C88007F4B93F819330BE0022B04D17C4B93F81C
:106C98000D33032B05E0032B06D1794B93F80D3305
:106CA800012B41F079810EE0774901220A7077487B
:106CB8004FF400711CF029FD754BC8221A60337817
:106CC8006FF30303BFE333785A1C01F05FB8704BCE
:106CD8001A6822B96D484FF400711CF016FDDFF8F0
:106CE80098816C4898F8001001F00F0101314901B2
:106CF8004118FFF7D5FD36B198F800305A1C62F3F9
:106D0800030388F800305F4B00221A8098F80010BF
:106D180001F00F02022A03D11A7842F010020AE0A9
:106D2800042A03D11A7842F0040204E0052A05D1A6
:106D38001A7842F040021A7001F02EB9062A04D1DE
:106D48004D4B6FF3030119707EE301F00F0101222F
:106D580012FA01F1198001F01FB9474E4E483178F7
:106D680001F00F01013149014118FFF799FD96F82B
:106D7800008008F00F08B8F1070F27DC18F0010FA2
:106D8800464B02D00020588002E04FF0FF31598076
:106D98004FEA6809062209F1010902FB09394FF097
:106DA800FF32A9F802204046FFF7D4FDFF2806D09D
:106DB8003B4B03EB40005823437401F0EDB800232C
:106DC800A9F8023008F1010801F08AB80021102260
:106DD80013A8F9F7DFFA0FA800211022F9F7DAFA59
:106DE80023780133237033786FF3030301F07BB802
:106DF800DFF884A09AF8008018F00F0840F03F816F
:106E0800284E337803F04003DBB2F3B926486FF01D
:106E18007F43817A0122009301F00F01FF23FFF7DE
:106E280061FD224B93F8692012F0400F08D093F8C7
:106E38006C3013F0040F03D0337843F04003337001
:106E48007378142262F3C7037370737813F0F80F22
:106E580030D0174800F12001A7E300BF0018014017
:106E6800002C01409A290020682400201A180020CC
:106E78002B0E0020CF33002019180020E64102080D
:106E88003C26002038350020DC210020000C014081
:106E9800AC2100208642020866430208BE34002066
:106EA800F40100202B320020580C0020BC3B0020AD
:106EB80086440208BC4B1B7803F04003DBB2002B6E
:106EC80000F0D980DFF80483DFF8049398F80030E5
:106ED80013F00C0B30D1B54E6FF07F4396F82B10A2
:106EE80006F12100009301F00F0101220523FFF7AD
:106EF800F9FC96F84C104FF4860A06F1420001F0AE
:106F08000F010122FF23CDF800A0FFF7EBFC96F854
:106F18004110FF2306F1370001F00F015A46CDF862
:106F280000A0FFF7DFFC042389F8003098F8003050
:106F380043F0080301F02EB803F00803DBB2002B7E
:106F480039D099F800A0BAF1000F03D0984800F1A1
:106F5800400138E0954E6FF07F4B717D06F10B00D4
:106F680001F00F010122FF23CDF800B0FFF7BAFCB2
:106F780096F82B1006F1210001F00F0101220723DA
:106F8800CDF800B0FFF7AEFC96F836104FF4860344
:106F9800009306F12C00FF2301F00F015246FFF782
:106FA800A1FC98F800306AF3C303DBB243F0040392
:106FB80088F800305AE099F800C0BCF1000F08D0FA
:106FC8007B4800F16001FFF76BFC99F80020303234
:106FD80008E2764E6FF07F40717DFF23009001F04C
:106FE8000F0106F10B000122CDF80CC0FFF77AFC67
:106FF8009AF80030DFF8C4B103F0100A5FFA8AFA91
:10700800DDF80CC0BAF1000F0CD098F800206CF332
:10701800820288F800205A1C62F303038BF80030C0
:1070280000F0BABF96F82B106FF07F42009206F17D
:10703800210001F00F0101220C23FFF753FC96F801
:1070480036104FF4860300935246FF2306F12C00B6
:1070580001F00F01FFF746FC9BF8003083F01002A7
:10706800C2F3001262F304138BF80030042389F88A
:10707800003000F091BF4E4800F1800195E2B8F170
:10708800010F3CD14A4800F1A001FFF709FC002E8E
:1070980000F082879AF80030444E5A1C62F30303CA
:1070A8008AF8003096F82B106FF07F4906F121001E
:1070B80042460F2301F00F01CDF80090FFF712FCB4
:1070C80096F82B1006F1210042460E2301F00F011D
:1070D800CDF80090FFF706FC96F82B1006F121007A
:1070E800424601F00F010F23CDF80090FFF7FAFB9D
:1070F8003048802142461CF008FB00F04DBF2C4868
:1071080000F1C001FFF7CCFB002E00F045872A4BA9
:1071180096221A609AF800306FF303038AF8003059
:1071280092E1264E317811F00F0A16D1244800F169
:107138002001FFF7B5FB204B1B68002B40F02C8784
:1071480013A8F9F777FB40221346014613A801F06C
:1071580023FA3378012200F019BEBAF1010F39D1B0
:1071680012486FF07F4390F82010002200931630E9
:1071780001F00F01FF23FFF7B5FB01F077FA0028B4
:1071880000F00A873378022262F3030333700D4B51
:107198001A7842F080021A700B4B5A7842F00202B9
:1071A8005A7000F0F9BE00BF2B320020580C0020A6
:1071B8008644020800100140AC2100201918002064
:1071C8006645020830320020CE36002040430020B9
:1071D800C744002001F00F0101F10E0303F00F0373
:1071E800012B44D89B4849014118FFF759FB9A489D
:1071F8006FF07F4390F8201000221630009301F0C2
:107208000F01FF23FFF76EFB19F0A6FF337803F099
:107218000F03022B13D116F0CBFA002800F0BC861E
:107228008E4B1A7842F040026FF304121A705A78A3
:107238006FF345125A703378032200F0A7BD16F099
:10724800A1FA78B116F040FB16F0F8F9844B00204B
:107258001A7858816FF3C7121A703378042262F3D0
:10726800030333707F4B1A786FF3000263E5BAF1BA
:10727800040F4DD1DFF8DC914901DFF81082494451
:107288004846FFF70DFB98F80010774B01F0040211
:10729800D2B27AB941F004016F4883F800A088F8A7
:1072A800001090F836104FF4860300932C3001F04C
:1072B8000F01EEE293F800A0BAF1000F40F06C86DF
:1072C80065486FF07F45417D01220B3001F00F01C9
:1072D800FF230095FFF706FB64480122817AFF230C
:1072E80001F00F010095FFF7FDFA98F8003005222C
:1072F8006AF3820388F800303378484662F3030360
:10730800337009F1A001FFF7CBFA554600F044BEEF
:10731800DFF84481FF2398F8201000226FF07F499E
:1073280008F1160001F00F01CDF80090FFF7DAFA26
:107338002BB2072B18D1337808F121006FF3030320
:107348003370237801220133237098F82B100E2311
:1073580001F00F01CDF80090FFF7C4FA44488021EE
:1073680000221CF0D2F90025424E96F86B3013F03B
:10737800040F00F0118698F857106FF07F43002231
:1073880000933D48FF2301F00F01FFF7ABFA96F891
:107398006B303A4A03F00F03012B137003D1002D11
:1073A80008BF01250CE0022B04D12BB2012B08BF2A
:1073B800032505E0032B03D12BB2032B08BF0725B8
:1073C800ABB213F0010F02D02D4A3121517713F0DF
:1073D800020F02D02A4A3221917713F0040F00F0ED
:1073E800DB853322264BDA7700F0D6BD1948254EC7
:1073F80000F1C001FFF754FA96F80090DFF85C80BE
:1074080019F00F090CD116F033F898F8003069F329
:10741800000388F8003033785A1C62F30303337092
:1074280016F0B8F898F8003013F0010F00F0B485A2
:107438000022154880211CF068F90A4B00225A7076
:10744800337862F30303337023780133237000F039
:10745800A3BD00BF66450208580C0020CE360020A8
:107468003032002046360020C744002001000020AA
:1074780000100140BC3B0020A50C00202A3200204F
:10748800F401002019180020001801404043002092
:107498008648874E00F1E001FFF702FA0FA8F9F7D6
:1074A800C9F90FA902468348F9F74AFA0021824828
:1074B800B18090F8C5106FF07F4300220093BB3075
:1074C800FF2301F00F01FFF70DFA7C4A92F86B10C9
:1074D80092F86C30327843EA012312F0010FB3803E
:1074E80010D0A3F1EB0292B20A2A04D9A3F5E673ED
:1074F8009BB2282B02D8F3880133F38033786FF3DB
:10750800000333707378002B40F04685684AD288B0
:107518007AB16B4A1BA8117863F3030111702278C2
:107528008DF86F300132227028228DF86C201CF003
:107538000BF90022F28000F02FBD624EDFF8ACA1FB
:10754800337803F004085FFA88F8B8F1000F15D112
:1075580009A841461522F8F71DFF5B4BCAF80080C1
:107568001B684546CDF827303368474643F0040387
:107578003360564BA3F8368300F00EBD03F080034A
:10758800DBB2002B67D1DAF80010002940F004853F
:107598004F48FFF785F94F484FF480511CF0ABF87E
:1075A800012806D04A4800F1A001FFF779F900F058
:1075B800F3BC4649B1F83623002A43D0093146487E
:1075C800013AF9F7BDF9444B03F1100113F8012B07
:1075D8000D2A01D00A2A02D1202203F8012C8B425D
:1075E800F4D13E4B4FF03C0808FB073808F11E0861
:1075F8004046F9F71FF9414602463948F9F74AF972
:10760800D8B9022F03D1336843F0100304E0032FE5
:1076180003D1336843F040033360327853005BB2E0
:1076280003EAC263DB173268DBB263F3C712326066
:107638001BB1FFF7C9F900F0AFBC0137FFB2042F47
:1076480008BF0227254B3C2606FB07363046F9F7CC
:10765800F1F8314626E0DAF80080B8F1000F40F082
:107668009B84737803F02002D2B2002A40D11D4BCC
:1076780009A81A889B781C498DF82630ADF8242073
:10768800F8F7E2FE114B5B7A302B07D1FFF79CF934
:10769800336843F40053336000F07EBC09A8F9F75F
:1076A800C9F809A9FFF770F900F076BC6645020829
:1076B8004636002008020020580C0020BC3B002061
:1076C80019180020B0210020073403081C3D0020B1
:1076D8006646020800080140040200200C00002051
:1076E800253D00200C34030810340308AC21002089
:1076F80003F04003DBB2002B40F08980B14800F171
:107708006001FFF7CDF8B048F9F794F88046AE4924
:10771800AE484246F9F7BEF8002873D1AC4B434453
:107728005B7A302B6ED1FFF74FF93368DFF8D092D0
:1077380043F48043336099F82B106FF07F43009334
:1077480009F12100082301F00F010122FFF7CAF80F
:107758006423CAF800307F201CF0BCFCDAF8003043
:10776800002BF8D1984699F88E10D633994E89F89F
:1077780086304B3B6FF07F4A89F88730964801F096
:107788000F0142467433CDF800A0FFF7ABF896F826
:10779800B91106F5D670033001F00F014246FF23F8
:1077A800CDF800A0FFF79EF896F8C41106F5DD7035
:1077B80001F00F014246FF23CDF800A0FFF792F831
:1077C80096F8CF1106F5E270013001F00F0142463C
:1077D800FF23CDF800A0FFF785F896F8DA1106F533
:1077E800E87001F00F014246FF23CDF800A0FFF733
:1077F80079F899F899107948CDF800A001F00F01AF
:10780800424646E07648F9F715F875494AE796F88A
:1078180002B0DFF8EC910BF0020B5FFA8BFBBBF1C7
:10782800000F3AD199F82010FF236FF07F4809F133
:10783800160001F00F015A46CDF80080FFF752F804
:10784800684B93F86B3003F00803DBB2002B00F0B1
:10785800A38399F82B10012209F1210001F00F01EF
:107868000323CDF80080FFF73DF83368554843F40B
:10787800003300F180013360FFF712F855485A468B
:1078880090F8E51100F5EC70CDF80080033001F0B8
:107898000F01FF23FFF726F87EE3CAF8008099F866
:1078A80020106FF07F4300934246FF2309F1160032
:1078B80001F00F01FFF716F82AB241F211139A42AC
:1078C8001DD1434B5B7A302B13D1FFF77DF833681A
:1078D800454668F3514368F38E3368F34D3333609C
:1078E800414B1A7868F303021A7023780133237026
:1078F80052E33E48F8F79EFF3C49FFF745F8394EFA
:1079080096F86B3013F0040F00F0468325B9384819
:1079180020211022F8F73EFD7F201CF0DBFB99F8B0
:1079280057106FF07F43002200933248FF2301F085
:107938000F01FEF7D7FF96F86B202F4B02F00F02CE
:107948000D2A1A7005D125B92C4A412191754FF499
:1079580080551A78062A08D12AB2B2F5805F04D178
:10796800264A3621D1754FF488551A78082A08D145
:107978002AB2B2F5885F04D1204A3821117641F243
:1079880010151B780B2B09D12AB241F210139A4219
:1079980004D11A4B2A225A7641F211150D486FF07C
:1079A8007F4390F8F0110022009300F5F370FF2355
:1079B80001F00F01FEF796FF96F86B3013F0010FF8
:1079C800AAD0E9E2664602081A010020253D0020F7
:1079D8001C3D002001000020DC0C0020E70C0020EA
:1079E800FC000020BC3B00201918002038010020B2
:1079F80004020020A50C00202A320020F4010020F7
:107A0800580C0020A34B1A7842B300221A700F209A
:107A1800FAF71AFB06460A20FAF716FB9E4B9F490F
:107A280058824A7812F0010F18D06436301A5883F9
:107A38009B4B1A78642A01D19B321A701B78984E96
:107A4800FF2B0BD00A21B3FBF1F1964B19311980AA
:107A580095481CF027FA337801333370DFF86482D5
:107A680098F8003013F00F0612D18E4B19228B486C
:107A78001A804378192143F0010343708A481CF0A7
:107A880011FA8A4800F12001FEF70AFF04967CE209
:107A9800012E68D1804B5A8BA2F1690189B2112954
:107AA80008D8049911F0010F04D141F00101C9B2BD
:107AB80004910592049A12F0020F0DD15B8A7C4A58
:107AC8001380A3F5C263023B9BB2D72B04D804985A
:107AD80040F00203DBB204931B20FEF783FF0599F5
:107AE800744B0AB2632A05DD642192FBF1F230324D
:107AF8001A7401E0092A0CDD059A11B2642291FB7F
:107B0800F2F002FB10120A2012B292FBF0F23032AD
:107B18005A74059802B2642092FBF0F100FB11211F
:107B28000A2209B291FBF2F002FB101230329A7469
:107B38005B4B1B78FF2B08D158495B484B786FF398
:107B480000034B7000211CF0ADF9049A032A40F0A1
:107B580023825248002143786FF300034370524850
:107B68001CF0A0F911E2022E03D1534BC8221A606F
:107B78000BE2032E16D1504B1B68002B40F00C82F1
:107B88004A4800F14001FEF78BFE1B20FEF72AFF52
:107B9800414B5B8AA3F51E630F3B9BB2542B00F24B
:107BA800FB81F2E1042E0CD13B4B988A0EF02EFF9C
:107BB800002840F0F1813D4800F16001FEF770FEB9
:107BC800E3E1052E07D1344B988A0EF01FFF0328F6
:107BD80040F0E281D9E1062E40F0D78122786FF398
:107BE800030301322270D5E1344800F12001FEF789
:107BF80057FE334B1B78002B00F0CE8123780133DE
:107C08002370304B1A786FF30302FFF794B82D4EA8
:107C1800DFF8A480337813F00F021AD12A4800F154
:107C28002001FEF73DFE2948F8F704FE27490246E1
:107C38002748F8F707FB2548F8F7FCFD254BA3F87C
:107C4800160233785A1C62F30303337019F03AFFB3
:107C580091E0012A16D1D8F80030002B40F09C8121
:107C680019F05CFF012840F097811B48F8F7E2FD06
:107C7800194902461948F8F70DFE002840F08C8192
:107C880011486FE0D8F80020002A40F085810B21C8
:107C98007BE000BF2E0E0020782900209A290020C2
:107CA80028180020540C0020002C01402647020808
:107CB8001C180020F4010020AC210020A64702086F
:107CC8001818002019180020E6470208740100203F
:107CD80018300020C040002092010020C140002040
:107CE800874E337813F00F080CD186484146FEF7CB
:107CF800D7FD33785A1C62F303033370824BA3F821
:107D0800028049E1B8F1010F18D1804804211BF025
:107D1800F2FC002800F040817A4800F12001FEF7CB
:107D2800BFFD33784FF0FF315A1C62F30303337001
:107D3800774B64221A60744B59802DE1B8F1020F19
:107D4800DFF8CC811BD1D8F80030002B40F024811B
:107D58006E4804211BF0CFFC002840F01D816A4BBF
:107D68005880684800F14001FEF79AFD33785A1CA4
:107D780062F3030333706423C8F800300CE1D8F8C9
:107D88000020002A40F008810C21217062F30303CF
:107D9800A9E0604910234FF40052CB700D3B8B7063
:107DA8000A805D481BF058FC0A2200215B48F8F75E
:107DB800F1FA80201BF0B4FB237801332370504B79
:107DC8001A786FF303021A70514BC8221A60E3E065
:107DD8005348DFF848A100F12001FEF761FD9AF849
:107DE8000030002B00F0D8804E48DAF80020444ECE
:107DF8000260BAF8042082809AF8062082713178ED
:107E080011F00F0159D1DFF80881D8F800100029C6
:107E180040F0C2809AF80410A2F5A6524FF0640B05
:107E2800103A0BFB01229AF805004FF00A0909FBEA
:107E380000200393F9F774FE3B49F9F77DFF0246EA
:107E48009AF80200039BA0F5A65010380BFB030B11
:107E58009AF80100354B09FB00B018600392F9F756
:107E68005FFE039A01461046F9F7AAFD304B1860E9
:107E7800F9F762FA1EA3D3E9002382468B46F9F785
:107E880035FD002800F08880504659461AA3D3E9EA
:107E98000023F9F721FD00287ED0FEF7DDFD3378B9
:107EA80048465A1C62F303033370C823C8F80030ED
:107EB80008F0B6FFC0B207906EE001296CD10D3012
:107EC8000799832200F044FD114BD3F80080B8F1E4
:107ED800000F61D140461BF023FB23780133237048
:107EE800337868F30303337056E000BFAFF30080C4
:107EF800736891ED7CFF7F400AD7A3703D008040F6
:107F08001918002046480208BE340020000C014021
:107F1800AC210020962900200010014030180020D4
:107F2800A64802080402002000007A442C18002009
:107F3800141800208448854E00F12001FEF7B0FC9B
:107F4800F37913F0010F27D0DFF8488298F80090F2
:107F580019F00F0920D17E4B0A2259781878103968
:107F680002FB0011B1701979D878103902FB0011A1
:107F78007170D9799B79103902FB0312327016F0AF
:107F8800F5FEF37969F30003F37198F800305A1C91
:107F980062F3030388F80030DFF8FC9199F8006079
:107FA80016F001063EF43BAE6A4B01221A7018F037
:107FB8002DFD2378092B01D00D2B28D101206649EE
:107FC80011F0F4FC654B664A5B7803F01F03D35C41
:107FD800644A522B137002D1634B01221A70634B0F
:107FE800634A03F1200153F8040B8B4242F8040B57
:107FF800F9D1002117A811F003FD17A80D2119F0D8
:10800800FDFC5C4B1A78013202F003021A7099F8F1
:10801800006006F00206F6B2002E00F08B800EF02B
:1080280051FF12F0D3FF06980322431C93FBF2F290
:1080380002EB42029B1ADBB20693002B79D1DFF8E0
:10804800488198F84960C246002E4DD0022E03D1CF
:1080580098F80130312B49D023780E2B13D146489C
:1080680046490522F8F716FC8246002840D1B21F7F
:1080780037484349F8F764FC344B5646DA7942F0FE
:108088000102DA7135E00D2B03D13E483A49072247
:1080980027E0032B22D13C4B002713F8012F2C2A71
:1080A80003D00137FFB2B742F7D113A832493A4695
:1080B800F8F746FC7B1C07E00AEB03025278303ADB
:1080C800D2B2092A03D80133DBB2B342F4D30AEBA4
:1080D8000701FA430FA80231D21802E0264909A87D
:1080E800721EF8F72DFC03E0069E02E0012600E070
:1080F80000261E4B204A03F1100153F8040B8B4253
:1081080042F8040BF9D1214B214A03F1100153F82D
:10811800040B8B4242F8040BF9D1402388F8113044
:108128001C3B88F82230023B88F84B3019F0EEF9F6
:1081380000E0002699F8003003F0F5036FF3000320
:1081480089F80030FEF76BBDE64802082C3A00209B
:108158001E1800202E0E00205D4000205C400020EC
:108168008C7F0208F432002018180020F401002047
:10817800A13300204B320020CB3C002013340308ED
:10818800D03C002030180020CA3C00200402002007
:10819800DC3C002019180020A43C0020AFF300802C
:1081A80010B5044640181146F8F7E6FA2046F8F7E5
:1081B80041FBC0B210BD42540131C8B27047000043
:1081C80010B50C4B0C4A1B780C460E2101FB0323FF
:1081D800997A31B101390523594301F56F5189B2B3
:1081E80001E04FF46F510019042208F02AFE201D07
:1081F800C0B210BDE1420020C012002010B5054BEE
:108208000C46197800190131042200F0A1FB201D49
:10821800C0B210BDE142002000F5224000F5CF7049
:1082280008B5013008F0FCFD10F0FF0F14BF002066
:10823800012008BD10B50A4600210446FFF7B0FF2B
:1082480001462046FFF7DAFF114A01462046FFF7AC
:10825800A7FF232201462046FFF7ADFF014620462F
:10826800FFF7AEFF5B2201462046FFF7A4FF23225B
:1082780001462046FFF79FFF01462046FFF7A0FF73
:108288007C2201462046BDE81040FFF794BF00BF9E
:108298001934030810B55D220446FFF78CFF0D2240
:1082A80001462046FFF787FF0023235410BD38B549
:1082B8001D460C4640182C1911461A4600F048FB7A
:1082C800E0B238BD2DE9F04118490446FFF7B2FF86
:1082D800174F0E263B78174D73430146EA5A20463E
:1082E8000423FFF7E4FF202201462046FFF763FF3F
:1082F8003B78014606FB035320469A7A0223FFF790
:10830800D6FF202201462046FFF755FF3B7801465D
:1083180006FB035520466A7A0323FFF7C8FF014688
:108328002046BDE8F041FFF7B5BF00BF1C34030885
:10833800E1420020C01200202DE9F047264E0E220F
:108348003378264F534337F90380FA1824494FF4FA
:108358007A73044698FBF3F8157AFFF76BFF4E2201
:1083680001462046FFF727FF1E4B1C2202FB05355E
:108378005FFA88F8B8F1030F01460CBF05F1120245
:1083880005F108022046FFF70BFFA14680460025AD
:1083980019E019F8013BA32B07D133780E2202FB11
:1083A8000373204629465A7A08E0242B09D13378EA
:1083B8000E2202FB03739A7A204629460223FFF70E
:1083C80076FF0135EDB24545E3D120462946BDE8A3
:1083D800F047FFF75FBF00BFE1420020C012002056
:1083E80026340308AC7F0208074B187800F0040015
:1083F800C0B240B11A686FF382021A60034B0022C0
:108408001A70034B18787047403200205418002027
:108418003C180020054B00211970054B05481A68C7
:1084280061F382021A601222F7F7B4BF54180020D1
:10843800403200203C18002038B5084C0849227802
:108448000546F7F7FFFE23780021E954054B1A6823
:1084580061F382021A60207838BD00BF54180020EA
:108468003C18002040320020064A07491378112B97
:10847800C85401D801331370044A136843F0040345
:1084880013607047541800203C1800204032002028
:10849800054B1B7813F0010F05D1044B181810F881
:1084A800010CFFF7E1BF7047551800202649020864
:1084B8002DE9F041334C002314F8101094F82A20C9
:1084C80001F00F0161F3030284F82A2004EB400055
:1084D80084F8293084F828304378DFF8B88063F3CB
:1084E8000712638C4FF4D277E38498F800302A2679
:1084F8007B4306FB0133244D2448E95A84F82A209B
:108508001BF0CEFC98F8003094F82A207B4302F048
:108518000F0206FB0233EB1859881C48013989B24F
:108528001BF0C2FC01210A4618481BF089FC0121F6
:1085380016481BF076FC98F8003094F82A207B4304
:10854800120906FB02331248E95A1BF0A9FC98F8F5
:10855800002094F82A3057431B0906FB0376AD190F
:1085680069880B48013989B21BF09CFC01210A4635
:1085780007481BF065FC06480121BDE8F0411BF0E7
:1085880050BC00BF561800203249020800080040BD
:10859800003401408218002030B5164C94F82B5056
:1085A800A38445F00105002384F82B50628484F8E5
:1085B800211084F8203019E0C55CA5F13002D2B250
:1085C800092A08D9A5F14102D2B2052A9ABFA5F114
:1085D8003702D2B22A46084D013305EB420292F81F
:1085E800495392F84823257062700234DAB28A42FD
:1085F800E2D330BD5618002032490208124B10B59C
:108608009A8C0024DA8483F8294083F8284022468B
:1086180001210E481BF014FC64210C481BF040FC9F
:1086280032210A481BF040FC0121224608481BF071
:1086380007FC642106481BF033FC05483221BDE8DD
:1086480010401BF02FBC00BF561800200008004047
:108658000034014010B500212C220348F7F79AFE98
:10866800BDE81040FFF7CABF5618002070B5214C6E
:108678002378042B39D8DFE803F0030D152A3000DE
:108688001D4B012093F82B3013F0010F30D02070D0
:10869800013870BD184B93F82000FFF709FF02233B
:1086A800237022E0144DEE8CFEB9FFF7A7FF95F872
:1086B800203095F821200133DBB29A4285F820302A
:1086C80001D8042300E003232370304670BD0A4B11
:1086D800D88C50B90123237070BD074BDD8C35B998
:1086E800FFF7B8FF2570012070BD002070BD002085
:1086F80070BD00BF8318002056180020044B0022CC
:108708005A701A709A7842F001029A70704700BF46
:1087180098190020202102480A46F7F73BBE00BFFF
:10872800F401002038B5044608460D46F8F782F8EB
:1087380098B10319202B094BC8BFC4F120001C199C
:10874800002308E014F8012BE02A14BFEA5C202279
:1087580004F8012C01338342F4DB38BDF401002016
:108768000D4B46F635321B689B6893420FD043F693
:10877800F82293420BD0122B09D0B3F5E97F08D029
:1087880046F6D9301B1A584240EB030070470120C7
:1087980070470120704700BFBC180020F0B51F4685
:1087A80087B006460C46084600211546F7F7F2FD45
:1087B800244B07B19F80B3F9041005A801EB86018B
:1087C800042208F03EFB002605AB9B5D013BDBB2B3
:1087D800B92B34D81D2B4FEA031208D8D31803F548
:1087E800164168465231112208F02BFB0BE016495E
:1087F800D3185B186A4603F11007186859680833DC
:10880800BB4203C2F9D12046F8F714F8C7B268464C
:10881800F8F710F83818A84203D8E0196946F7F7AE
:10882800ABFF6846F8F706F87B1C1B18AB4203D26F
:10883800E0190649F7F708FE0136042EC4D107B03F
:10884800F0BD00BF98190020441603083E34030801
:1088580010B500216C220446F7F79CFD0123A37094
:1088680010BD002343700370837843F001038370C5
:10887800704700002DE9F0419378804613F0010F0E
:108888000D4614463AD06FF30003937018F016FEA5
:108898006378002B32D123780BB90A336370A3783D
:1088A800174F6FF30003A37018F008FE217807EB49
:1088B80008066118073130462A46F8F741F830466D
:1088C800F7F7B8FFC6B2AE420DD80AD2002323701C
:1088D80006EB08000A33637038182021AA1BF7F743
:1088E80059FDAE420AD12278A3181B7A1BB1013276
:1088F8002270BDE8F08123700A236370BDE8F0811F
:10890800F4010020054B1A780AB100221A701B786E
:1089180046F68A4202FB0311FFF704BF9F180020A6
:10892800F8B505460C460818002108F06FFA013C16
:10893800E4B26719384608F073FAC6B2202E03D895
:108948003846002108F062FA0CB1202EEFD9F8BDA4
:1089580002F00F03032B22F07F0230B5D2B20CD9FC
:108968004FF47A7491FBF4F42025E4B2057002B157
:1089780014B13034047000220130B1F57A7F05DB80
:108988004FF47A7491FBF4F504FB1511022B0BD903
:10899800642491FBF4F42025E4B2057002B114B10B
:1089A8003034047000220130632904DD642491FB13
:1089B800F4F504FB1511012B0AD90A2391FBF3F3F3
:1089C8002024DBB2047002B10BB1303303700130E4
:1089D800092904DD0A2391FBF3F203FB121130315C
:1089E800017030BD13B5104B01461B689A899C7BFA
:1089F80012F0100214BF0220012034B10B4C9B7CF2
:108A08002478634303FB001109B23AB10DF1060063
:108A1800022208F016FABDF8060002E0084608F03F
:108A2800FFF900B21CBD00BFBC1800204919002086
:108A380010B50F4B1B689A899C7B12F0100214BF6B
:108A48000221012134B10B4C9B7C2478634303FB46
:108A5800010000B22AB108490222BDE8104008F01E
:108A6800EAB9054B1968BDE8104008F0CFB900BF56
:108A7800BC18002049190020601900203038C0B205
:108A8800092894BFFF20002070470000024B1A7885
:108A98006FF300021A7070478919002070B5FFF74C
:108AA800F5FF884B1A781E2A01D91E221A70864CA7
:108AB8002678254606F0F006202E72D108F028FD0B
:108AC80000286ED1814B1B7833B92378C3F3031286
:108AD800013262F307135EE07D4B1B7803F08003DD
:108AE800DBB2002B59D07B48F7F7A4FEC5B27A4C0D
:108AF800BDB1204679493246F7F722FF0A2D0BD837
:108B08002A4620467349F7F71BFF60193146C5F11D
:108B18000A02F7F73FFC04E020466E490A22F7F7FD
:108B28000FFF6F4B1B7813F0010F01D0472300E0B4
:108B38002023E372684C042204F10C00A521F7F706
:108B480029FC684B1A7852B1FF23012A237306D9EE
:108B5800022A637303D0032AA37318BFE373624C1A
:108B6800257815F0600502D194F8A33013B95F4851
:108B78005F4902E05D4804F1A3010622F7F7E0FE31
:108B88005C4B1B78452B40F09A81002D40F0978173
:108B9800237843F08003237070BD4F48564932460E
:108BA80082E12C7804F0F004102C3FD108F0B0FCDE
:108BB80000283BD1202251494748F7F7C1FE4648D3
:108BC8004E492246F7F7BCFE4D4B1B7813F0010FB8
:108BD80006D04C48F7F72EFE4A4902464A4805E0B7
:108BE8004A48F7F727FE494902464748F7F7A8FEDB
:108BF800364B1B781BB946484649102254E1444875
:108C080045491022F7F79CFE314B1B7803F080038F
:108C1800DBB22BB13B48F7F70DFE02463F484FE069
:108C28003A48F7F707FE02463C4842E02B7803F043
:108C3800F003302B7ED108F06BFC00287AD1264C4B
:108C4800202237492046F7F77BFEA521052204F1AB
:108C58000B00F7F79FFB334B1B78042B02D9FF233C
:108C6800E37300E002D1FF23A37301E0032B02D1D9
:108C7800FF23637301E0022B02D1FF23237300E07B
:108C88000BB1FF23E372284B5B7813F0600F05D01C
:108C98003F23E37223736373A373E373234B1B783C
:108CA80003F02003DBB233B11848F7F7C3FD0246DF
:108CB8001F481649F8E01348F7F7BCFD02461C4860
:108CC8001049F1E09519002089190020DC210020C5
:108CD800B0210020B4210020F401002030DC02087B
:108CE800D8420020A9220020E42100200E02002002
:108CF8004BB2020884180020EEDB02083312030886
:108D0800CE3600207D130308010200209E130308BD
:108D1800040200200018030854120308110200205E
:108D2800F0B2020867240020A02900204032002069
:108D38000F0200202B7813F0F0030CD12022604999
:108D48006048F7F7FDFD604B5E4819888322BDE84F
:108D58007040FFF7FDBD602B1ED108F0D9FBD8B9D4
:108D68005A4920225748F7F7EBFD5948F7F762FDB3
:108D7800574902465748F7F7E3FD5748F7F75AFDB2
:108D8800554902465548F7F7DBFD5548F7F752FDB8
:108D980053490246534887E02B7803F0F003102B21
:108DA80006D108F0B5FB18B146484F4920227BE0B0
:108DB8002B7803F0F004402C02D0502C78D108E036
:108DC80040484A492022F7F7BBFD494B1B784BB96D
:108DD8004CE03C4847492022F7F7B2FD464B1B7848
:108DE8003BB943E0454B5A7882B11B78022B14D12A
:108DF80005E0434B1B7813F0010F07D00DE0414805
:108E0800F7F718FD3F4902463F4835E03F48F7F776
:108E180011FD3E4902463C482EE03D48F7F70AFD61
:108E28003B4902463848F7F78BFD402C0BBF334BC4
:108E3800384B5B78DB78022B0AD0042B0FD0012B40
:108E48001CD13548F7F7F6FC3349024633481BE096
:108E58003348F7F7EFFC32490246304814E031480E
:108E6800F7F7E8FC2F4902462C480DE02E48F7F7A3
:108E7800E1FC2D4902462448F7F762FD2B48F7F735
:108E8800D9FC2A4902462548F7F75AFD284B1B7892
:108E9800ABB9202107222148F7F77CFA2248F7F7D7
:108EA800C9FC214902461D48BDE87040F7F748BD96
:108EB800204A6FF3071313701F4B00221A6070BD0E
:108EC8008DB20208F40100209A1800206CB2020842
:108ED8006CAB0208F801002076AB020808020020FB
:108EE80071AB02080F020020CFB202087512030806
:108EF8002832002096120308DC2100203A2E002098
:108F0800D84200203B130308FD010020E0130308AA
:108F18007D13030884210020B71203080D020020E6
:108F2800D8120308F9120308BF1303081A13030819
:108F38001F2C002089190020BC180020204B70B578
:108F4800F022204D1A702B7813F0010F0BD01E4C15
:108F5800207810F0010006D11C49FFF7D3FC2378D4
:108F680043F0010323701A4E3378532B0ED1164C5D
:108F7800237813F0010F07D000201649FFF7C2FC31
:108F880023786FF300032370FFF780FD3378232BDA
:108F980014D10D4B1B7813F0010F0FD1FFF776FD9D
:108FA8002B780D4A43F006032B701378013BDBB294
:108FB80013700A4A52F82320094B1A6070BD00BF8B
:108FC8009519002089190020C118002004080308F9
:108FD80084180020E3070308771900207819002077
:108FE800BC1800202DE9F0415E4BF0225E4D1A704E
:108FF8002A7802F01003DBB2002B2DD15B4963F312
:1090080047120B601C462A70594A9A5C2D2A01D0D7
:109018000134E4B20133112BF6D1564E3A213046D1
:10902800F7F736FA38B1801BC0B201303018214644
:109038000222FFF78DFC504B1B78452B40F08F80A8
:1090480000242046013412F019F8112CF9D12B789C
:1090580043F010032B703CE0484C237813F0010FC9
:1090680017D1424E4648FFF7F3FB424F3168384666
:1090780001310222FFF76CFC2D23BB70307846F6D5
:10908800615340496522FFF789FB237843F00103C8
:10909800237003200D213A4AFFF7ECFB2D78324E5E
:1090A80015F0E00545D110203749FFF72BFC324B6E
:1090B8001B78442B11D12D4A136801331121B3FBBE
:1090C800F1F101EB01115B1A2949C95C2D29F4D092
:1090D8001360BDE8F041FFF7D9BC532B0DD13278AE
:1090E8004E3B63F347123270204A28491268062023
:1090F80000FB02125380BDE8F081232B2FD11B4BBC
:109108001D60337803F0EF0365F347133370FFF7FF
:10911800BDFC23781E4A43F0060323701378013BF5
:10912800DBB213701B4A52F823201B4B1A60BDE8B0
:10913800F081104C10201949FFF7E4FB04F11000EE
:109148002821F7F7A5F950B1001B3178C0B20130DA
:10915800201849098022BDE8F041FFF7F9BBBDE8B6
:10916800F08100BF95190020C11800206019002067
:109178008D340020F4010020841800208919002073
:10918800981900209F19002080070308BE3400208A
:109198007719002078190020BC180020A1070308BF
:1091A800454B2DE9F041F022444E1A703378444D76
:1091B80043F0010333702B68424C9B7C022B06D191
:1091C800414B1B7803F04003DBB23BB10FE0012BAE
:1091D8000DD13E4B1B7813F0010F08D108F00AFBA4
:1091E800236800206FF355532360394944E0A3787E
:1091F800344F03F02003DBB2C3B908F0FBFAF87868
:1092080000F02000C0B288B92968324B897C1A78EE
:1092180061F301021A703B682D4943F400133B6067
:10922800FFF770FB2C4B802283F843200CF09EFF45
:10923800804678B12B689B7C012B08D1234B5B7847
:1092480003F01003DBB213B10020244914E000201E
:10925800234911E00CF0BAFF074610B140462149F6
:109268000AE00CF0FBFF10B138461F4904E01A4B26
:1092780093F8433013B91D49FFF744FB1C4B1B7887
:10928800232B16D1FFF702FC337843F00603337023
:1092980008F0B0FA23686FF3555323600BF05AFEB9
:1092A800144A1378013BDBB21370134A52F8233087
:1092B8002B60BDE8F08100BF9519002089190020B6
:1092C800BC18002040320020B0210020CE360020FB
:1092D80025080308D3360020311D0020670803083D
:1092E80046080308A908030888080308CA080308E9
:1092F8008418002077190020781900202DE9F341FF
:109308006E4B6F4DF0221A702B686E4C9B7C1BB90C
:10931800637843F0100302E0637843F008036A4E71
:109328006370337843F001033370238823F47E633A
:1093380023F01E03DB04DB0CB3F5805F08D0634B1E
:109348001B7883B15F4B5B7803F00803DBB253B142
:10935800637800206FF341035D496370FFF7D2FA29
:10936800F8F7AEFE84E06378564F03F00203DBB2F1
:10937800FBB9BB78EBB9574B93F8008018F001089C
:1093880017D1F8F79DFE7B7843F002037B702B68BA
:10939800B3F91030022B7B780CBF43F0040368F359
:1093A800820300217B70082001220B460091F9F707
:1093B800A3F9A378434A032B28D003D8012B0BD059
:1093C8000DD806E0052B2DD0517825D3FF2B32D1AF
:1093D8002BE000203E4949E000203F4946E03F4855
:1093E800F7F728FADFF82C81C7B23C4908F11000DA
:1093F8003A46F7F7A5FA0F2F3AD807F1100040447C
:109408002021C7F11002F6F7C5FF31E0344B187878
:1094180000282DD1334929E06FF341015170002014
:10942800314923E00020314920E06FF341015170B8
:1094380000202F491AE0053BDBB26FF34101022BF4
:10944800517002D100202B4910E0012B02D10020DD
:1094580029490BE0032B02D10020284906E0052BFF
:1094680002D10020264901E026490020FFF74AFAE8
:10947800637803F00203DBB20BB9F8F721FE224B45
:109488001B78232B18D1FFF701FB3378002243F018
:10949800060333706378A27003F0E50362F3820376
:1094A8006370F8F70DFE194A1378013BDBB21370AD
:1094B800174A52F823302B60BDE8FC81951900202B
:1094C800BC180020D8420020891900203A2E00201C
:1094D80025080308DE42002068040308E74200204C
:1094E800DC420020890403082D0903080D05030840
:1094F80070050308AA040308CB040308EC04030856
:109508002E0503084F05030884180020771900204A
:1095180078190020F40100207B4B2DE9F341F0225B
:109528007A4E1A7033787A4D43F0010333702B6802
:10953800784C9B7C022B11D1774B1B7803F04003AE
:10954800DBB293B1754B1B7803F02003DBB2BBB1E0
:10955800A37803F04003DBB23BB111E0012B0FD13C
:109568006F4B1B7813F0010F0AD1F8F7A9FD236898
:10957800002023F480036FF3D753236069498FE0F9
:10958800A778DFF8908107F04003DFB2002F34D1CD
:10959800F8F796FD2968644B897C1A78384661F398
:1095A80001021A70D8F800305E4943F4800367F36B
:1095B800D753C8F80030FFF7A5F92B68198A21B9E5
:1095C8000091082001220B4615E00BB2022B0CD1AA
:1095D80001223B46082039460097F9F78DF8534B8E
:1095E8001A7842F008021A7007E0012B05D100979B
:1095F8000E2039463A46F9F77FF80CF0B7FD0746D2
:1096080078B12B689B7C012B08D1454B5B7803F024
:109618001003DBB213B10020454941E00020454961
:109628003EE0414B3946187800F00300F8F780FE19
:10963800FF280FD13D4B1B7803F01803182B31D0AE
:10964800A07800F08000C0B210B138463A4927E04F
:109658003A4925E00CF0BAFD8046E0B1334B187862
:1096680000F008085FFA88F8B8F1000F0AD1F8F797
:10967800B3FFC0B2022801D840460AE0062811D834
:10968800404604E000F01000C0B210B138462C4942
:1096980006E02C4904E00CF0E1FD18B12A494046E7
:1096A800FFF730F9294B1B78232B29D1FFF7EEF967
:1096B800337843F006033370F8F702FD236823F488
:1096C80080036FF3D7532360184B1A786FF3C302E4
:1096D8001A701F4A1378013BDBB213701D4A52F807
:1096E80023302B60104B1B7803F00303022B02D1AD
:1096F8000CF012FD20B102B0BDE8F0410BF02ABC1D
:1097080002B0BDE8F08100BF95190020891900203A
:10971800BC18002040320020B0210020E4210020A5
:10972800CE36002025080308D3360020C01A0020B2
:1097380067080308460803082D0903084E090308AB
:109748000C090308EB08030888080308841800209C
:10975800771900207819002010B5FFF797F9124BF8
:109768002522DA77114B124C1B6818219A7C01FBD1
:109778000242517801F00F000F2814D00A2803DDA7
:109788000A2060F3030151709B7C182202FB0344FA
:1097980063780A2103F00F03594306486B32BDE88A
:1097A8001040FFF7D5B810BDF4010020BC18002008
:1097B80054320020100200202DE9F74F984BDFF8B3
:1097C800B0A2F0221A70DAF80030D0469C6847F24E
:1097D800DB13E11A4C4244EB0104D83A6243914B43
:1097E8009D5C9F18C5F30005EEB29946002E29D15D
:1097F80030468D49FFF786F88C4B1B78232B40F0B9
:1098080038857B7866F304137B70FFF73FF9884B44
:109818001A7842F006021A70864A1378013BDBB2C6
:109828001370854A52F82330CAF80030834B1D70F4
:10983800834B1D70834B1D70834B1E60834B1D70C3
:1098480000F017BD824E814D337893B1814A4FF4B1
:10985800A071137803F01F005B0959430A2303FB27
:1098680000137D49CB18DB78002B40F0668213701B
:1098780084E06E4B1B78532B40F0FC8095F80080F9
:10988800B8F1000F2ED14046214614F00CFE5FFAC5
:1098980080FABAF1000F25D07B7868F304137B7047
:1098A8006E4F3A781AB9204614F014FD13E0531E8F
:1098B8006B49002B184603EA0101B8BF02F11E00EC
:1098C8004011002903DA013961F01F01013114F058
:1098D8004DFD00233B7014F079FE85F800A00022AE
:1098E800594BE2E02B78002B00F0278256490A6892
:1098F8000F460B2A01D10C2316E00C2A11D1013B8B
:109908006101544A59181170554903EA01010029A7
:1099180003DA013961F01F010131204614F026FDF8
:109928001CE0092A02D10A230B60D0E10A2A27D1B8
:109938004B49013B03EA0101002903DA013961F0CF
:109948001F010131204614F053FD2B786201D31812
:10995800DBB2404A591E1170404A13704FF000089C
:10996800C7F80080FFF792F8182303FB04935A788E
:1099780042F010025A7085F8008014233370DCE13D
:10998800043A042A3FD83749D2B20878364F60B330
:1099980000200870397841B13448401810F8010C9B
:1099A800032802D0002840F0C881013B0A20584310
:1099B8004FF4A07E0EFB0400DFF89CE07044801892
:1099C800417160011B18D8B200EB800000F5EC4033
:1099D8005F30801807F01AFA387818B1013814F097
:1099E8005DFEAAE10DF01AFBA7E101200870013B1A
:1099F8000A214B434FF4A07101FB04331649CB18DD
:109A08009A1853790AE00F4F3B7823B901223A702C
:109A18000A4A137091E1FFF739F800233B708CE193
:109A28009519002054320020BBC002088418002079
:109A3800891900207719002078190020A118002022
:109A4800CA18002049190020601900205319002065
:109A5800981800204A190020A5370020051A002070
:109A68001F0000805F190020041A002068240020CD
:109A7800BC180020432B1AD1964A1278002A40F0CD
:109A880043812B78002B00F05881934B1A78002AD9
:109A980040F05381914B19680C2903D00A2903D04F
:109AA8002A7014E10B2200E009221A600FE1232B2F
:109AB8007ED1884A1278002A40F026812978DFF87A
:109AC80018A2002935D09AF8003053B184490F2BD9
:109AD8000A7084490A7000F2308101338AF8003034
:109AE8002BE17E4A1368082B1ED84FF4A0776743F2
:109AF80001394FF00A0E0EFB01717B4F181F7918C0
:109B0800C9780627013907FB0101784800EB810174
:109B180051F8040F0133002840F0D880032B40F29D
:109B2800D580082BF4D9D1E0092B40F00681023307
:109B3800CCE07B786E4E61F304137B7032781AB9EF
:109B4800204614F0C7FB13E0531E6A49002B184641
:109B580003EA0101B8BF02F11E004011002903DA2F
:109B6800013961F01F01013114F000FC002333704A
:109B780014F02CFD0DF052FAFEF788FF5E4B1A78B0
:109B880042F006021A705D4A1378013BDBB213708B
:109B98005B4A52F82330524AC8F800300023137049
:109BA800504A8AF8003013704C4A2B70136060E3F7
:109BB8002A2B3CD1474A1278002A40F0A580464912
:109BC8000B784BB14648012B02704648027040F2B0
:109BD800B480013B0B70B0E02878002800F0AD801D
:109BE8003E4A1368002B00F0A880092B1AD84FF4BE
:109BF800A071614301384FF00A0E0EFB00103A497C
:109C08001F1F0818C1780620013900FB0171374869
:109C180000EB810151F8040D013B002856D1032BBC
:109C2800F8D853E00B2B40F08880023B4EE0442BE1
:109C38001AD1284A1278002A66D1274B1B78002BA4
:109C48007BD12878431EDBB21E2B76D8214614F030
:109C58002AFCC0B2002870D0204A13680C2B6CD0A4
:109C68000A2B6AD028701BE0552B4DD1194A12785F
:109C7800002A49D1184B1B78002B5ED1287801287F
:109C88005BD90238214614F01FFCC0B2002854D01A
:109C9800124A13680C2B50D00A2B4ED01949087061
:109CA800043B042B13D84FF4A071614301380A27F1
:109CB80007FB00100C490818C1780620013900FB81
:109CC80001330A4951F823300BB904331360FEF706
:109CD800DDFE32E05F1900204919002060190020DC
:109CE800A1180020CA180020A53700204C0D00201C
:109CF800051A00201F00008089190020771900200C
:109D08007819002053190020303BDBB2092B14D8F6
:109D18009C4A1268043A042A0FD89B4A117861B900
:109D28009A4A12784AB19A4A0A27107807FB0033F0
:109D3800DBB2402B137088BF11702F78DFF8B48224
:109D4800002F5FD198F8000010F0010012D114B96B
:109D58002046904900E09049FEF7D4FD98F800307D
:109D680043F6DF2043F0010388F8003007F058F885
:109D78008A4B1870337813B989488A4901E08848B2
:109D880089490A22F6F7DCFD204614F07BFB874D53
:109D98000146022205F11900FEF7DAFD844B1B7813
:109DA80003F08003DBB22BB3824B1B88EB81337843
:109DB80003BB814B18781A4618B9204614F056FA96
:109DC80018E07E4B411E01EA0303002B03DA013B36
:109DD80063F01F0301334FF4A07161430A2505FBAB
:109DE80003137749CB18DB7813B914F01DFB01E096
:109DF80000231370182303FB0494637843F01003C3
:109E0800637036E24FF4A0736343013F0A2202FBFA
:109E180007336B4EF31893F803B06301FF1898F8F3
:109E28000030FFB213F0010F46D16648FEF710FD6F
:109E380007EB071101F5E241DF311022624807F014
:109E480000F8604B594811229A7144230370173B5C
:109E5800C370791C01300F3AFEF77AFD494B1B6835
:109E680013B9102059491FE0012B02D1102058497D
:109E78001AE0022B02D11020564915E0092B02D115
:109E88001020554910E00A2B02D1102053490BE04D
:109E98000B2B02D11020524906E00C2B02D11020C6
:109EA800504901E050491620FEF72CFD98F8003083
:109EB80043F0010388F80030334B1A789846002A9B
:109EC80000F0EB8007EB071707F5E247DF371022B2
:109ED8003648394606F0B5FF00229146334B995C67
:109EE8009A4641B109F101095FFA89F90132B9F1DC
:109EF800100FF3D106E003EB09002021C2F1100294
:109F0800F6F748FA98F8000048450BD90138C01907
:109F180006F086FF30B91C4B202118780138C0198B
:109F280006F074FFDFF8D09099F8003018460193D6
:109F3800FEF7A4FD4A46019BDFF8C09018B9432BF1
:109F480040F0858001E0432B04D1002389F80030DC
:109F5800202173E0DFF8A8E024499EF800C02448D7
:109F68009C454FD10B78ACF1300C0133DBB24FF08C
:109F78000A0E0B700EFB0C33C35C002B54D10B7014
:109F880052E000BF60190020491900205F19002025
:109F9800041A002060C10208E4C1020882330020CC
:109FA800FA01002089C20208AAC20208F4010020AE
:109FB800403200203D340308051A00201F000080AD
:109FC800A5370020981900209F190020B2C3020865
:109FD80091C30208D3C302083EC502085FC5020840
:109FE80080C50208A1C50208C2C50208CA18002017
:109FF800A04C02088919002084180020A11800200C
:10A008009E1800208EF8003099F800304FF0000CB0
:10A0180081F800C043B198F800300F2B04D803F141
:10A02800010E954B83F800E0402389F8003013783F
:10A038000978303B0A2202FB0313C15C98F8000040
:10A0480001380AF80010381806F0E0FE0EE08B4BD5
:10A058001B7803F08003DBB243B199F800302BB9C9
:10A0680098F80030FF22534403F8012C99F8003087
:10A0780013B1834A013B137099F80030012B11D1B9
:10A0880098F800300F2B02D87B4A013313707D4AB1
:10A09800002389F80030137004E004200C217A4A68
:10A0A800FEF7E8FB794B1F681FBB4FF4A0725443BF
:10A0B8002B780A22013B02FB0344361975782D09D7
:10A0C8000F2D00F0D680724CA52104F11C00063A31
:10A0D800F6F760F9FF232377002D00F0CA80012DE1
:10A0E800637700F0C680022DA37700F0C280E37783
:10A0F800BFE0012F18D14FF4A07254432B780A21E6
:10A10800013B01FB03443619737803F00F030F2B4F
:10A1180000F0AF80092B04DC01335E485943BD3A97
:10A12800A2E05C4859436AE0022F38D10BF1FF3BAB
:10A138005FFA8BFBBBF1070F98BF574BDFF85081D5
:10A148009CBF5B4493F8647008F11B0088BF00272C
:10A1580020210522F6F71EF92878C7EB08080138F0
:10A16800002318E04FF4A07262430A2101FB002289
:10A17800B25C08EB07011A4112F0010FC7F10002A7
:10A1880002D08A18DB2101E08A18A52182F8201064
:10A19800013308F10108DAB2BA42E3D369E0032FC8
:10A1A8002FD14FF4A07254432B780A25013B05FBAD
:10A1B8000343F218F35C13F0400F02D01020374924
:10A1C80006E093785A1ED2B2FD2A06D934491020E7
:10A1D80003B0BDE8F04FFEF795BBFE2B02D110206F
:10A1E8003049F5E710203049FEF78CFB2F4B3048FB
:10A1F8001B78013B05FB03442E4D2C19A1788322C3
:10A2080032E0043F042F34D80622FFB20BF1FF3BA3
:10A2180002FB0B7B284B294853F82B100A31F6F721
:10A228008FFB274B1B7893B1144B1B7803F08003EB
:10A23800DBB23BB123482021022203B0BDE8F04F36
:10A24800F6F7A8B8204B1F48197882220CE02B7823
:10A258000A22013B53434FF4A07202FB043436191F
:10A26800F71918487979BE3A03B0BDE8F04FFEF700
:10A278006FBB03B0BDE8F08F4919002040320020C1
:10A28800A1180020CA180020981900206019002081
:10A29800F40100200F020020A04C0208FCC40208B0
:10A2A800F4C3020815C402081DC50208531900208A
:10A2B80011020020A53700204C0D002004020020C8
:10A2C8005F19002012020020041A00202DE9F0472F
:10A2D8004C4C4D4F2378F02243F0010323704B4B35
:10A2E800DFF85C911A703B68494A9E6847F2DB13B5
:10A2F800F01A464246EB000618217143555C531884
:10A30800C5F300055FFA85F89246B8F1000F23D12E
:10A3180040464049FEF7F6FA99F80030232B6FD1F2
:10A32800FEF7B4FB23783C4A43F006032370137806
:10A33800013BDBB21370394A52F823303B60384B8B
:10A348001D70384B1D70384B1D70384BC3F800809A
:10A35800374B1D70BDE8F08799F80020232A23D1D8
:10A368005A786FF304125A7014F030F90CF056FE54
:10A37800FEF78CFB2378284A43F0060323701378F2
:10A38800013BDBB21370254A52F82330244A3B6064
:10A3980000231370234A1370234A1370234A13604F
:10A3A800234A1370BDE8F087532A0DD15A78C2F3B7
:10A3B80000144CB942F010025A702146304601345C
:10A3C80013F0D4FF202CF8D1304614F05BF8182392
:10A3D80003FB06A67378C1B213F0100F0AD0202928
:10A3E80002D10020134901E013490020BDE8F047DD
:10A3F800FEF788BA11480222BDE8F047FEF7A8BA6E
:10A40800BDE8F08789190020BC18002095190020A4
:10A4180054320020BBC002087719002078190020A8
:10A42800A1180020CA18002049190020601900202E
:10A43800531900203D0B03085E0B03080D02002092
:10A44800841800202DE9F0412D4E2E4F307800F56C
:10A45800E240BD3006F0E4FC3B78C4B213F0010FD3
:10A4680026D0294D2B78552B0AD1EC2C01D0013C54
:10A47800E4B23078214600F5E240BD3006F0C6FC73
:10A488002B78442B0DD1A4F11403DBB2D72B01D9BF
:10A498000134E4B23078214600F5E240BD3006F0E0
:10A4A800B5FC2B78532B03D1FEF7F0FA0CF0B6FD70
:10A4B800164B1B7803F08003DBB253B13B7813F0E3
:10A4C800010F06D0124820210422BDE8F041F5F71B
:10A4D80061BF14F0800F0F4805D12B230A210374A4
:10A4E8006143113006E02D230374373B5C43113080
:10A4F80004F520610322BDE8F041FEF729BA00BF48
:10A5080049190020891900208418002040320020B1
:10A5180004020020F40100201FB5204B20491A78BE
:10A528001AB1087840F00100087009781C4C11F045
:10A53800010F31D01B490978532901D00AB103E032
:10A5480082B901221A700DE023290BD1002018705E
:10A558001549FEF7D7F9FEF799FA237843F0060371
:10A56800237019E01B78012B16D120210A460F48C9
:10A57800F5F710FF0E4B68461B681022996806F025
:10A5880060FC002409491DF8040001EB4401013472
:10A5980018F0E0F8102CF5D11FBD00BF49190020B4
:10A5A8008919002084180020760E0308F401002081
:10A5B800BC180020034B1B78532B01D1FEF766BA59
:10A5C800704700BF84180020084BFF281A6893685A
:10A5D80007D1917B41B10649927C097801FB02338E
:10A5E80002E0927C02FB003318467047BC1800203A
:10A5F800491900204328F8B504460D46174608D1E6
:10A60800114B0A261A7891FBF6F66FF3C3021A70FB
:10A6180000E00E462046FEF731FA90B10A4B303C76
:10A628001A780A2602F00801C9B2002918BF0025C5
:10A6380006FB05466FF3C30236B21A70BE42A8BFC6
:10A648003E4630B2F8BD00BF89190020634B2DE9A2
:10A65800F3411A689846157C977C614C2DB1614886
:10A6680021780222FEF774F900E02570FF012378B3
:10A6780007F50C473C3707EB43075B4E0BB90DB1A9
:10A688000FE015B901A8394601E001A8B91E022258
:10A6980006F0D7FB9DF80430F3759DF80530337646
:10A6A80005E006F117003F210222F5F773FE5B2350
:10A6B800B375023373764D4B1B7813F0010F61D0DD
:10A6C8004B4B1B78A3F13002D2B2092A35D8227835
:10A6D8000AB9002D40D1474A117814469942464A92
:10A6E80001D000211170DFF814E10DF1080C9EF87B
:10A6F80000E0A3F13000E644DFF80CC1117800EB6C
:10A708008000604400EB010C0131C9B240189CF88C
:10A718006CC090F86C000EF804CC117008B10329D5
:10A7280001D90021117023700DB9384600E0B81E18
:10A7380001A9022206F07FFB17E0232B04D12F4B3F
:10A748001A7892B9013205E02A2B05D12B4B1A78D9
:10A758005AB1013A1A7008E0532B06D1284A533BE4
:10A768001370264A1370FFF725FF264B1B7803F05A
:10A778008003DBB2002B2FD0204B1B78F618202348
:10A78800F37529E045B31A4B1878A0F13003DBB212
:10A79800092B10D81A4A137803B92370013303F030
:10A7A80001031370D8F800302178B3F91020FFF7AF
:10A7B80021FF207005E0432803D1114B1B7803B912
:10A7C8002370104B1B7803F08003DBB223B10548DC
:10A7D80020210222F5F7DEFDBDE8FC81BC1800202F
:10A7E800CB18002002020020F40100208919002063
:10A7F800841800209E180020CA1800209C180020E9
:10A808005319002040320020A04C0208F7B5394EF9
:10A81800394D3378394C6FF34103337016F040FCEF
:10A82800FFF7C8FE02238DF807302B788BB1344A26
:10A83800D17941F00101D171324A207802EBC3038A
:10A84800D3F8A07093F8A5203978FFF7D3FE3870B5
:10A858000DE0337813F0010F06D02378303BDBB2DC
:10A86800062B9CBF264AD37003238DF80730337814
:10A8780013F0010F12D0244B1B7803F08003DBB2D6
:10A8880063B129781F4B214803EBC10393F8A43027
:10A898009DF80720C0182021F5F77CFD2378232B8D
:10A8A80009D11B4A2B781268927C013A934202DA4A
:10A8B800114A0133137023782A2B04D12B7813B152
:10A8C8000D4A013B13702378532B0FD114F04EFA25
:10A8D8000B4B00212970DA7961F30002DA71FFF776
:10A8E80069FE0C4B9A7942F004029A710023237096
:10A8F800FEBD00BF891900205319002084180020CC
:10A908002C3A0020A04C020840320020F40100201C
:10A91800BC180020B41A00202DE9F74F864E874C4A
:10A928003378874D232B874F25D12368986843F6C2
:10A93800F123984217D1DFF83482296898F800008B
:10A9480000F56A50713006F061FA98F8000001309D
:10A9580000F0010088F8000000F56A50713006F038
:10A968005FFA286007E000B2FEF73CF828603B7801
:10A9780043F008033B703378532B40F06E81236813
:10A9880048F6E9329B68934202D12A686E4B15E07B
:10A998004AF28A32934202D12A686C4B0EE04AF29C
:10A9A8000732934202D12A68694B07E048F63A42D7
:10A9B800934204D12A68674B02B101221A702368B6
:10A9C8009A6843F6DD239A420AD1634B29681A78BC
:10A9D80061F300021A7006F09BFD08B106F0B6FD9F
:10A9E800236843F6E0229B68934206D15A4B2968B4
:10A9F8001A7861F3C7121A7019E043F6EA229342F3
:10AA080006D1554B29685A7861F300025A700EE056
:10AA180043F6E72293420AD12968504B19B11A68C4
:10AA280042F0005202E01A6861F35D721A6023680E
:10AA38009A684AF220439A420AD12968484B19B1C8
:10AA48001A7842F0200202E01A7861F345121A706F
:10AA580023689A684AF2AD439A4202D1287817F0DF
:10AA680087F8236843F6DA229B68934202D12A6862
:10AA78003C4B05E043F6E822934203D12A683A4B5F
:10AA88001A7008E048F6F232934204D12B6813B9E1
:10AA98002B4B01221A6023689A684AF2AE439A4205
:10AAA8000BD1324A2B6812783149032B8B5404D1CD
:10AAB800304B5A7942F010025A71236848F63242F4
:10AAC8009B68934202D129682B4A05E048F6354233
:10AAD800934203D12968294A117016E048F6364294
:10AAE800934203D12968264A117015E048F6384286
:10AAF800934203D12968234A11704DE048F6394240
:10AB0800934202D12A68204B13E043F60452934241
:10AB180002D12A681D4B0CE049F24062934202D1EF
:10AB28002A681B4B05E04AF29E32934234D12A68C8
:10AB3800184B1A703BE000BF84180020BC18002096
:10AB48006019002089190020DC210020283200200B
:10AB58001F2C002082180020061A002040320020F6
:10AB6800D8420020BA3C0020A03200204919002019
:10AB7800B812002084210020A03700209E37002032
:10AB8800D136002045360020341B0020F610002066
:10AB9800651700203A18002048F6EA32934206D199
:10ABA8002A68A14B01201A7001460DF041F823686C
:10ABB800986843F6F12398420DD1DFF87882296826
:10ABC80098F8000000F56A50713006F01FF900236C
:10ABD80088F8003002E000B2FDF72AFF23689A687F
:10ABE80043F698139A4236D12968DFF844B2DFF861
:10ABF8004CA20BEBC1031B79DFF83882C3F3411376
:10AC0800012BDFF83C9221DD98F8000000F5665032
:10AC1800203006F0FBF898F80030DAF8001009EB5D
:10AC2800030211720BEBC1021279C2F34112032A1B
:10AC38000CD17E4A126890681030C01806F0E6F809
:10AC480098F80030DAF800204B441A7498F800306D
:10AC58002A6809F80320FFF7ADFC3B78DFF8E481A8
:10AC680013F0010F00F0F080216843F698128B680A
:10AC7800934240F081806E4A2B68914602EBC301F3
:10AC88000979C1F34111012906DD6A4A1278072AB8
:10AC980002D9FDF7FBFEE3E03278442A36D15FFAA9
:10ACA80083F82DE008F10108614B5FFA88F803EB9F
:10ACB800C8031B79C3F34113012B06DD5E4B1B78D8
:10ACC80023BB5C4B1B78072B20D8DFF868A19AF8C8
:10ACD80000303F2B08D806F01BFC70B109EBC80305
:10ACE8001B7913F0100F08D19AF800303F2B07D9C1
:10ACF80009EBC8031B79DB0902D0C5F8008005E021
:10AD080009EBC8031B7913F0080FCBD03378552B08
:10AD180040F0A6802E782CE0013EF6B209EBC6037F
:10AD28001B79C3F34113012B09DD434B1B78002B1F
:10AD380040F096803F4B1B78082B00F29180DFF89B
:10AD4800F48098F800303F2B08D806F0E1FB70B18A
:10AD580009EBC6031B7913F0100F08D198F80030DF
:10AD68003F2B06D909EBC6031B79DB0901D02E60FE
:10AD780076E0002ED0D173E04AF2AE4293420BD077
:10AD880006DCA3F52242A2F5CF72012A0ED803E011
:10AD98004AF20B52934209D133782F2B60D9B1F97B
:10ADA8001020303293425BDC303B30E043F6F12236
:10ADB800934207D11F4B1B7823B13078B5F90010A7
:10ADC8003B222CE006F0A4FB18B3236843F6C42109
:10ADD8009A688A4203D047F2CD018A4204D130787A
:10ADE800B5F900102D221AE0A2F56A51613905293A
:10ADF80003D943F6E9218A4201D1012307E043F64A
:10AE0800E0218A4202D00A318A4203D100232B6012
:10AE180026E023683078B5F90010B3F91020FFF761
:10AE2800E9FB28601CE000BF46350020BC18002064
:10AE380014040020491900204A0D00206019002040
:10AE480068240020891900202368B3F90800FDF759
:10AE5800C9FD286098F8003043F0080388F80030EE
:10AE6800FFF7A8FB236843F6D222986890420BD1DB
:10AE78002B6813B99C489D4901E09B489C490222D4
:10AE8800F5F75EFD0226B0E14AF20B5290420AD174
:10AE98002B6813B99748984913E0012B95480CBFC4
:10AEA800964997490DE04AF2AE42904218D12B6874
:10AEB800012B02D18F48934903E0022B05D18D481D
:10AEC80091491022F5F73CFD8EE1032B02D1894808
:10AED8008E49F6E7042B87480CBF8D498D49F0E76A
:10AEE8004AF29E3290420AD12B6813B981488A49A6
:10AEF800E7E7022B7F480CBF88498949E1E74AF216
:10AF08009F3290420AD12B6813B97A488549D8E70D
:10AF1800012B40F0698177488349D2E748F63742E8
:10AF2800904203D043F6EE2290420ED128680A21BF
:10AF3800B0FBF1F201FB12017C4B3031D977303292
:10AF48002E2199775A7703264FE143F6F122904252
:10AF58003ED1774B1B78E3B9022229687548FDF783
:10AF6800F7FC43F6F220FDF73DFD022201465E485C
:10AF7800FDF7EEFC3B7813F0010F00F086816E4B75
:10AF88001B7803F08003DBB2002B00F07E81694858
:10AF980019E0FDF727FD022201466648FDF7D8FCB7
:10AFA800022251482968FDF7D3FC3B7813F0010FC2
:10AFB80000F06B81604B1B7803F08003DBB2002B41
:10AFC80000F06381484820210222F5F7E3F95CE1AB
:10AFD80043F69812904240F0F5802B68574EDFF800
:10AFE800508156F8331010224248F5F7A9FC0DF1AC
:10AFF800060298F800000DF107010EF05BFE4246CC
:10B00800334620B316784E49895D03291FD0296835
:10B0180003EBC1010979C1F34111012917D1072EA9
:10B0280015D948490B224848F5F78AFC4748711C4E
:10B038000222FDF78DFC9DF80710454801310222D8
:10B04800FDF786FC9DF806104248013118E02E688D
:10B05800157803EBC601097903EBC6063679C1F307
:10B068004111012906F00706C8BF05F00705012EA2
:10B078000ADC394934480B22F5F762FC3348691C6D
:10B088000222FDF765FCAFE0022E0BD133490B22FB
:10B098002D48F5F755FC32462C48691CFDF758FC3D
:10B0A8000E36A2E0032E0BD12D490B222648F5F7C8
:10B0B80047FC2648691C0222FDF74AFC0D3694E03D
:10B0C800042E51D127490B221F48F5F739FC1F4898
:10B0D800691C0222FDF73CFC1D4805F1090102220A
:10B0E800FDF736FC0C3680E012020020704D020895
:10B0F800724D0208040200205AFA02089CFA02085B
:10B108007BFA020831F9020852F9020873F90208B9
:10B1180094F9020810F90208FFFA020841FB020834
:10B1280020FB020883FB0208A4FB0208F4010020AC
:10B13800491900200F02002040320020140400208A
:10B1480068240020E8140308F9010020FA0100200F
:10B15800FE01002001020020A614030801140308C0
:10B168008514030843140308052E11D148490B22FE
:10B178004848F5F7E5FB4848691C0222FDF7E8FB5B
:10B18800464805F109010222FDF7E2FB0B362CE0E7
:10B19800062E29D142490B223E48F5F7D1FB3E48FD
:10B1A800691C0222FDF7D4FB3C4805F10901022283
:10B1B800FDF7CEFB3B4805F111010222FDF7C8FB64
:10B1C8000A3612E0B3F91060092E04DD632ECCBFF5
:10B1D8000326022600E0012633482968801B46F032
:10B1E8008002FDF7B5FB00E010263B7813F0010F55
:10B1F8000BD02E4B1B7803F08003DBB22BB12A480F
:10B208002021801B3246F5F7C5F8294EB37803F0A4
:10B218000203DBB2002B38D0FDF7A2FA254D034616
:10B2280028B92878F11D6522FDF7B8FA08E0B27947
:10B238002978B388F01D01FB023109B205F001FE3F
:10B24800236847F2CD029B68934213D006DC43F68D
:10B25800C42293420ED043F69A5209E047F24D12A7
:10B26800934207D048F6F232934203D047F20D12C8
:10B2780093420AD105200B210D4AFDF7FBFA2978E4
:10B288000D4801310222FDF763FBBDE8FE8F00BFC8
:10B2980022140308F9010020FA010020FE01002011
:10B2A8006414030802020020140200204032002027
:10B2B8009819002049190020F5010020F0B5114B1C
:10B2C8001F78114B303F1E680DE0D6F814C01CF8EB
:10B2D80003C00133644501D112E00023DAB282428F
:10B2E800F3D301350D70094B0622094902FB0733D8
:10B2F8000D785B1993F8D440002CEED10C70F9321C
:10B308001046F0BD84180020BC180020A04C02088C
:10B31800CA1800202DE9F74F964C974E23689A6873
:10B3280043F605539A4203D133780BB9013333708E
:10B338002368924F99689B7C3A78B3F1010848BF1B
:10B3480003F106084FEAE808337808F1010812F01B
:10B35800010F03FB08188A4D00F0AD80894B1A785D
:10B368009946432A4DD128780FFA88FA0AEBD0007B
:10B3780005F056FD2268844B916846F2C4629142FA
:10B38800186001D12A783AB12A78012102F007021F
:10B3980011FA02F250401860287819780AEBD000A8
:10B3A80005F034FD236847F2AD129B68934209D13A
:10B3B800734B1A78754B03EBD203734A126883F800
:10B3C800A0211EE046F67532934205D1317800205F
:10B3D80001310CF081FF14E046F28B7A4FF0000B3C
:10B3E80023689B68534504D101200BEB00010CF046
:10B3F80073FF0AF1080A46F2CB739A450BF1010B69
:10B40800EED199F80030232B10D122682B78927C4A
:10B41800013A93420ADA5A4A013313705C4B9B781B
:10B4280003F00203DBB20BB1FDF768F999F80030BD
:10B438002A2B0CD12B7853B1514A013B1370544B32
:10B448009B7803F00203DBB20BB1FDF757F999F8CB
:10B458000030552B14D12368997C0F2910D92A78EC
:10B4680008398A42464B01DA083200E000221A7095
:10B47800474B9B7803F00203DBB20BB1FDF73EF9B3
:10B4880099F80030442B42D123689A7C0F2A3ED980
:10B4980029783B4B072902D90839197001E0083A85
:10B4A8001A703B4B9B7803F00203DBB2002B2ED0C3
:10B4B800FDF724F92BE048F6A93399420ED1314B18
:10B4C8001B78A3F13101C9B2072907D842F0060257
:10B4D8003A7007225343284A573B137023689A68E7
:10B4E80043F605539A4212D133781B2B08D9284BBF
:10B4F80046F661429A809A7842F002029A7006E013
:10B508005901C918234B0020C918FDF7FBF9FFF7AB
:10B5180051F8214A2B7811789346994288BF1370C5
:10B5280012780F32934202DD1B4A0F3B13702368D7
:10B538004FF0000A93F81290B9F10F0F9ABFC9F1B2
:10B5480020095FFA89F94FF010099BF800004FFABB
:10B558008AF318180FFA88F202EBE000019305F05D
:10B568005FFC9BF80020019B5FFA80FC9B1803F0AE
:10B5780007032AE0BC180020491900208919002077
:10B588005319002084180020601900206824002026
:10B5980098190020B4FD02084B1900204CFA03F05A
:10B5A8006549013300F0010000280CBFA520DB200D
:10B5B800DBB201F809000AF1010A09F10109082BB7
:10B5C8005FFA8AFA5FFA89F903D0B9F1200FE5D159
:10B5D80009E0B9F1200F06D023684FFA8AF19B7C65
:10B5E80089189942B1DB3B7813F0010F15D0236815
:10B5F80052499B7C09780F2B01F0800198BFC3F159
:10B608001003C9B294BFDBB2002331B129781031DD
:10B618008A1A4949CB185F219954DFF8288198F88C
:10B628000230474603F00203DBB2002B64D0FDF77B
:10B6380097F8034600BB226846F6753192688A423D
:10B6480006D024318A4203D043F6E5118A4204D158
:10B6580030783B496522002309E043F605518A42C8
:10B6680008D130781C38C0B208F107016522FDF70F
:10B6780095F818E02878F7E7236846F635329B688E
:10B68800934203D043F6F822934202D1BA79317833
:10B6980001E0BA792978BB88294801FB0231BA79D7
:10B6A80009B205F0CEFB23689A7C102A02D905203E
:10B6B8000B211EE09B6846F6353293420ED006DC1D
:10B6C80043F6E512934209D043F6F82204E046F621
:10B6D8007532934202D02432934201D1102007E000
:10B6E80043F60552934202D10020102101E00020C8
:10B6F8000721144AFDF7BEF8226846F6D931936847
:10B708008B4216D046F693218B4212D043F6ED2198
:10B718008B4202D1084BDB219977937C102B08D9F7
:10B72800297809480131022203B0BDE8F04FFDF73E
:10B738000FB903B0BDE8F08FF401002040320020BB
:10B748009F19002098190020F5010020114B0022B4
:10B7580070B50D461A7118B11B7803B920234370D0
:10B76800BDB10D48F5F766F80446681C5CB10A4996
:10B778002246F4F767FD022C0BDC601C28182021F8
:10B78800C4F1030201E020210322BDE87040F4F770
:10B7980001BE70BD381900203919002038B505469A
:10B7A800002408E0601905F03BFB3038C0B20928D6
:10B7B80008D80134E4B2044B1B78303B9C42F1DBDF
:10B7C800012038BD002038BDA018002008B505F0BC
:10B7D80027FB0023C0B2064AD25C824201D120284E
:10B7E80004D10133082BF6D1002008BD012008BD83
:10B7F800B04D020870B506460D4600240DB12D2344
:10B808002B55A0190021013405F000FB062CF5D1B9
:10B8180070BD00002DE9F04F954C964E226896F8C1
:10B828000090936892F8128099B208FB091847F6BD
:10B838001000834287B01FFA88F80BD18E49087828
:10B84800497800F00700C1F3420101EBC00108EBA1
:10B85800C10825E047F6D01083420CD18649087804
:10B868004D7800F0070088214843C5F34205773931
:10B8780001FB05010DE047F6885083420BD17E4954
:10B888000878497800F00700C1F3420101EBC001D4
:10B898008901884404E0B3F5E97F08BF01EB490852
:10B8A800764F774D397811F0010F52D146F6D5729F
:10B8B800934204D046F6D552934240F04681714AED
:10B8C80012782A2A3CD1704A92F800A00AF1010A9B
:10B8D8000AF0010A82F800A0BAF1000F1BD046F660
:10B8E800D552934208D1694B46F661429A809A78BC
:10B8F80042F002029A7028E1202110226448F4F7ED
:10B9080049FD4FEA49139944624B002009EB0301B2
:10B91800FCF7F8FF19E15D48FCF79AFF23685046E9
:10B928009A6846F6D5539A420CBF5B495B49FCF7C7
:10B93800E9FF31785A4801310222FDF709F804E19C
:10B94800552A02D0442A40F000814F4B00221A7039
:10B95800FBE05069F4F76EFF4A4B834693F800A06A
:10B968009946BAF1450F02D14E4B00221A70504643
:10B97800FDF784F800284FD04B4B5FFA8BFB1A7801
:10B9880052450ED15846FFF799FCFF2804D1584676
:10B99800FFF794FCFF283FD0444B1A7801321A7005
:10B9A80015E0DFF808A100228AF800205846059320
:10B9B800FFF784FCFF28059B04D09AF80020013289
:10B9C8008AF8002099F80020FF281A7024D02168EE
:10B9D800374A4B6910601B5C886846F6D571884207
:10B9E8001360924610D1562B01D0542B0CD13378CA
:10B9F800123BDBB2022B07D82B780FFA88F0C0185D
:10BA080005F00EFACAF800002B780FFA88F0C01873
:10BA1800DAF8001005F0FAF999F80030552B17D12B
:10BA28002368997C0F2913D92A7808398A42144B3C
:10BA380001DA083200E000221A70144B9B7803F0F8
:10BA48000203DBB20BB1FCF759FE184B00221A7047
:10BA580099F80030442B3AD123689A7C0F2A36D9BA
:10BA68002978074B072925D90839197024E000BF20
:10BA7800BC180020491900204E19002089190020FF
:10BA880053190020841800209419002098190020C8
:10BA9800F4010020D7F50208E8F302082AF40208A6
:10BAA800F50100209C1800209E180020CA180020CC
:10BAB80060190020083A1A70964B9B7803F002032D
:10BAC800DBB20BB1FCF71AFE934B00221A7099F8FF
:10BAD8000030432B0DD123680FFA88F05B69197881
:10BAE8008E4B19602B78C01805F090F98A4B00220C
:10BAF8001A7099F80030232B13D122682B78927C86
:10BB0800013A93420DDA864A01331370824B0022C0
:10BB18001A70804B9B7803F00203DBB20BB1FCF781
:10BB2800EDFD99F800302A2B0FD12B786BB17C4AA8
:10BB3800013B1370784B00221A70764B9B7803F008
:10BB48000203DBB20BB1FCF7D9FDFEF733FD754AF2
:10BB58002B7811789246994288BF137012780F3269
:10BB6800934202DD6F4A0F3B137023684FF0000BBE
:10BB780093F81290B9F10F0F9ABFC9F120095FFA33
:10BB880089F94FF010099AF800000FFA88F318188D
:10BB98005844059305F044F9634A02F8090009F18D
:10BBA80001095FFA89F9B9F11F0F059B05D82168CA
:10BBB8000BF1010B897C8B45E5DB397811F0010F1E
:10BBC80017D021685948897C00780F2900F0800037
:10BBD80098BFC1F11001C0B294BFC9B2002140B1F1
:10BBE80028789AF800C010305218CCEB00005F217A
:10BBF80011542268906849F23E6290420AD14C4B37
:10BC08001B78532B30D105F00BF94A4B187005F00F
:10BC180001FA29E0B0F5E97F26D1454A1278532A7E
:10BC280022D11846FFF7D2FD8046E8B93378DA000A
:10BC3800D31A03F11200FFF7B1FD68B1FF23009397
:10BC48003D4BCDF804801B7879200133029341469F
:10BC58000422434605F062F933780021DA00D31A4A
:10BC680003F11200FFF7C6FDDFF8A89099F802303B
:10BC7800C84603F00203DBB2002B68D0FCF770FD66
:10BC8800034688B9226847F6885192688A420BD0E1
:10BC980046F6D5518A4214BF2878307809F1070151
:10BCA8006522FCF77BFD12E0236898F806209B6864
:10BCB8002248B3F5E97F0CBF31782978B8F8043009
:10BCC80001FB023198F8062009B205F0BAF823689A
:10BCD8009A7C102A13D89B6847F6100293420BD11E
:10BCE8003B7813F0010F01D010202CE0202107220F
:10BCF8001348F4F74FFB2AE0B3F5E97F02D105209A
:10BD08000B2121E046F6D55293421BD10020102189
:10BD18001AE000BF98190020CA18002060190020F6
:10BD2800531900204B190020F40100204032002054
:10BD380084180020A0180020491900209F1900200D
:10BD48000402002000200721094AFCF793FD23681C
:10BD58009B7C102B08D9297806480131022207B0AC
:10BD6800BDE8F04FFCF7F4BD07B0BDE8F08F00BFA9
:10BD780098190020F50100202DE9F04F7A4E8BB07C
:10BD880033689D6893F81290122D01D00B2D09D1BC
:10BD9800764A122D92F80090A9F130095FFA89F9D4
:10BDA80015D01DE04AF2BB439D4203D028339D4283
:10BDB80040F055836E482821F4F76AFB8046002836
:10BDC80000F0508301302821F4F762FB4AE39F7B9F
:10BDD80037B9684BB846D879FEF7F6FB044615E044
:10BDE8000027B846FF20FEF7EFFB4AF2AC239D423E
:10BDF80004460BD14AF28B3005F012F8C0B2089015
:10BE080020B15C4B9B790BB1FCF740FE33685A4D6F
:10BE18009A68122A1AD19B7BC3B12B7813F0010FB1
:10BE280008D12046FFF7BAFC544B10B101221A7012
:10BE380000E018704F4B9B7943B12046FFF7AEFCEA
:10BE480020B14E4B1B780BB1FCF720FE2978DFF8A8
:10BE580048A111F0010100F089819AF80030DFF85B
:10BE68003CB118460793FCF709FE079B002800F031
:10BE7800B7804349002008704248434A90F800C000
:10BE880013609C45414940F08B8033689B8903F0DF
:10BE98000F03032B21D1ACF1300C0A2000FB0CF06E
:10BEA8003B4BDFF8F0C093F800E005907044099030
:10BEB8000EF1010E1CF80000DDF814C05FFA8EFECA
:10BEC800106083F800E00CEB0E00DFF8C8E01EF805
:10BED8000000002871D118706FE0082B2BD12C4876
:10BEE800ACF1300C03780CEB8C0E0993294B9E4473
:10BEF800099B734493F86CE00993264BBEF1000F3D
:10BF080001D180F800E090F800E00CEB8C0C634461
:10BF180003EB0E0C0EF1010E5FFA8EFE73449CF8D3
:10BF28006CC093F86C30C2F800C080F800E0002BB9
:10BF380043D1174811E0072B11D1BCF1300F10D1B4
:10BF48001348037823B14FF02B0EC2F800E001E04C
:10BF5800C2F800C0013303F0010303702DE0062B83
:10BF68002BD10B78013327E0BC180020A018002043
:10BF78000402002056190020891900202F0E0020E5
:10BF8800BF3C00209E180020601900205319002093
:10BF9800CA180020A04C020884180020A11800200C
:10BFA800DFF898E203709BF800304FF0010C8EF830
:10BFB80000C013B10B7863440B7040238BF800303A
:10BFC8000B784B4503D39B4B09F1FF301870087869
:10BFD8001168201804F01AFF2B7843F004032B7023
:10BFE8009AF80030232B2FD1924B09F1FF311A78A0
:10BFF8008A4229DA72B932684AF2BB4192688A42A7
:10C0080008D028318A4205D02046079304F008FF5B
:10C01800079BC8B118780130C0B21870201804F016
:10C02800FFFE28B9834B20211878201804F0EEFE73
:10C03800814B40221A702B78804A43F004032B70FE
:10C0480000238BF8003013709AF800302A2B10D197
:10C05800784B1A786AB1013A1A70774B40221A70F5
:10C068002B78764A43F004032B7000238BF80030BA
:10C0780013709AF80030432B1FD16E4B187848453F
:10C0880005D220182021079304F0C0FE079B9BF8D7
:10C0980000203AB91B7809F1FF32934202DA654A67
:10C0A800013313702B78644A43F004032B70002388
:10C0B8001370624A8BF8003013709BF8003013B18C
:10C0C8005F4A013B13709BF80030012B0ED1594B8E
:10C0D8001A784A4501D201321A70584A002313705F
:10C0E8002A7842F004022A708BF800302B7803F08B
:10C0F8000402D2B2002A71D0524A6FF3820313703D
:10C10800002111225048F4F745F9504A494B11785B
:10C118001B78994288BF137011780F318B4202DD6A
:10C128004A490F3B0B70117847481022611804F0F8
:10C1380088FE4548F4F77EFB33684AF2BB419B68AA
:10C14800C2B28B4202D028318B4205D122B9404875
:10C15800F4F770FB421CD2B20F2A3FD83A4820218C
:10C168008018C2F11002F4F715F937E0DFF8D8B0FB
:10C1780011225846F4F70EF933684AF2BB429B681D
:10C18800934202D02832934209D1214604222E48F4
:10C1980004F057FE40463946FFF7D8FA1EE021461C
:10C1A8001022584604F04DFE5846F4F743FB024669
:10C1B8002021C2F110025844F4F7ECF821464A460F
:10C1C800244804F03EFE244A1020937882F8069012
:10C1D80043F0020393700146FCF74CFB9AF80030D9
:10C1E800532B75D133689A684AF2AC239A4208D126
:10C1F800204604F015FE20B14AF28B30012104F0EC
:10C2080005FE3368DFF838A09B68122B40D1204622
:10C21800FFF7C4FA8346002830D0104BFF22197864
:10C228000F4BF9B9009201911B78782001330293E2
:10C23800FB3A1FE053190020BF3C0020CA18002019
:10C24800A118002089190020381900204B19002056
:10C2580039190020D3180020CC1800202F0E0020F8
:10C26800491900200021009201911B787A2001339E
:10C27800029304220B4604F051FE09E08AF80000FC
:10C288007D492046FFF7B6FA7C4B83F800B0EFE013
:10C2980020464946FCF744FB794B00201870336868
:10C2A8008AF800009B6849F25262934202D10090DA
:10C2B800013005E04AF2CE22934206D101230093D1
:10C2C8000146024603460CF033F86E48FCF7C0FA04
:10C2D800FEF770F92B7813F0010F17D033684AF284
:10C2E800BB429B68934202D02832934204D1404615
:10C2F8003946FFF72BFA09E05F4B634A03F1100157
:10C3080053F8040B8B4242F8040BF9D133689A684E
:10C31800122A1ED19B7BE3B12046FFF73FFAC0B13A
:10C328002B7813F0010F14D1584B9A7922B9DA7986
:10C33800574B1B789A420CD0564B1A780023303A48
:10C3480005E055492A20C91801330874DBB2934225
:10C35800F7DB326893680B2B01D0122B0AD14A4BBA
:10C36800991D13F8010B202802D10D3003F8010C98
:10C378008B42F6D192684AF2AC239A4214D1434BCD
:10C388009B798BB1089878B14FF0000909EB04004C
:10C3980004F046FD18B1404B2A224B441A7409F1A7
:10C3A8000109B9F1100FF1D12B7813F0010F25D045
:10C3B8003A4B1B7803F08003DBB2FBB133689A6811
:10C3C8004AF2BB439A422D4B03D04AF2E3418A42D8
:10C3D8000CD11B7833B9B8F1000F0FD05F3388F850
:10C3E80001300BE057B15F22FA5407E0244A1B786A
:10C3F800127810339B1A284A5F21D154284CA3780D
:10C4080003F00203DBB2002B32D0FCF7A9F9204974
:10C41800034628B908786522E11DFCF7BFF912E048
:10C428003068B4F90430A27984680978122C01FBC9
:10C43800023105D1807B18B91449C97902FB013151
:10C44800184804F0FEFC33689B68122B10D10820B2
:10C45800134A01460BB0BDE8F04FFCF70BBA0027B2
:10C46800B84600E0074609F1FF395FFA89F9B9E4EF
:10C478000BB0BDE8F08F00BF381900205319002019
:10C488004B190020CC180020040200205619002067
:10C4980049190020A0180020F40100204032002093
:10C4A800981900209F19002024282DE9F0411446EE
:10C4B80026D16B4B43F638321B686A4D9B686A4E2F
:10C4C800934206D12B7813F0010F0ED02438674918
:10C4D80009E04AF2E34293420AD12B7813F0010FA4
:10C4E80003D063490020FCF70DFA2978490800E0D9
:10C4F8002978301901310222FCF72AFA0234AAE01D
:10C50800E72809D1574B5848197880180131032278
:10C51800FCF71EFA03349EE0A3282AD1514D2B784C
:10C528003F2B15D810465349FCF7ECF95148F4F75E
:10C5380081F92A2124184C48E4B2F3F7A9FF00280E
:10C5480000F08A80297802220131FCF701FA83E0A1
:10C558005901494DC918691801F582411046DF3162
:10C56800FCF7D0F905F59240FE30F4F763F924188A
:10C5780071E0F22821D13B4F3B4D3978072605EB76
:10C588000208B1FBF6F1404601310222FCF7E0F95E
:10C5980039782D23B1FBF6F688F80230F3009E1B9C
:10C5A8008B1B364FDBB207EB83031988E21CA952B9
:10C5B8009B78A818837006344DE025280BD1304BA2
:10C5C80046F661429A8045229A719A78053842F077
:10C5D80002029A703CE05E280BD1294B46F6615264
:10C5E8009A8045229A719A783E3842F002029A70EF
:10C5F8002EE07C280BD1224B46F244129A8011225D
:10C608009A719A785C3842F002029A7020E0EC281D
:10C618000BD11B4B46F6A5529A8045229A719A78FF
:10C62800CC3842F002029A7012E0A7280BD1144BC2
:10C6380046F6C5529A8045229A719A78873842F010
:10C6480002029A7004E0E02801D1541C03E018B1FA
:10C65800054B18550134E4B22046BDE8F08100BF0F
:10C66800BC18002049190020F40100203CEE020803
:10C67800FAED0208B6F50208B8AB020831D802088C
:10C688009819002038B50A4B46F68A451B780024CD
:10C6980005FB030507E0074B22461978FFF704FF5F
:10C6A800041B2D190446287808B11F2CF3D938BD6E
:10C6B8009F1800204919002070B5002543F61C6416
:10C6C800204604F0ADFB064604F1080004F0A8FB80
:10C6D80016F0FF0F06D020F07F0010F0FF0F01D0FA
:10C6E8000135ADB246F23B139C4201D00934E7E76D
:10C6F800284670BD38B5B0F900500B4C05EBC505A0
:10C7080005F578552435284604F08AFBC1B211F0A6
:10C71800800F07D023882846013B01F07F01238042
:10C7280004F074FB208838BD9A180020454B2DE989
:10C73800F74F1B88444A044689461788DFF80C815E
:10C7480023B14FF0000A0AE09A4608E00529FBD118
:10C7580098F8003043F0040388F8003070E098F847
:10C76800003013F0030F0BD013F0010F02D0B4F117
:10C77800FF3F05D103F00203DBB21BB1012C01D04E
:10C788003F19BFB23BB2B3F1FF3F04D0B3F57A7F94
:10C7980008BF002701E040F2E7370FFA87FB0BEBF1
:10C7A800CB0303F5785303F11C00019304F038FB25
:10C7B80010F0FF0F019B16D0B9F1050F09D103F155
:10C7C800240004F02DFB20F07F0010F0FF0FC6D0EE
:10C7D80022E0B9F1000F1FD003F1240004F020FB80
:10C7E80000F07F0618E00AF1010AB4F1FF3F1FFAD2
:10C7F8008AFA04D198F8003043F0010305E0012CCF
:10C8080005D198F8003043F0020388F80030BAF5F3
:10C818007A7F0DD03D46A2E74E4505D0B9F1000F0D
:10C8280002D0B9F1050F9AD1BAF1000F05D000E096
:10C838003D46054A2DB2156002E0034BC3F800B02F
:10C84800BDE8FE8F9A1800206019002064190020A6
:10C85800F0B503789BB05A1ED2B2792A0F4600F27F
:10C86800C8805E01644AF3189B18644A46F68A46F3
:10C878001278457806FB0236E7213046F3F708FEC2
:10C888000446F0B930467C21F3F702FE0446C0B9ED
:10C8980030462521F3F7FCFD044690B930462421A3
:10C8A800F3F7F6FD044660B930464021F3F7F0FD92
:10C8B800044630B93046F921F3F7EAFD044600286A
:10C8C80076D0A41B0FB14E4800E04E4831462246B0
:10C8D800A619F4F735F83046E721F3F7D9FD30B15A
:10C8E80028466946652246F6A553FBF757FF3046AA
:10C8F8007C21F3F7CDFD50B1691EC9B201EB0111DE
:10C9080001F5C24168464431112204F09AFA3046D2
:10C918002521F3F7BDFD38B1681EC0B2694665220E
:10C9280046F66143FBF73AFF3046F921F3F7B0FDCD
:10C9380038B1681EC0B26946652246F66153FBF7F6
:10C948002DFF30464021F3F7A3FD50B1691EC9B24F
:10C9580001EB011101F5E2416846DF31112204F0D3
:10C9680070FA30462421F3F793FD50B10FB12448F3
:10C9780000E02448001929460222FBF7E9FF0234A7
:10C988000BE00FB11E4800E01E4800196946F3F796
:10C99800F3FE6846F3F74EFF0419002F29D01A4A10
:10C9A8009378141943F0020393700023E37116E09F
:10C9B8003046F3F73FFF05461FB9124831462A466D
:10C9C80015E0102810DD2A460D483146F3F7B8FF68
:10C9D8000D4A9378551943F002039370EC711020B7
:10C9E8000146FBF747FF04E0084831461022F3F7F9
:10C9F800A7FF1BB0F0BD00BF9BDD02089F180020F9
:10CA08009F190020B62A002098190020040200204F
:10CA18000C4B1B7813F0010202D000200A4905E0F4
:10CA280003F00200C0B218B108491046FBF76ABF0C
:10CA380003F00403DBB20BB10549F7E70548012110
:10CA4800FFF706BF6419002074B3020853B3020845
:10CA580095B302088B19002070B5124D124C0020B6
:10CA68001249FBF75FFE2846A1780222FBF770FF08
:10CA7800E81CE1780222FBF76BFF05F10800217939
:10CA88000222FBF765FF05F10B0061790222FBF733
:10CA98005FFFA17905F10E000222BDE87040FBF7A7
:10CAA80057BF00BFF40100208B190020B94D0208C0
:10CAB8002DE9F341504F514C3B689D7C237813F08E
:10CAC800010F2FD1022243F61A610DF1060004F07E
:10CAD800B8F94B4EBDF806304FF0FF3033602946A9
:10CAE800FFF724FE237843F001032370454B1B789E
:10CAF80013F0030F14D1B6F90010434801EBC1013C
:10CB080001F578511C31092204F09BF93F4B1B8831
:10CB18001BB13046FFF7EEFD10B90020F9F7EAFA2D
:10CB2800FFF79AFF3A4E3378552B0DD1DFF8D480B2
:10CB38003848FBF78DFE98F800304FF0FF306FF360
:10CB4800410388F800300DE0442B2BD1DFF8B48086
:10CB58003048FBF77DFE98F8003001206FF30003A2
:10CB680088F800302946FFF7E1FD98F8003013F007
:10CB7800030F15D1224D2448B5F90010092201EB05
:10CB8800C10101F578511C3104F05BF91F4B1B887A
:10CB98001BB12846FFF7AEFD10B90020F9F7AAFA35
:10CBA800FFF75AFFFFF734FF3378232B22D1154BB9
:10CBB800184E1A7802F0FC026FF382021A70FBF723
:10CBC80065FFB3786FF34103B370134B1D7835B924
:10CBD800FBF794FD3046FBF73BFE3D600AE0227808
:10CBE800013DEDB242F0060222701D700B4B53F866
:10CBF80025303B60BDE8FC81BC1800208919002065
:10CC080060190020641900208B1900209A18002050
:10CC1800841800209819002077190020781900201E
:10CC28002DE9F0411646104A0F4653780E21C3F3FA
:10CC380042034B43117803F5EE43A0330B4D01F04B
:10CC48000701044603EB4101022204F0FAF8E8194F
:10CC580021780222FBF77CFE6178A8190222BDE840
:10CC6800F041FBF775BE00BF4E190020F40100200B
:10CC7800044B02225978044BC1F3420118180131C0
:10CC8800FBF766BE4E190020F401002010B5074BD3
:10CC9800074C1B78074A03F0070304EB83031C883F
:10CCA800111814529B788B7010BD00BF4E190020CC
:10CCB80031D80208F4010020084B1B789B0902D0E8
:10CCC800012B06D102E01020054904E01020054997
:10CCD80001E005491020FBF715BE00BF4E190020E2
:10CCE80016C0020837C0020858C002082DE9F041F2
:10CCF800DFF868800F4698F80010174DC1F38201DD
:10CD08000446164605F1080001310222FBF720FE11
:10CD180098F80010042201F01C0101F50A41204690
:10CD280001F5C47104F08DF8E81921780222FBF7A7
:10CD38000FFEF81C281861780222FBF709FEA819D3
:10CD4800A1780222FBF704FEF01CE17828180222E1
:10CD5800BDE8F041FBF7FCBDF40100209D18002060
:10CD6800064B1B7803F08003DBB233B1435C044805
:10CD78002021C0180222F3F70DBB70474032002073
:10CD8800F40100202DE9F743654D664C2B682178A6
:10CD98009B68022203EB41010DF1060004F051F8F3
:10CDA8002B68A9469A6843F6F4239A4208D10020D2
:10CDB8005D49FBF7A7FDBDF806804FF4B46303E0B7
:10CDC800BDF806804FF46163B8FBF3F103FB1188EB
:10CDD8003C221FFA88F8B8FBF2F302FB1388CFB2A3
:10CDE800DEB2022251483946FBF7B2FD5FFA88F8F5
:10CDF80002224F483146FBF7ABFD02224D4841461F
:10CE0800FBF7A6FD4C4B1B7813F0010F6ED04B4B74
:10CE18004B4D1878232804D12B78012B62D8013385
:10CE280005E02A2805D12B78002B5BD0013B2B701D
:10CE380058E0A0F13003DBB2092B01D943284BD1CC
:10CE48002B7873B9D9F8003039B29A6843F6F423CD
:10CE58009A4201D10A2200E01122FDF7CBFBC7B2AA
:10CE680016E0012B0ED1D9F8003031B29A6843F69A
:10CE7800F4239A4201D1172200E03B22FDF7BAFBC6
:10CE8800C6B205E041463B22FDF7B4FB5FFA80F8E5
:10CE9800D9F800309A6843F6F4239A4209D13C2322
:10CEA8005E434FF4B46303FB0767B844ADF80680EC
:10CEB80006E03846314642460EF037FAADF806002D
:10CEC800D9F8003020789B680DF1060103EB40008B
:10CED800022203F0B0FF05E0532803D100232B7092
:10CEE800FDF768FB17482978FFF73AFFD9F80030B3
:10CEF8009A6843F6F4239A4210D0207812496522A2
:10CF08000023FBF74BFC05200B21104AFBF7B2FC72
:10CF180021780F4801310222FBF71AFDBDE8FE8394
:10CF2800BC180020491900203BF202080402002026
:10CF38000A0200201202002089190020841800200B
:10CF480053190020CA4D02089F1900209819002083
:10CF5800F501002073B5994B994D1A7812F0010F1D
:10CF680005D12A7812F0380204BF2A706A701A783C
:10CF7800924E42F001021A702B78914C13F038024D
:10CF88003ED190490978552904D113F0070F2FD0C5
:10CF9800DA1D0AE044290CD103F0070201323D39B9
:10CFA80092FBF1F1C800411A521A62F3020323708E
:10CFB8001EE053290AD1C3F3C201013161F3C5034D
:10CFC8002370637862F34303637011E023290FD160
:10CFD800FBF75CFD33787C4A43F006033370137823
:10CFE800013BDBB21370794A52F82320784B1A6060
:10CFF80000207849FBF786FC1C20FFF747FEDBE0A2
:10D00800082A2CD174490020FBF77CFC0620FFF786
:10D018002FFE0C20FFF73AFE1521182201A8FFF772
:10D02800FFFD684B1B78552B06D1637803F0FE0390
:10D03800C3F34202013A07E0442B09D1637803F0B5
:10D04800FE03C3F34202013262F343036370B3E0A9
:10D05800532B28D0232B40F0AF802378A6E0102A4A
:10D0680051D15D490020FBF74DFC0620FFF700FE7B
:10D078000C20FFF70BFE1521182201A8FFF7D0FDA1
:10D088006178564801F00101FFF76AFE4D4B1878A8
:10D09800232801D02A2804D16378DA4362F30003F5
:10D0A800D4E7532804D12378C3F3C202013280E0C5
:10D0B800A0F13003DBB2092B01D943287CD16B786E
:10D0C80002AA03F001033B21D41883F001024B4369
:10D0D800172606FB023214F8041CFDF78BFA04F835
:10D0E800040C6B780E22C3F342035343287803F5EC
:10D0F800EE43A03300F0070003EB400001A90C3A0F
:10D1080003F099FE58E0182A4DD133490020FBF767
:10D11800F9FB0620FFF7ACFD0C20FFF7B7FDFFF782
:10D12800CBFD284B1B78552B07D1237813F0C00F64
:10D1380042D0C3F38112013A06E0442B07D1237889
:10D148009A09012A38DC013262F3871333E0232B72
:10D1580004D12378C3F3C202023A2AE0532B2BD11D
:10D16800FBF794FC33781E4A43F006033370164BE2
:10D178001648197840F82120013119702378C3F333
:10D18800C201013161F3C503C3F381112370104B50
:10D1980011B1012904D101E01C3202E0114A00E07A
:10D1A800114A1A6008E0114A00211170C3F3C20243
:10D1B800013A62F3C50323707CBD00BF89190020C2
:10D1C8004E190020841800207719002078190020B3
:10D1D800BC180020D4BF0208F5BF0208CD4D0208D4
:10D1E800D04D0208084E0208244E020853190020A8
:10D1F80073B5494B494D1A7812F0010F04D12A78BA
:10D2080012F0030208BF2A701A78434E42F0010256
:10D218001A702B78414C13F003022ED1404A127831
:10D22800552A03D1C3F38202013A04E0442A06D105
:10D23800C3F38202013262F38403237017E0532A96
:10D2480003D15A1C62F30103F7E7232A0FD1FBF736
:10D258001DFC3378334A43F0060333701378013BDF
:10D26800DBB21370304A52F82320304B1A6001A801
:10D2780010211B22FFF73AFD4DE0012A4BD101A8EE
:10D2880010211A32FFF732FD254B1878232804D1D4
:10D298002378C3F34112013205E02A2807D1237805
:10D2A800C3F34112013A62F3461323702DE0532869
:10D2B80004D12378DA1C62F30103F6E7A0F1300306
:10D2C800DBB2092B01D943281FD12B7802AAC3F35B
:10D2D8004113D4180C215A1C03F001034B4302F0EC
:10D2E80001021F2614F8041C06FB0232FDF782F91E
:10D2F80004F8040C287801A900F01C0000F50A4085
:10D3080000F5C470042203F096FD29780848C1F39B
:10D318004111FFF725FD7CBD891900209D180020CB
:10D32800841800207719002078190020BC180020E4
:10D33800404E0208064B1B7803F08003DBB233B182
:10D34800435C04482021C0180322F3F723B8704730
:10D3580040320020F40100204328F8B504460D4669
:10D36800174606D1104B00261A786FF3C3021A70BD
:10D3780000E00E462046FBF781FB90B10A4B303C9B
:10D388001A780A2602F00801C9B2002918BF002538
:10D3980006FB05466FF3C30236B21A70BE42A8BF39
:10D3A8003E4630B2F8BD00BF891900202DE9F3418F
:10D3B8006E4F6F4E3B7843F001033B70347844B9AD
:10D3C8004AF2033003F02CFD6A4B6B491860204683
:10D3D80017E0012C02D10020684912E0022C02D18A
:10D3E800002067490DE0032C02D10020654908E0C0
:10D3F800042C02D10020644903E0052C03D16349C1
:10D408000020FBF77FFA3178D9B9614B1B78312BB3
:10D4180001D1013101E0302B05D1564B4AF20330DE
:10D42800196003F0F3FC5B4B1A785B4B02F0800247
:10D43800D2B20AB1202202E04E4A12683032DA77BC
:10D448006EE001290BD002290CD003290DD0042944
:10D458000ED04AF2FF25052918BF00250AE04AF236
:10D46800EF2507E04AF2F32504E04AF2F72501E048
:10D478004AF2FB252946042201A803F0E2FC474BA7
:10D48800474A03F1100153F8040B8B4242F8040B8E
:10D49800F9D1032243489DF80410FBF759FA0322F7
:10D4A80041489DF80510FBF753FA03223F489DF8C1
:10D4B8000610FBF74DFA3E4803229DF80710FBF7CC
:10D4C80047FA334B3B4C1878232804D12378022B96
:10D4D80022D8013304E02A2804D12378E3B1013BA0
:10D4E800237019E0A0F13003DBB2092B01D94328DE
:10D4F80012D194F8008002AA904418F8041CFF2264
:10D50800FFF72AFF08F8040C207802AA131813F86A
:10D51800041C281803F07AFC27482178FFF70AFF33
:10D528001B4B1B78532B1FD1224B00221A703378C8
:10D538000133DBB2062B337004D0012B14D10D4B11
:10D548001B688BB1FDF736F8002333703B781B4A14
:10D5580043F006033B701378013BDBB21370184AA3
:10D5680052F82320174B1A60BDE8FC818919002066
:10D578004919002060190020C10B0308EA0C0308B0
:10D588000B0D03082C0D03084D0D03086E0D030841
:10D598008418002040320020F401002030340308B1
:10D5A8000402002005020020090200200D020020CC
:10D5B8001102002053190020444E02087719002058
:10D5C80078190020BC18002070B5174C0D46064687
:10D5D800002120464FF4C172F2F7DCFEFF2D0AD17C
:10D5E800B10001F5D84120466131042203F029FC3D
:10D5F80023789BB970BDFE2D01D1173E02E0FD2DA9
:10D6080002D10136267009E0B60006F5D84061302F
:10D61800401903F005FCC0B2207020B10248BDE8F3
:10D62800704015F0F3BD70BDAC1B00202DE9F04132
:10D6380015F01EFE60B110208F49FBF763F98F4B80
:10D648001B78432B40F0EE81BDE8F04115F032BE67
:10D6580015F020FE002826D0894C23786BB11020C5
:10D668008849FBF74FF988482D211030F2F710FF51
:10D67800002800F0D781217810E010208349FBF7BB
:10D6880041F981482D211030F2F702FF04460028A5
:10D6980000F0C88115F016FE014620468222BDE83A
:10D6A800F041FBF755B97A4C43F6CC2223689B68C6
:10D6B800934250D0774E744D307803EB800003F0DE
:10D6C800AFFB032201467448FBF742F923689868C8
:10D6D80046F6C55398422BD0203B984228D0337841
:10D6E800013000EB830003F09BFB0322014605F1A8
:10D6F8001500FBF72DF9236830789B68023303EB9C
:10D70800800003F08DFB0322014605F11900FBF7A9
:10D718001FF9236830789B68033303EB800003F01C
:10D728007FFB0322014605F11D00FBF711F90EE00E
:10D738002D2103225948F2F72DFE2D2103225848A6
:10D74800F2F728FE57482D210322F2F723FE202363
:10D758002B772B762B75544B1B7813F0010F00F0A9
:10D76800BD80236843F6CC229B68444D934261D028
:10D778004E4E484F32783878D31803EB800003F0C8
:10D788004FFB4B4B0146186028789846A0F13002B1
:10D79800D2B2092A01D943280FD109B2BA22FCF71B
:10D7A80029FF236832789B680146C8F8000038785A
:10D7B800D31803EB800003F029FB2B782A2B04D124
:10D7C800337813B1394A013B13702B78232B0ED1D0
:10D7D8003378022B0BD8226846F6A55192688A4204
:10D7E80005D020318A4202D0304A013313702B7899
:10D7F800552B01D0442B0FD1236831789B68A3F5B2
:10D80800D843B3F1610248BFA3F15E023B7803EB52
:10D81800A202D0B2FFF7D8FE264B1B7803F0800394
:10D82800DBB23BB13278184B03EB820320225A74E7
:10D838009A74DA742B78532B06D023689A6843F6C7
:10D84800CC239A4240F0EE80FBF720F9236846F695
:10D8580061429B68934203D10E4B0220197806E07F
:10D8680046F6C552934227D10A4B00201978013158
:10D87800BDE8F0410AF030BDF0F402088418002039
:10D88800F0100020C7F30208F401002011F5020887
:10D89800BC180020491900200502002009020020B8
:10D8A8000D020020110200208919002053190020C0
:10D8B800601900204032002046F6A552934204D158
:10D8C800594B012019780918D2E746F6615293425C
:10D8D80040F0A880544B03201978C8E7236849F220
:10D8E80052629B6893423ED14F4E10204F49FBF73E
:10D8F80009F831784E4D01EB011101F5164152310D
:10D908001022284603F09DFA2B4605F110012A46FD
:10D918001078474F78B94749FAF7F4FF3846E721B6
:10D92800F2F7B6FD78B13178401B3818013103227F
:10D93800FBF70EF807E013F8010B10B9203003F8D5
:10D94800010C8B42E4D13C4D2B782A2B03D1307843
:10D95800FD21FFF739FE2B78432B63D130782368FC
:10D968000130C0B259E043F6CC229342324E1AD06D
:10D9780010203249FAF7C6FF33782A2B52D1304BA0
:10D988001B689B68A3F5D843B3F1610248BFA3F1B4
:10D998005E02254BFF211B7803EBA202D0B2BDE843
:10D9A800F041FFF711BE33781F4D552B04D12B786A
:10D9B800142B01D1033B2B703378442B05D12B78E2
:10D9C800122B02D1184B15221A702B78DFF87480AD
:10D9D8005901C918414401F5944100201F31FAF753
:10D9E80091FF08F59241102017312F78FAF78AFF36
:10D9F8003378112F8CBF032700272A2B05D12878CD
:10DA0800FE21C01BC0B2FFF7DFFD3378432B09D1DD
:10DA18002B78173BDF1B2368F8B2997CBDE8F041EF
:10DA280015F00EBCBDE8F08149190020CFF40208BA
:10DA3800F4010020DFD50208841800208DF40208C4
:10DA4800BC180020B8AB020810B50E4B1B78452B4C
:10DA580017D10D4B1A7842F006021A700B4A137848
:10DA6800032B0ED80A490B4C086844F823000133ED
:10DA7800137083680B60FAF74DFEBDE81040FBF7A2
:10DA880005B810BD841800208919002077190020D6
:10DA9800BC1800207819002010B50C4B044621460C
:10DAA800D8790DF006FC60B1204655210DF060FADA
:10DAB80048B120460DF0F2FAD0F1010038BF00203D
:10DAC80010BD022010BD022010BD00BF5619002055
:10DAD80008B50DF0DDFBC0B208BD00002DE9F04728
:10DAE800634B644C1A78994612F0010F624D65D069
:10DAF8002078FFF7D1FF614A2B181178604F93F80F
:10DB0800A831604E44293870336090460AD12D2BD5
:10DB180008D038B995F8A91101233B7031602078F5
:10DB2800FFF7D6FF98F80030552B10D133682D2B0E
:10DB38000DD03B785BB1013B514ADBB21370EB1857
:10DB480093F8A8114F4B20781960FFF7C1FF98F898
:10DB58000030232B19D14C4B20781B689B7C013B50
:10DB6800984212DA434B0130C0B21870FFF794FFA5
:10DB78003870281890F8A8313360444B9B7803F02C
:10DB88000203DBB20BB1FAF7B9FD98F800302A2B83
:10DB980014D1207890B1374B0138C0B21870FFF714
:10DBA8007BFF3870281890F8A8313360374B9B7882
:10DBB80003F00203DBB20BB1FAF7A0FD344EFCF719
:10DBC800F9FC237832789A4288BF337032780F3262
:10DBD800934202DD2E4A0F3B1370DFF8C480002702
:10DBE80030783818C0B2FFF757FF281890F8A831D6
:10DBF8000137102F08F8013F07D0254B1A78224B20
:10DC0800BA181B689B7C9A42EADB99F8003013F03B
:10DC1800010F13D01F4B1A781F4B02F08002D2B2AB
:10DC28002AB1227831781032521A5F2105E0227821
:10DC380031781032521A134909689954134DAB7848
:10DC480003F00203DBB25BB12078E91D652246F6DA
:10DC58006153FAF7A3FD05200B212A46FAF70AFEBD
:10DC680021780E4801310222BDE8F047FAF770BE6C
:10DC78008919002053190020A04C0208841800209C
:10DC88009C18002060190020BC180020981900205A
:10DC98004B19002040320020F4010020F50100203B
:10DCA8000302002038B5054600240123A3402A7842
:10DCB800E0B29A4205D10E49102246F6A553FAF76A
:10DCC8006DFD0134082CF0D1083C0A4BE0B2E31892
:10DCD8009A782B78934206D12BB10549102246F643
:10DCE800C553FAF75BFD0134042CEED138BD00BFF3
:10DCF80086180020561900202DE9F04107461046E5
:10DD08000D461446F2F796FDC3B28046B3B1AB4256
:10DD180014D80B4E20212A46F019F2F73BFB204677
:10DD2800F2F788FDC8EB05056D08EDB2EF1902465C
:10DD38002146F019BDE8F041F2F784BABDE8F08158
:10DD4800F4010020F0B5134B0C781A1895781F468B
:10DD5800E5B100233A1892781A4112F0010F4FF0FA
:10DD680001020BD0AC420E7803D09A4042EA060674
:10DD780002E09A4026EA02060E7004E09A400E7805
:10DD880026EA02020A700133082BE3D10B7803B9A3
:10DD98000C70F0BD5619002031220023017819417A
:10DDA80011F0010F02D00449C9180A750133013274
:10DDB800082BD2B2F2D17047F401002070B57B4B2A
:10DDC800044631B11B78532B40F0EF80533B03706E
:10DDD80070BD1A78302A34D1754A53785BB1754BC7
:10DDE80075491B78172000FB03135B7913F0100F9C
:10DDF80001D001235370714B20781978014012D05B
:10DE08009278002A40F0D1801978114111F0010F61
:10DE180005D001219140207820EA010121700132CA
:10DE2800082AF1D141E01A780A4112F0010F04D012
:10DE380001228A4020780243227001310829F2D158
:10DE480033E0A2F13101C9B2072938D858494A78D4
:10DE58005AB1584A58481278172505FB02025279D8
:10DE680012F0100F01D001224A701B78534A313B3F
:10DE78001278DBB21A4112F0010F00F09680227876
:10DE880052FA03F010F0010F09D08978002940F008
:10DE98008C80013111FA03F322EA030204E0012124
:10DEA80011FA03F343EA02022270002112224448C5
:10DEB800F2F770FA2046BDE87040FFF7F3BE132A68
:10DEC8000CD0552A17D13B4B3B4A1B78172101FB35
:10DED80003235B7913F0200F03D170BD344B01226B
:10DEE8005A7000202146FFF72DFF344B9B78002BFA
:10DEF8005BD0002051E0142A0CD02A2A17D12D4BD0
:10DF08002D4A1B78172101FB03235B7913F0200F9F
:10DF180003D170BD264B01225A7001202146FFF71C
:10DF280011FF264BDB78002B3FD0012035E0152A66
:10DF38000CD0232A17D11F4B1F4A1B78172101FB2E
:10DF480003235B7913F0200F03D170BD184B012216
:10DF58005A7002202146FFF7F5FE184B1B79002B5B
:10DF680023D0022019E0162A0CD0442A1DD1114BC7
:10DF7800114A1B78172101FB03235B7913F0200F4B
:10DF880003D170BD0A4B01225A7003202146FFF7C6
:10DF9800D9FE0A4B5B7943B103200949102246F6A2
:10DFA800C553BDE87040FAF7F9BB70BD841800206E
:10DFB8002F0E00204C190020CF33002056190020C6
:10DFC800861800202DE9F04F87B09DF84050804614
:10DFD800072D0E4605929A4637D1002427463378F6
:10DFE800234113F0010F2CD0012523B24FF0000874
:10DFF8000293512029462A462B460095CDF80480E5
:10E0080002F08CFF1B20414662194346CDF8008080
:10E01800F4F772FB37B9112039463A462B46009778
:10E02800F4F76AFB534B204613F8242001276FF3BB
:10E03800000203F824201199F5F7CEF92046F5F7E8
:10E04800D5FB0134082CCAD1F7E1012D03780CD196
:10E058000BB90B7823B3FF2300930021464B0191A2
:10E068001B780C200133029316E0022D09D10BB95D
:10E078000B78ABB10021FF2300930191029134206A
:10E088000AE0062D0CD10BB90B784BB10021FF2308
:10E09800009301910291652004220B4602F03EFF95
:10E0A800BAF1010F98F800302BD13BB1334B002067
:10E0B800D979024653460090F4F71EFB33783BB1FA
:10E0C8002E4B0120D979002203460092F4F714FB65
:10E0D8000020F5F773F998F80030002B5BD0284B37
:10E0E8001978002957D1274BDB78002B53D0FF2311
:10E0F80000933A2001220B460191029102F00EFF93
:10E1080049E063B1052D4FF0000102D100910F20C5
:10E1180001E000910B200A460123F4F7EDFA337869
:10E1280083B1052D4FF0000106D110200A460123C6
:10E138000091F4F7E1FA12E00C200A46012300915D
:10E14800F4F7DAFA022D25D0032D01D10E4B02E0A7
:10E15800042D02D10D4B1F781DE0052D01D10C4B6C
:10E16800F9E7012D01D1044BF5E7062D0CBFFF2778
:10E17800002710E028150020091600205619002055
:10E18800161500202F0E0020601B0020973B002052
:10E198003F360020FF2798F80030002B00F09D80C4
:10E1A800914C237803F02003DBB26BB18F4B1978C5
:10E1B80011F0010108D1FF230093282001220B460A
:10E1C8000191029102F0AAFE237803F01003DBB25A
:10E1D80073B1864B197801F00201C9B241B9FF2326
:10E1E8000093292001220B460191029102F096FE2C
:10E1F800E37813F0010F0ED07C4B197801F004017D
:10E20800C9B241B9FF2300932A2001220B4601918C
:10E21800029102F083FEE37803F00203DBB273B1EC
:10E22800724B197801F00801C9B241B9FF23009374
:10E238002B2001220B460191029102F06FFEE37838
:10E2480003F00403DBB273B1684B197801F01001D5
:10E25800C9B241B9FF2300932C2001220B4601913A
:10E26800029102F05BFEE37803F00803DBB273B1BE
:10E278005E4B197801F02001C9B241B9FF23009320
:10E288002D2001220B460191029102F047FE0FF06A
:10E29800C3FA70B1554B197801F04001C9B241B9C0
:10E2A800FF230093492001220B460191029102F0BD
:10E2B80035FEE37803F04003DBB273B14B4B1978BA
:10E2C80001F08001C9B241B9FF2300934E20012219
:10E2D8000B460191029102F021FE119B444A1978E4
:10E2E800444B51B198F80010117032781A70337895
:10E2F8000BB1542005E0522003E01170327853200E
:10E308001A7003F0EBF9119B00241A783A4B1A7033
:10E3180098F80030234113F0010F2DD021460598BD
:10E3280014F0FDF90122014628B923B201900092A8
:10E338000293104605E0002123B200920191029356
:10E3480024200B4602F0EAFDBAF1010F05D12B4B50
:10E358008020DA790521013208E0022D07F1010257
:10E3680002D18020072101E0802006212346F5F70D
:10E378004DFD2046F5F70EFA3378234113F0010FCF
:10E3880057D000214FF0010B23B2029302205A46C6
:10E398000B46CDF800B0019102F0C0FDDA45DFF878
:10E3A80068900CD119F8243013EA0B0334D1134ABE
:10E3B8000520D1790093594404EB0B022AE019F89F
:10E3C800243013F0010327D1022D1FD10C4B1B78E9
:10E3D80003F02403042B04BF0A4B83F800B0002386
:10E3E8000093072014E000BF40320020CB16002025
:10E3F8007415002075150020E81600205619002015
:10E40800F2160020280E0020281500200093062070
:10E41800791C621CF4F770F911992046F4F7DCFFB7
:10E428002046F5F7E3F919F824306FF3000309F8EB
:10E4380024300134082C7FF46BAF07B0BDE8F08FAF
:10E448002DE9F04180460E46174646F28B750024AA
:10E458003846214614F063F988B1294608220B484A
:10E4680002F0EFFC0948414614F006F9074814F099
:10E4780029F920B90123A3403278134333700134BA
:10E488000835082CE4D1BDE8F08100BFE016002073
:10E498002DE9F04387B08046894604A847F2B511B4
:10E4A800082202F0CEFC002440462146E7B214F0D0
:10E4B80036F9002843D03846F3F75AFE0025661C83
:10E4C8000246314611202B460095F4F715F9012331
:10E4D80021462A460420FF080095F4F70DF94AF270
:10E4E800B340381802F09CFC04F00703C1B219418C
:10E4F80011F001014FF002024FF001030AD000921F
:10E50800019336B27720294692182B46029602F0DC
:10E5180005FD14E00092019336B2232004220B4635
:10E52800029602F0FBFCB9F1000F08D004A82146BE
:10E5380014F0F5F818B10548214614F0DAF801345A
:10E54800402CB1D107B0BDE8F08300BF51150020C1
:10E558002DE9F74F174698463B7805460C469DF837
:10E5680030909DF834B09DF83820DFF8B4A043B15E
:10E5780002EA03033B7009789AF800208A18D31A34
:10E588000370237883B121482146F5F7DBF8204949
:10E598001E4814F071F81D480121FFF779FF1B4848
:10E5A80041462246FFF74CFF1A4B00261E70297879
:10E5B80043F6F72002F02AFC494646F2C96002F009
:10E5C80025FC204639464A46F4F7BCFE124B39462C
:10E5D8001E7142464B462046CDF800B00195FFF724
:10E5E800F1FC2846F7F7BEFD2B780C480C498AF851
:10E5F8000030F5F7A7F888F800603E7026702E7096
:10E6080003B0BDE8F04F02F079BF00BFE916002063
:10E618006C150020881900202F0E0020CC16002031
:10E628001615002010B50B4B0B4C024603CB20608F
:10E6380061600A48114614F040F82146074814F072
:10E648001BF8064814F03EF8D0F1010038BF00204E
:10E6580010BD00BFF8250020D6160020E0160020C7
:10E6680010B50A4C637C4BB100200949FAF74AF906
:10E67800084B1B78432B01D1433B6374607C20B962
:10E688000549BDE81040FAF73DB910BD86180020CD
:10E6980021D602088418002000D60208034B1A78F5
:10E6A80001321A7001230370704700BF88190020D7
:10E6B80010B50C48FAF7CCF80B4A002414700B4A32
:10E6C8000B4B14700B4A5C7114700B4A1C7114705C
:10E6D8000A4A5C7014700A4A1470FAF7D7F9094BA1
:10E6E8001C6010BD981900205619002085180020BC
:10E6F8002F0E00208A19002096190020C01800202B
:10E7080088190020BC1800202DE9F04F934B944E37
:10E7180093F800903368DFF894829C7C914BF02248
:10E728001A7098F800308BB00C2B354647463DD10F
:10E738008D4B93F805C0BCF1010F02D900208B491D
:10E748002FE01AD100245C71894A8A4B8A498B4888
:10E758008B4D04701C7014700C70CDF800C00194BF
:10E768002D780295FFF7F4FEFAF790F985483460A2
:10E778000BB0BDE8F04FFAF76BB883487E49F4F761
:10E78800E1FF824B824A03CB824B10601B785160B9
:10E79800532B57D198F800307F49013388F800305F
:10E7A80000200BB0BDE8F04FFAF7ACB8082B0FD13A
:10E7B800784B1B78532B3DD1784B00221A700C23D1
:10E7C80088F80030764B1A7842F006021A707FE219
:10E7D8000D2B37D16F4B1B78532B2BD171496A48BE
:10E7E80013F04AFF6848FFF71DFF044640B198F848
:10E7F80000300522013B88F800305B4B5A7167E214
:10E80800082246F2CA61624802F01BFB604966486A
:10E8180013F053FF01230093594B01941B78574879
:10E8280002935549524A534BFFF792FEFAF72EF9D5
:10E8380034604DE2232B40F04B820BB0BDE8F04F23
:10E84800FFF736BF631E48BFA31DDB10013303FB70
:10E8580009F91FFA89F909F5CC46A9F5B649A9F1CC
:10E868004D094F4BCDF81C901A78CA3612F0010F9B
:10E878004A4C00F01E81474B1A789946432A40F0CB
:10E88800C7803B780C2B40F0C3803F48217813F0B9
:10E8980046FF002800F0BC803D48217813F03FFF78
:10E8A800002840F0B580079920780FFA81FB0BEB20
:10E8B800D00002F0B5FA23784FF0010A03F00702FE
:10E8C8000AFA02FADFF8E8805FFA8AFA10EA0A0F11
:10E8D800C8F8000027D0244BDB78002B40F0988044
:10E8E800274BD879F7F79CFB002800F09180D8F8DF
:10E8F8000010CAF1FF0A20780AEA0101C8F80010DE
:10E908000BEBD00002F082FA20780FFA86FB0BEBB3
:10E91800D00002F085FA00EA0A012078C8F8001051
:10E928000BEBD0005FE032B202EBD300059202F0AD
:10E9380077FA10EA0A0FC8F800003BD140EA0A014A
:10E94800059B2078C8F8001003EBD00002F05EFAAF
:10E958002178154813F0CDFE5AE000BF4919002070
:10E96800BC180020951900202F0E0020C6D60208DA
:10E978008A1900208518002096190020C018002048
:10E988005619002098190020E9160020F8250020C3
:10E998000C150020841800208CD702085319002079
:10E9A80089190020611500206C15002088190020A5
:10E9B80060190020924BDB7823B9924BD879F7F78E
:10E9C8002FFBB8B92078DDF814C0CAF1FF0A0CEBA8
:10E9D800D00002F025FA8C4A00EA0A01059B20784B
:10E9E800116003EBD00002F011FA2178874813F088
:10E9F8008BFE0DE020780BEBD00002F011FA40EA14
:10EA08000A012078C8F800100BEBD00002F0FEF9DC
:10EA180099F80030232B10D12A682378927C013A88
:10EA280093420ADA7A4A013313707A4B9B7803F0DF
:10EA38000203DBB20BB1F9F761FE99F800302A2B1B
:10EA48000CD1237853B1724A013B1370714B9B78F8
:10EA580003F00203DBB20BB1F9F750FE99F800306E
:10EA6800552B12D129682278897C694B08398A424A
:10EA780001DA083200E000221A70664B9B7803F036
:10EA88000203DBB20BB1F9F739FE99F80030442BD9
:10EA98000FD122785E4B072A9CBF2A68927C083ADD
:10EAA8001A705C4B9B7803F00203DBB20BB1F9F7E9
:10EAB80025FEFBF77FFD584A237811789246994244
:10EAC80088BF137012780F32934202DD524A0F3B0F
:10EAD80013702B684FF0000B93F81280CDF818B024
:10EAE800B8F10F0F9ABFC8F120085FFA88F84FF005
:10EAF800100839784FFA8BF30C2905D19AF80020C1
:10EB08009B18DB10454A04E09AF800209B18444AF9
:10EB1800DB10D35C9AF8002005934FFA8BF39A1810
:10EB28000C2902F007094FEAE20202D13D49895C4B
:10EB38000691DDF81CC004930FFA8CF0101802F04F
:10EB48006FF9C0B2049B08909AF8000032B2181806
:10EB580002EBE00002F064F939789AF80020049B8F
:10EB6800C0B209919A1846E0059BDDF824C043FA23
:10EB780009F12D4B01F0010100290CBFA521DB2172
:10EB8800BCF10C0F03F8081014D128494FEAE20C25
:10EB980011F80C1041FA09F111F0010F08D0DDF855
:10EBA80018C04CFA09F111F0010F03D0582110E0F8
:10EBB8002D210EE0DDF820C04CFA09F111F0010F0B
:10EBC80001D0502105E040FA09F111F0010F02D0FF
:10EBD800542103F8081009F101095FFA89F90BF1CA
:10EBE800010B08F101080132B9F1080F5FFA8BFB3C
:10EBF8005FFA88F81CD0B8F1200FB5D125E000BF26
:10EC08002F0E002056190020601900206C150020D6
:10EC180053190020981900204B1900206115002075
:10EC2800C11500200C150020F4010020E916002071
:10EC3800B8F1200F09D09AF800304FFA8BF2D218A9
:10EC48002B689B7C9A42FFF654AF23490B7813F04C
:10EC5800010F17D02B68214A9B7C12780F2B02F0EA
:10EC6800800298BFC3F11003D2B294BFDBB2002375
:10EC780042B122789AF800101032521A1849CB186B
:10EC88005F219954174EB37803F00203DBB293B1B6
:10EC9800F11D652246F661432078F9F77FFD2B6860
:10ECA8009B7C102B02D905200B2101E000200721B5
:10ECB8003246F9F7DFFD2B689B7C102B08D92178A9
:10ECC8000948013102220BB0BDE8F04FF9F740BE08
:10ECD8000BB0BDE8F08F00BF89190020403200203A
:10ECE800F401002098190020F50100202DE9F043D7
:10ECF800002387B08DF81730754B1B78012B00F077
:10ED08006082744B1A78984672B1734BDB78002B8B
:10ED180040F05782714C2378002B40F0A780F9F718
:10ED2800B5FE08232370A1E06C4B19781C4607290F
:10ED380000F29C806A490978232913D11A70F9F7DF
:10ED4800A5FE6849684A0B7853B16848013B0478C6
:10ED5800DBB244F0060404700B70654951F82330A7
:10ED680013609FE2614B1A7812F0010F04D1012160
:10ED78000A438DF817101A70F4F7F0F828B92378B9
:10ED88001BB90DF11700FFF789FCF4F7F5F830B956
:10ED98002378012B03D10DF11700FFF77FFCF4F75F
:10EDA800F9F830B92378022B03D10DF11700FFF7DA
:10EDB80075FCF4F7FBF830B92378032B03D10DF178
:10EDC8001700FFF76BFCF4F7FFF848B9F4F718F9E8
:10EDD80030B92378042B03D10DF11700FFF75EFC3F
:10EDE800F4F74CF930B92378052B03D10DF117004E
:10EDF800FFF754FCF4F736F930B92378062B03D122
:10EE08000DF11700FFF74AFCF4F7ECF830B9237856
:10EE1800072B03D10DF11700FFF740FC9DF81730C1
:10EE280023B32378072B1FD8DFE803F004070C0F60
:10EE38001215181B00202F4901E02F490020F9F76F
:10EE480061FD13E000202D49F9E700202C49F6E781
:10EE580000202C49F3E700202B49F0E700202B493C
:10EE6800EDE700202A49EAE7F9F710FE1B4F3B7847
:10EE78003D46082B40F0B0801C4E194F317811F0F8
:10EE8800010151D1234C12222046F1F783FA0123C4
:10EE98006374214A98F80030137003B96374637C73
:10EEA80013B11E4B00221A70FFF7DAFB1A48617C77
:10EEB800FEF784FF337803F0FD0343F0010333705A
:10EEC800174B1A7872B33A7000221A702CE000BF00
:10EED80095190020161500202F0E002088190020F3
:10EEE8008418002077190020BC18002089190020F8
:10EEF8007819002072DC020851DC020893DC020851
:10EF0800B4DC0208D5DC0208F6DC020817DD0208CA
:10EF180038DD020886180020C0180020280E0020BE
:10EF28004D19002030233B703B78884E13B9737815
:10EF3800102B4DD1DFF86492854CFFF791FB844884
:10EF480099F81110FEF73AFF237823B10020102119
:10EF58004A46FEF7D1FE98F8003024787D4A24EA24
:10EF6800030111707C4A23EA040111703A78A2F176
:10EF78005200C0B2012803D97078744F10280CD100
:10EF8800002373701CB911B10133009311E10423FC
:10EF980073712B7801332B701AE0432A18D1BBB94F
:10EFA800FC78ACB96D4BD879F7F73AF838B96C49B1
:10EFB800F9F7A8FC05237B7107332B7004E0204682
:10EFC8006849F9F79FFC7C71674A684B1A6069E1E8
:10EFD8005F48FEF7E1FE65E1092B31D15D4808F095
:10EFE80071F9C6B2594C36B36379042B02D10020AB
:10EFF8005F4903E0022B04D15E490020F9F782FC47
:10F0080002E00BB904336371314602225A48F9F71A
:10F018009FFC5A4B1E78232E00F0D3803046F9F718
:10F028002DFD002800F03E81312E40F03B812B78E9
:10F0380001332B7002E03B7801333B70042332E04C
:10F048000A2B32D1434808F023F9C6B23F4C36B3F5
:10F058006379042B02D10020494903E0022B04D133
:10F0680048490020F9F74EFC02E00BB904336371FC
:10F07800314602224048F9F76BFC404B1E78232E9C
:10F0880000F09F803046F9F7F9FC002800F00A816B
:10F09800312E40F007812B7801332B7002E03B784A
:10F0A80001333B7008236371FCE00B2B40F0FA80BE
:10F0B800284808F0D3F80021C4B2264808F0A4F87C
:10F0C800002C6DD0214E33792BB9BE2014F014F9E1
:10F0D80033790133337173791C4A092B02D9002023
:10F0E8001F4915E010D11D4B00241C705471264B8C
:10F0F800194A1849164801251C7014700C700470C0
:10F108000095019402949EE0082B04D11F49002029
:10F11800F9F7F8FB11E0062B02D100201C49F7E7AC
:10F12800042B02D100201B49F2E7022B02D1002058
:10F138001949EDE70BB9083353717379082B3CD89B
:10F148000D4821460222F9F703FC36E02F0E002075
:10F15800C0180020961900208A190020561900208E
:10F16800C6D6020842D602084C4E0208BC18002037
:10F178004AD702086BD70208F4010020841800203F
:10F1880008D7020829D702088518002063D6020884
:10F1980084D60208A5D60208E7D6020886180020F9
:10F1A800012542484249434A2B460095F4F77CFC26
:10F1B8000095414B01941B7840E0404F3C78232C4C
:10F1C80002D1FFF775FA6DE02046F9F757FC0028E1
:10F1D80068D0303CE4B2631EDBB2012B3C7039D8F6
:10F1E800022C354D1ED1E879F6F71AFF002838D0E1
:10F1F8002E48FFF717FA002833D1082246F2CA61D1
:10F208002F4801F01EFE29492D4813F040FA2C49D9
:10F21800082246F2CA6001F00EFE2949294813F077
:10F228004CFA06E0012321482149224A0093F4F7C9
:10F238003BFC01230024009301942B78029322487D
:10F248001C49224A1A4BFFF783F9F9F71FFC204B98
:10F258001C6027E0032C25D1174BD879F6F7E0FE80
:10F2680010B90C2373711DE000241048214613F0D7
:10F2780056FA28B1E02014F03FF8204614F078F848
:10F288000134402CF1D1134A0023137073712B7889
:10F29800114A01332B700E4B1A60104B1A7842F04A
:10F2A80006021A7007B0BDE8F08300BFE916002017
:10F2B800851800209619002056190020841800206F
:10F2C8000C1500206C150020C01800208A19002099
:10F2D800BC180020531900204C4E02088919002040
:10F2E8001FB5044611B100200B4901E008460B493F
:10F2F800F9F708FB217810220139C9B201EB011195
:10F3080001F5C2414431684601F09BFD10200146D9
:10F318006A46FEF7F1FC1FBDC8AD02080AAE020836
:10F328000B4B1B78442B06D0552B037801D013B117
:10F338007047013B01E003780133037003780BB990
:10F34800403302E0412B01D1403B0370FFF7C8BFB7
:10F35800841800202DE9F74FDFF8C881DFF8D4A121
:10F3680098F80030554643F0010388F800309AF8C1
:10F378000130624C23F07F039B46D3B100206049E3
:10F38800F9F7C0FA5F482A21F1F782F818B1217815
:10F398008222F9F7DDFA2278002A40F0AB802B6848
:10F3A80062F3CF332B60584B1A7842F003021A707D
:10F3B800A0E0DFF85491237099F800304E4603F02E
:10F3C8000202D2B20192514F002A40D013F0010834
:10F3D80013D058464E49F9F795FA3B78232B20D19C
:10F3E8004C4B4D4A4D481A600121FFF779FF33789D
:10F3F80003F0FE036BF3410312E040464849F9F776
:10F4080081FA3B78232B0CD1424B434A43481A607C
:10F418000121FFF765FF337868F3000368F34103C0
:10F4280033703B782A2B65D1337803F0FE036FF3F2
:10F43800410333702B6843F400432B600F23237080
:10F44800364B187803B0BDE8F04F0DF073BC0DF0E3
:10F45800BBFB054600282DD001213048FFF760FF8F
:10F468003B78532B12D13378019A03F0FD0362F3F2
:10F4780000033370DAF8003043F40043CAF8003070
:10F488000F232370254B18780DF054FC3B78232B61
:10F4980030D13378002203F0FD036FF3000333709B
:10F4A8001E4B1A70F9F7F2FA1E4A137843F0060356
:10F4B800137015E01C49F9F725FA3B78232B19D16D
:10F4C80099F8003065F3410365F3000389F80030CB
:10F4D800F9F7DCFA98F8003043F0060388F80030B2
:10F4E800124A1378013BDBB21370114A52F82320F9
:10F4F800084B1A6003B0BDE8F08F00BFA23C0020A3
:10F508004CAE0208F40100204B350020841800207E
:10F518006DAE0208BC180020684E0208531900207E
:10F528008EAE020889190020AFAE020877190020B4
:10F5380078190020403200202DE9FF412C4D2D4C38
:10F548002B7843F001032B70217801F00401C9B234
:10F5580011B92948FFF7E4FE284E3378232B21D12F
:10F568002378274F13F004080AD0224A6FF3820346
:10F578001370244B20483B600021FFF7B1FE11E0D7
:10F58800F9F784FA2B78204A43F006032B70137896
:10F59800013BDBB213701D4A52F823303B60164B17
:10F5A80083F800803378532B1FD12378052243F04A
:10F5B80004032370104B16491C78013CE4B204EB99
:10F5C800840000F5CA40843001F035FC0020114960
:10F5D800F9F798F9FF23002100930134162004223B
:10F5E8000B460191029401F099FCBDE8FF8100BF30
:10F5F800891900204B350020531900208418002059
:10F60800BC180020844E02087719002078190020C1
:10F61800A04E02082BAE02082DE9F041984B044693
:10F628009A7812F0010F00F017811B88002B40F028
:10F638001381944D95F820303F2B40F2D780012C50
:10F6480014D1914B1B7803F00203DBB2002B00F0BE
:10F65800C48095F820208B4B402A03D1013283F8CF
:10F668002020FBE0482283F82020B6E0022C03D1BA
:10F67800482385F82030B0E0844E337803F0200228
:10F68800D2B28AB195F82020402A0DD1032C0BD094
:10F698007F4B804A03F1100153F8040B8B4242F868
:10F6A800040BF9D1412395E003F01003DBB28BB1D1
:10F6B80095F82030412B0DD1032C0BD0764B754A91
:10F6C80003F1100153F8040B8B4242F8040BF9D1F3
:10F6D80042237FE0F37813F0010F0FD095F8202034
:10F6E800422A0BD16D4B6B4A03F1100153F8040BFE
:10F6F8008B4242F8040BF9D143236BE003F002027A
:10F70800D2B27AB195F82020432A0BD1644B614AD2
:10F7180003F1100153F8040B8B4242F8040BF9D1A2
:10F72800442357E003F00402D2B27AB195F82020BE
:10F73800442A0BD15B4B574A03F1100153F8040BD1
:10F748008B4242F8040BF9D1452343E003F0080348
:10F75800DBB28BB195F82030452B0DD1032C0BD0A3
:10F76800514B4C4A03F1100153F8040B8B4242F8F9
:10F77800040BF9D146232DE00EF04EF8A0B14B4B07
:10F788001B788BB195F82030462B0DD1032C0BD06C
:10F79800474B404A03F1100153F8040B8B4242F8DF
:10F7A800040BF9D1472315E0F37803F04003DBB2EB
:10F7B8009BB195F82030472B0FD1032C0DD03D4B32
:10F7C800344A03F1100153F8040B8B4242F8040B3E
:10F7D800F9D1482385F8203078E095F820300133B6
:10F7E800DBB2472B85F820307FF629AF95F82060EB
:10F7F800472E04D9234B002683F8206001E0013608
:10F80800F6B206F14007FFB212E02B48314612F07B
:10F8180086FF08B1032C04D1284B9B5D23B1032C30
:10F8280002D185F820600FE00136F6B2BE4203D05F
:10F838003F2EEAD9402E07D1214B1E221A704023B1
:10F8480085F82030BDE8F08195F82000114965223F
:10F8580046F66143F8F7A2FF012C37D1194B0D4A40
:10F8680003F1100153F8040B8B4242F8040BF9D151
:10F87800044B93F820303F2B3CD9002012493EE03E
:10F8880098190020F40100201715002040320020AC
:10F8980000B502089F19002021B5020842B50208E8
:10F8A80063B5020884B50208A5B50208A037002090
:10F8B800C6B5020808B60208C11500207715002051
:10F8C8005419002000180308BEB40208104BD87859
:10F8D80000F02000C0B220B1022C06D000200D4953
:10F8E8000DE0032C01D10C4909E00C4B93F82030B2
:10F8F8003F2B02D800200A4901E00A490020F9F705
:10F9080001F81020084A0146BDE8F041F8F7B2BFF7
:10F9180040320020D9AB0208DFB40208F40100200D
:10F928007CB40208E7B502089819002010B5F9F769
:10F93800ADF8084B1B7803F00403DBB22BB1064982
:10F948000020BDE81040F8F7DDBF0220BDE81040F8
:10F95800FFF762BE17150020AEB2020870B5224B41
:10F9680006461B78214CF3B9257819E0204829462A
:10F9780012F0D5FE78B123689D4202D9FF2E02D03D
:10F9880007E0FF2E02D19D4208D202E036B91DB928
:10F9980013B9256012E00EB9013500E0AD19EDB2DA
:10F9A8003F2DE3D90AE0013B2021124810222360B1
:10F9B800F0F7F0FC00201049F8F7A4FF0F48F8F71B
:10F9C80047FF46F6614320780D496522F8F7E6FEC1
:10F9D800084D216805F1100001310222F8F7B8FF3F
:10F9E8002D23AB7470BD00BF491900206019002099
:10F9F800C2180020F40100207CF6020898190020A3
:10FA08009F190020F8B5544BF02254481A70037817
:10FA1800044613F00E0518D1514A43F0020315604D
:10FA280000F8013B12F020FE2C464E4BE35C1BB164
:10FA38004D48214612F05DFE0134402CF5D14B4B68
:10FA48001A7842F001021A70F8BD13F00C0543D180
:10FA58002E464548294612F062FE08B10136F6B234
:10FA68000135402DF5D11EB9237843F0040331E068
:10FA780000253F482946EFB212F051FE68B1394BD4
:10FA8800EB5C53B13B4B01371F700020FFF766FF5B
:10FA9800237843F00803237002E00135402DE8D1B4
:10FAA800354D3A212846F0F7F3FC38B1401BC0B277
:10FAB8000130281831460222F8F74AFF2F4B1B78ED
:10FAC800532B47D12B4B00201870FFF747FF2378A3
:10FAD80043F008032370F8BD6FF34103037003F08C
:10FAE8000403DBB2254D23B100202549F8F70AFFAE
:10FAF8000EE02B78552B01D1FF2002E0442B02D1D8
:10FB08000120FFF72BFF13200D211E4AF8F7B2FE44
:10FB18002B78232B1ED1227802F00204D4B90F4986
:10FB280002F0FB0264F3C3020A700D4A1460F8F78E
:10FB3800ADFF0E4B1A7842F006021A70124A13787B
:10FB4800013BDBB21370114A52F82320104B1A60A4
:10FB5800084B1C70F8BD00BF95190020C118002083
:10FB68006019002068240020C2180020891900208C
:10FB78001815002049190020F401002084180020DD
:10FB8800C207030898190020771900207819002067
:10FB9800BC18002070B505460C4616463BB143001C
:10FBA8004AF28D3018184018114601F02FF9054B0C
:10FBB800172202FB0535F3092C1906F07F0663703E
:10FBC800E67070BDCF33002038B510B3A0F1410303
:10FBD800DBB2432B1FD9C50900F07F040BD0052CDD
:10FBE80019D90021601E0A460AF0E6FBD0F101008F
:10FBF80038BF002038BD082C0FD9601EC0B2294676
:10FC08002A460AF057F850B9402C8CBF0020012032
:10FC180038BD012038BD002038BD284638BD2846EB
:10FC280038BD0000F7B5614C31232374604F0133B0
:10FC38002376053B637463763B784AF28D305B002C
:10FC4800181801F0EDF8C0B220F07F0200F07F0133
:10FC5800D2B28DF804108DF8002004F1120359B9BE
:10FC6800544A04F115001188927861829A70202113
:10FC78000222F0F78FFB0CE0D20904EB8202526AF1
:10FC880010886082927804F115009A700222F8F7C1
:10FC98005FFE3878400000F5224000F5C77001F09B
:10FCA800BFF8C0B220F07F0300F07F01DBB28DF80F
:10FCB80005108DF80130404851B93E4B20311A8863
:10FCC8009B786283837002220330F0F763FB0BE0BA
:10FCD800DB0904EB83035B6A1A8862839B78022240
:10FCE80083700330F8F734FE344B1B7813F0010FA0
:10FCF8005AD0334D02A92A788B1813F8041C13F82C
:10FD0800086C304B1B78232B04D1002A41D1223BAD
:10FD18002B703EE02A2B04D1002A3AD0013A2A70EF
:10FD280037E0552B46EA010611D10DE02B7802AADF
:10FD3800D318013E13F8081CF6B23046C90913F867
:10FD4800042CFFF741FF98B9002EEFD121E0442B96
:10FD580019D115E02B7802A9CB18013613F8081C25
:10FD6800F6B23046C90913F8042CFFF72DFF38B155
:10FD7800134B3878197832460123FFF70BFF08E058
:10FD8800902EE7D905E0532B03D1533B2B70FAF79C
:10FD980011FC0D4B1B7803F08003DBB223B12B78E9
:10FDA8002022023304F83320FEBD00BFF4010020F6
:10FDB80049190020BF1303080E02002089190020EA
:10FDC80053190020841800204032002002480021E6
:10FDD8000922F0F7DFBA00BF6519002070B50A469E
:10FDE800002405E01B19811A2A2501345D54E4B268
:10FDF8000E4D0F4B295D09B19442F3D1801A0019B9
:10FE080018182021121BF0F7C5FA0A4B1E785EB1AC
:10FE1800432E04D10CB1013CE4B200232B553046EB
:10FE2800F8F72CFE00B12E5570BD00BF65190020F3
:10FE3800F40100208418002038B5184C184DA0781B
:10FE480000F01000C0B250B91649F8F75BFDFFF793
:10FE5800BDFF236843F4801323600F232B702A7897
:10FE68002AB92368FF2062F31453236038BD0E4873
:10FE7800C5792DB91C200821FFF7B0FF284638BDE9
:10FE880023680A496FF3145308222360F0F702FD30
:10FE980000280CBF0120FF2038BD00BF40320020E1
:10FEA8009719002011B3020865190020FE320308D3
:10FEB800F0B55B4C85B0667806F01006F6B2002EF9
:10FEC8003ED1584B1A78584B013A53F82230574ACA
:10FED800934204D1564B1A7842F0020207E002F12D
:10FEE8001C018B4208D1524B1A7842F004020221BD
:10FEF80061F3C7021A7019E03832934216D1FFF73E
:10FF08009BFF002800F08A800128494D06D12B78F4
:10FF1800022243F0010362F3C70306E03046454975
:10FF2800F8F7F0FC2B7866F3C7032B70424B1A786E
:10FF380042F001021A70236843F4805323606DE095
:10FF48003B4D2B7813F0F80606D03C49002005B04D
:10FF5800BDE8F040F8F7D6BC13F0070F3FD003F028
:10FF68000202D7B24FB1122031460EF01DFEFF2318
:10FF7800009301960296432028E003F00406F6B2A7
:10FF880096B1394638460EF00FFE0EF025F809F006
:10FF9800A3FC0CF041FEFF23009301970297442035
:10FFA800394604223B4614E013F0010F13D0012117
:10FFB80043F61C600EF0F8FD3046F6F79BF8204B30
:10FFC80045201E80FF2300930196029631460422A5
:10FFD800334600F0A3FF00201A49F8F793FC2B786A
:10FFE80003F0FA036FF341032B70174B1B78232B95
:08FFF80014D123686FF30C33F0
:020000040801F1
:100000002360F8F747FD0E4B1A7842F006021A708B
:10001000064A1378013BDBB21370054A52F82320DD
:100020000C4B1A6005B0F0BD40320020771900205B
:1000300078190020A84E0208253A002032B30208A1
:10004000891900205E0B03089A1800203D0B030855
:1000500084180020BC1800201FB50446F6F73AF9B2
:10006000A8B14B2001F03EFBFF2300930121FF3B91
:100070000193392004220B460134029400F052FF10
:10008000064B01205A7842F004025A7004E0044BF7
:100090001888003818BF012004B010BD3835002082
:1000A000B83C0020F0B5204E0024337A05460133D9
:1000B00085B00F463372102021460122234600945A
:1000C000F2F71EFB55B9FF2300934F202946042267
:1000D0002B460195029700F025FF0EE0012D0CD173
:1000E000FF230093502023462146042201940297C7
:1000F00000F018FF337A013B3372337A052B11D1AC
:10010000FA3301210024009327200B460422019496
:10011000029400F007FF044B1C7205B0BDE8F040EC
:1001200001F0B2BA05B0F0BD56190020074B1722F6
:1001300002FB00335B7913F0100F05D0044B163A25
:100140009A715A7009329A70704700BFCF330020FD
:100150002F0E00202DE9F04F9A4B87B01A780746F2
:1001600099461AB1012A40F0E68130E0964B1A68B0
:10017000964B9A4200F0E181F5F732FD944B5B78A3
:1001800003F00203DBB253B9924B5B7803F08003B8
:10019000DBB223B901F09EFA08B909F0A1FB8E4B3E
:1001A0001A686FF310421A608C4B1878F8F76AFCE3
:1001B000002800F0C281FFF70DFE894B3C221A7027
:1001C000F8F7ACFA99F80030013389F80030844B25
:1001D0001C7874B9834B791C1A78204664F3C302E7
:1001E00064F304121A70C9B2FFF75CFF89F800408B
:1001F000A3E17D4D384609F0ABFBF8F783FA002008
:100200007A49F8F783FBDFF8F4812B78AA46434458
:1002100013F8313C23B91B200621FFF7E3FD8CE1E5
:10022000704A0B21137804A8C3F3C004C3F300166B
:1002300003F0F7036FF304131370002389F8003001
:10024000062200F002FE2A78414604A8303AEFF771
:10025000CBFF804628B14FF000084FF01209454609
:100260002AE049F23F6000F0DFFD0028F3D0604D46
:1002700085F80880F5F714FE0446002840F05D81FB
:100280005C4A514B21461A60FF2300930190029073
:1002900004220820234600F045FE012223460E20BA
:1002A00021460094F2F72CFA534B1A7842F00402DC
:1002B0001A700123AB7140E14946062204A800F000
:1002C000C4FD9AF8002004A84C49303AEFF78CFF9F
:1002D000002840F021812846FFF7BEFE002840F0AC
:1002E0002C81DFF80CB101218BF808002846F5F7C6
:1002F000E5FD8146F5F7D4FDDA46002840F0B580EB
:1003000048463F49F0F74EF9B0B901F0FBF82E4BE3
:1003100014B916B93B4A23E036B13B4A1A603B4B4D
:100320001A786FF3410205E0394A1A60374B1A78A0
:1003300066F341021A70D7E048463649F0F732F9C1
:1003400020B148463449F0F72DF970B9002C40F03F
:10035000F480002E40F0F18001F0D4F82F4A1A4BBF
:100360001A603846FFF7E2FEBEE048462C49F0F737
:1003700019F950B949F23D60012100F04BFD164AD0
:10038000136843F400531360E0E748462549F0F74B
:1003900009F938B9002C40F0D080002E40F0CD8013
:1003A000214A0CE048462149F0F7FCF8002841D1E9
:1003B000002C40F0C280002E40F0BF801C4A024B4F
:1003C0001A6091E0B8180020BC180020FC4E02080A
:1003D0002A2C0020473500204032002084180020BD
:1003E0009719002064190020A0180020B8AB02085B
:1003F00056190020184F0208A1210020651900207D
:100400008934030864510208EC520208891900205B
:1004100008530208053403089536030824530208DC
:1004200040340308423403085C5302085236030880
:10043000B053020848464249F0F7B4F8002853D1B7
:1004400001F060F83CB13F4A3F4B1A603F4B1A78CD
:100450006FF3410270E0002E6FD03D4A3A4B1A60B4
:100460003A4B1A7864F3410266E048463449F0F7A3
:1004700099F8064620B901F045F8002C5DD01BE044
:1004800048463449F0F78EF8002856D0484632499D
:10049000F0F788F838B9002C4FD1304A2A4B8BF846
:1004A00007501A6049E048462D49F0F77BF80646A8
:1004B00050B9A4B101F026F8224A234B1A60234B0D
:1004C0001A7866F3410237E048462649F0F76AF8A1
:1004D00020B148462449F0F765F800B96CBB234ABF
:1004E000194B1A6001F00EF808F56A5078308AF856
:1004F000075000F099FC8AF800009AF8070000F510
:10050000D640353000F090FC8AF801001848F5F725
:100510000DFE402D11D108E00135EDB2402D08F15E
:10052000010809F107097FF4C7AE791C0020C9B2A0
:10053000FFF7B8FD01E000221A7007B0BDE8F08FA8
:100540004434030808530208BC180020891900200D
:10055000EC5202084234030852360308B053020832
:10056000893403080534030840340308CC530208D7
:100570005619002010B52148214903680A789C7B50
:10058000944203D99C8914F0200F18D09A8912F054
:10059000800F01D105E01C3B9A8912F0400FFAD080
:1005A00000E01C33036000230B7003689B8913F089
:1005B000200F16D0134BDA79114B1A7011E001326B
:1005C000D2B20A70986843F60553984209D101E007
:1005D0000132D2B2162A03D80B4853B29840F7D44E
:1005E0000A700A4A136843F480731360F8F796F8A8
:1005F000074B1A7842F006021A7010BDBC18002092
:1006000049190020561900200006008840320020B9
:100610008919002010B52349234A0B78D3B11068FB
:10062000848914F0200F15D1013BDBB20B70846874
:1006300043F60552944228D104E013B1013BDBB2EA
:1006400000E0837B162B03D8184C5AB29440F4D4A4
:100650000B701AE01368988910F0400F01D106E082
:100660001C33988910F0800FFAD0136002E00E4816
:100670001C3B036013689A7B0A709B8913F0200F60
:1006800003D00B4BDA79074B1A700A4A136843F40C
:1006900080731360F8F742F8074B1A7842F00602AD
:1006A0001A7010BD49190020BC18002000060088EF
:1006B000561900204032002089190020084B1A6882
:1006C000084B9A4204D003F580630C339A4205D15B
:1006D000054B1878003818BF01207047002070477C
:1006E000BC180020FC4E020816150020074B084AD3
:1006F0001B68934202D03832934205D1054B1878DB
:10070000003818BF0120704700207047BC18002037
:10071000B0530208161500202DE9F04F804B814D93
:100720001970A0F11103DBB2012B87B00E462870BF
:1007300006D8122801D1113800E00020F5F73CFD61
:100740002B78522B0DD1F2F7E9FC28B9F2F7DAFC3D
:1007500010B9F2F7FBFC20B1734B1A7842F0080293
:100760001A70724B724C1B78002B2DD12168714A84
:10077000914229D0704A23601370704A70481178F2
:10078000037063F3C30163F3000163F30711117096
:100790006C4A117863F3010111706B4A117863F3AD
:1007A000C5011170694A1370694A117863F34101F8
:1007B00063F3000163F382011170664A116863F309
:1007C0000C311160644A13702368002B40F05F8184
:1007D000604F7B7803F02003DBB273B15F4B93F87B
:1007E0000080B8F1000F08D149F23D60414600F0A9
:1007F00011FB3B6868F34D333B60594B187810F0A0
:100800001E0002D00020574907E0574B93F807908D
:100810009846B9F1000F05D0544907B0BDE8F04F34
:10082000F8F774B8524F97F801B0BA46BBF1000F11
:100830002DD0BBF1070F15D94E48F8F70DF84E49EA
:10084000B878652246F66153F7F7ACFF387807238E
:1008500010F003007B700EBF484948464849F8F73E
:1008600055F80CE0BBF1020F09D84248437823B198
:10087000F7F7F2FF87F80190ABE202237B701020BC
:100880003C4A014607B0BDE8F04FF7F7F7BF3D4FD0
:10089000BB795BB187F806B000F02AFC8E20594680
:1008A00001225B46CDF800B0F1F72AFF0020F2F7F5
:1008B00089FD224A20491378334843F00603137018
:1008C00000230B70314923600B7088F8033088F8DF
:1008D00001300370173303FB06FC2D49934611F8D2
:1008E0000CC089461CF0080F04D130460593FFF771
:1008F00031FC059B03FB06935B7913F0100F04D0CA
:100900002A78133AD2B2032A46D913F0200F79D0AD
:100910002B78442B40D03DD8232B3DD02A2B3AE0D6
:100920004C1900208418002069150020951900201A
:10093000BC1800204C4E02087719002089190020AD
:10094000531900209D1800204E1900205519002031
:100950006419002040320020941900201615002050
:10096000A13C00201BAC02082F0E00207ADD0208FB
:1009700050190020981900209F19002023AD02086B
:1009800002AD0208561900204D1900204919002017
:10099000CF330020552B35D18C4B1B78002B31D118
:1009A0008B4B93F80090B9F1000F2BD143F6DB206D
:1009B00000F03AFA012825D13F23FB7188F80300A3
:1009C00043F6373000F030FA3870F87900F5D64049
:1009D000353000F029FA78707E48F5F7A7FB9BF8D0
:1009E0000030304669F341038BF8003008F0B0FF67
:1009F000F8F750F8784B79482360794BC3F80090AA
:100A00002B7803702B78432B0AD1714B1B783BB9A1
:100A1000013388F80330734B3046236008F098FFA9
:100A200028781738C3B2072B27D86F49FF220AF05E
:100A300089FC9AF800106D4B60F301018AF80010F0
:100A400001F00301022918D00122032041B10090D6
:100A500001929B7868309B1802930021033206E0D4
:100A6000009001929B786C200133029304220B4684
:100A700000F058FAFF238AF8013098F80630002B6E
:100A800000F0A78152232B70594B00229A712268E3
:100A9000544B9A4250D12878A0F14303DAB2122A7B
:100AA00022D8544A5BB29A401ED5432840F0918127
:100AB000464B1B78002B40F08C8100F02DFD4E4BF7
:100AC00048B11A7803201109013191FBF0F000EBD5
:100AD0004000091A04E01A781109013101F00701F8
:100AE00061F307121A7074E1F7F7CCFF002823D0E6
:100AF000414F3A7812F0F00308D163F307123A70CD
:100B000023603E4B1A7842F008020EE0102B13D1FE
:100B100000F002FD80B13B786FF307133B700023B8
:100B20002360364B1A7842F0100230461A7007B034
:100B3000BDE8F04FFFF70EBB314B1E211A78264F50
:100B400061F346021A702B78232B1CD12368BB4219
:100B500019D12C4B172202FB0636737913F0100FB4
:100B600011D0294B1B7873B11A4EF7F793FFFDF79D
:100B7000A3FDF07900F56A50783000F055F9307037
:100B8000AA20F2F71FFC1C4E337813F0010F43D05C
:100B90002368BB420BD01D4A934208D0FFF78EFD5D
:100BA00028B9FFF7A3FD10B9AA30F2F70BFC2268B1
:100BB000174B9A4202D10020F2F704FC2B78522BFB
:100BC00040F0CC80134B53221A70C7E0161500205A
:100BD000B818002056190020CC5302084D190020E7
:100BE00078190020FC4E02085219002050190020EC
:100BF0002F0E0020002000C0891900206419002059
:100C0000061A0020CF330020771900204C4E02082E
:100C100004540208841800202368BB420BD06E4A9B
:100C2000934208D0FFF74AFD28B9FFF75FFD10B9DE
:100C3000AA30F2F7C7FB2B78552B1ED1FFF7EAFC41
:100C40003378664843F0060333708378644F03F0CB
:100C50000203DBB24BB1F7F7FFFD23681868FBF71F
:100C600015FD3B786FF341033B705E48837803F0DA
:100C70000203DBB20BB1F7F7EFFD2B78442B1ED14B
:100C8000FFF778FC3378554843F0060333708378D8
:100C9000534F03F00203DBB24BB1F7F7DDFD2368DE
:100CA0001868FBF7F3FC3B786FF341033B704D484A
:100CB000837803F00203DBB20BB1F7F7CDFD2B789D
:100CC000522B09D13378002243F001033370464B95
:100CD0001A70464B45321A70454B00271F702B780F
:100CE000232B3BD1434B3D481F70434B1F70F7F7FD
:100CF000B3FD3C48F7F7B0FD3378404943F00603B5
:100D000033700B78364A1BB33D4A013B17703D4A9E
:100D1000DBB20B7052F823303B4A23609B6893424E
:100D200002D109F09DFD19E002F5D2718B4203D08A
:100D300002F50C718B4204D10120014606F07CFFC4
:100D40000CE002F51372934208D1304B1F7005E09E
:100D5000117863F30711117023603AE02C4BDB78B4
:100D600013B10020F2F72EFB23681F7B17F00F074B
:100D700002D1FCF76DFE1BE0012F02D1F9F7D0FD87
:100D800016E0022F02D1FAF749FD11E0082F05D82D
:100D90004FF09C53BB4001D5FAF7F2FF042F03D16B
:100DA00023689B69984703E0052F01D1FAF7B6FA4B
:100DB000337803F00203DBB21BB123681868FBF73A
:100DC00065FC33786FF3410333702B780BB1084A1D
:100DD000137007B0BDE8F08F4C4E02089819002040
:100DE00089190020CC1800205319002084180020F5
:100DF0009E18002055190020941900207719002012
:100E0000491900207819002020540208CB1800202E
:100E10002F0E002007B502AB03F8011D1946012271
:100E2000002305F0B3FB0EBD07B5002302A901F8AE
:100E3000013D012205F012FC9DF807000EBD08B52A
:100E4000002305F0A3FB002008BD034610B50846AB
:100E50001446194605F002FCE0B210BD10B5034679
:100E6000002484540846194605F0F8FB204610BDBE
:100E700037B50546002400E01446012260190DF143
:100E8000070105F0EBFB9DF80730621C203BDBB24D
:100E90005A2BF1D920463EBDF8B500252C461E4BF5
:100EA0001C21585D01FB0431400000F57450623094
:100EB000043102220134FFF7C2FF1C355C2CEED155
:100EC0004FF46F5420B2042205341449FFF7B7FFE2
:100ED000A4B243F6E8339C42F4D1002548F63C47DF
:100EE0002C4615E007EB460004EB440100B259180C
:100EF0000222FFF7A4FF0136F6B2094B5A19927885
:100F0000B242EFD8013480370335142CBFB201D080
:100F10000026F2E7F8BD00BFAC7F020807340308E3
:100F2000BC8902082DE9F347044615468A46022289
:100F300043F61A610DF106001E46BDF930909DF88A
:100F400028809DF82C70FFF780FF2F4B2F499A784F
:100F5000BDF906008A705A7800EBC000CA701A7991
:100F600000F578500A715A791C304A719A791B78C9
:100F700045EAC6158A710C7081F80190CB710D722B
:100F800000B20922FFF75BFF1EB1214B1A88013224
:100F90001A80BDF8063001339BB2B3F57A7FADF805
:100FA000063002D30023ADF8063002220DF106010F
:100FB00043F61A60FFF743FFBDF80600154B188093
:100FC00000B200EBC00000F5785000F11C052430A1
:100FD00000B2FFF729FF10F0800F03D00C4B1A88E6
:100FE000013A1A8028B20021FFF714FF0A4B03F8D8
:100FF000148003EB44046770BAF1000F02D00120A3
:10100000F5F77CF8BDE8FC872C3A00206E1900202B
:101010009A180020282C0020BD2900202DE9F74334
:10102000324B1D78303DEDB2C5F10606F6B23EB347
:1010300005F11207402413E008F101080FFA89F0C6
:1010400000215FFA88F8FFF7E5FE09F10109B045D4
:101050001FFA89F9F0D1013C0737E4B2BFB21CB1E5
:10106000B9464FF00008E7E70B35013428B20021FC
:10107000E4B20135FFF7CEFEB442ADB2F5D132E0B5
:10108000122425B2684629460622FFF7DEFE9DF8A7
:10109000003043B19DF805302BB99DF803308DF831
:1010A00004308DF805300734062228466946A4B27C
:1010B000FFF7C5FEB4F5E97FE3D168460B210622B0
:1010C000FFF7C3FE9DF8003043B19DF805302BB902
:1010D0009DF803308DF804308DF805300B206946FB
:1010E0000622FFF7ACFEBDE8FE8300BFA01800207B
:1010F00070B509F0B5FB0BF035FE05F093FF05F078
:10110000B9FEF2F7C5FBA748F5F72AF843F6D12058
:10111000FFF78AFEA44BA54C187043F6D020FFF7CA
:1011200083FEA34B187043F6DC20FFF77DFEA14B36
:10113000187043F60350FFF777FE9F4B187043F685
:101140000450FFF771FE9D4B187043F6DA20FFF74D
:101150006BFE9B4B187043F6D920FFF765FE994B49
:10116000187043F6CF20FFF75FFE974B187043F6D9
:10117000CC20FFF759FE954B187043F6D220FFF7AD
:1011800053FE934B187043F6DF20FFF74DFE914B53
:10119000187043F6E820FFF747FE8F4B187043F6B0
:1011A000DD20FFF741FE237801280CBF43F0010347
:1011B0006FF30003237043F6E020FFF735FE23783A
:1011C00001280CBF43F080036FF3C713237043F66D
:1011D000E720FFF729FE814B01281A6843F6ED202E
:1011E0000CBF42F000526FF35D721A60FFF71CFEF5
:1011F0007B4B18B91A7860F3000202E01A7842F0CB
:1012000001021A7043F6EA20FFF70EFE6378012808
:101210000CBF43F001036FF30003637043F66E21CC
:1012200011227048FFF711FE6F4800210322EFF7EB
:10123000B5F800246B48235C312B03D122302146C2
:1012400011F05BFA0134112CF4D1224643F6F61169
:101250006448FFF7FAFD224643F63A216348FFF758
:10126000F4FD47F2D71104226148FFF7EEFD47F283
:10127000DB1104225F48FFF7E8FD0DF03BF9F5F7BD
:1012800077FA43F6E120FFF7CFFD5B4C237860F35C
:101290000003237043F6E220FFF7C6FD237860F3D6
:1012A0004103237043F6E420FFF7BEFD237860F38B
:1012B000C303237043F6E620FFF7B6FD237860F3FF
:1012C0004513237043F6E920FFF7AEFD237860F362
:1012D0008613237043F6E520FFF7A6FD237860F31D
:1012E0000413237043F6EB20FFF79EFD237860F391
:1012F000C713237043F6E320FFF796FD237860F3CE
:10130000820323703D48FFF78FFD3D4B3D49052289
:1013100018703D48FFF799FD3C48FFF785FD3C4BB1
:1013200018703C48FFF780FD3B4B18703B48FFF7B7
:101330007BFD3B4B18703B48FFF776FD3A4B18702E
:101340003A48FFF771FD3A4B18703A48FFF76CFDC9
:10135000394B18703948FFF767FD394B1870FFF7A4
:101360005DFE3848FFF760FD374B18703748FFF7D0
:101370005BFD374B18703748FFF756FD364B18703A
:101380003648FFF751FD364B18703648FFF74CFDD5
:10139000354B18703548FFF747FD354B002869D1AC
:1013A000187069E0B41800202A0E0020061A0020E8
:1013B000290E00202C0E002089140020F610002099
:1013C000BA3C002000000020DE1600209F180020FC
:1013D0002B0E002082330020A0320020403200205B
:1013E000A02900208D340020AF3400209E3400203E
:1013F0005832002070320020CB160020328CFFFFC4
:10140000A0370020AEA4FFFFB8120020358CFFFFEC
:101410009E370020368CFFFFD1360020388CFFFF2E
:1014200045360020398CFFFF341B00204096FFFF1B
:10143000651700209EA3FFFF3A1800203E96FFFF8D
:10144000A01800208AA3FFFF2832002007A3FFFF77
:101450001F2C002004A3FFFFB32A002006A3FFFFD8
:10146000272C002005A3FFFF212C00203A8CFFFF32
:101470008218002001221A704AF28D35002428B209
:10148000FFF7D2FC002102460B462046FEF786FB02
:10149000681C00B2FFF7C8FC012102460023204669
:1014A00001340235FEF77AFB082CADB2E7D10E48C5
:1014B000FFF7BAFC0D4B18700D48FFF7B5FC0D4B4C
:1014C00001281A780C480CBF42F020026FF3451235
:1014D0001A70FFF7A9FC094B18700948FFF7A4FC24
:1014E000BDE8704010F048BBEA8BFFFF4635002096
:1014F00020A4FFFFD8420020E98BFFFFDC21002061
:10150000ADA4FFFF034B1E211A7861F346021A7047
:10151000704700BF061A0020024B187800F0010047
:10152000704700BF061A0020014B1878C0097047A9
:10153000061A002008B5FFF7F7FF38B9044B1B78EF
:1015400013F07E0F0CBF0020012008BD012008BD54
:10155000061A0020F8B547F2CD042046FFF764FCD8
:101560002D2803DD20462D21FFF754FCA4F55C5601
:10157000353E3046FFF758FC414FC0B207EBC00084
:101580000579C5F30015A5B90DE03D4B3D4953F86C
:101590003500EFF707F820B930462946FFF73AFC47
:1015A00007E00135EDB207EBC5031B7913F0080F17
:1015B000EBD0013447F20D139C42CED143F6C42444
:1015C0002046FFF731FC2D2803DD20462D21FFF7B3
:1015D00021FC013443F6CC239C42F1D1012143F696
:1015E000E120FFF717FC012143F6E220FFF712FC90
:1015F000012143F6E420FFF70DFC012143F6E6202C
:10160000FFF708FC012143F6E920FFF703FC012165
:1016100043F6E520FFF7FEFB012143F6E320FFF749
:10162000F9FB012143F6EB20FFF7F4FB002143F621
:10163000E020FFF7EFFB002143F6EA20FFF7EAFB8B
:10164000002143F6EC20FFF7E5FB012143F6DC2007
:10165000FFF7E0FB002149F23F60FFF7DBFB48F6B4
:10166000A8300121FFF7D6FB47F2B5142046FF2131
:10167000FFF7D0FB013447F2BD139C42F6D1F8BD11
:1016800014040020B616030810B508F013F90BF087
:1016900033FB074B4FF416721A80012147F2C51035
:1016A000FFF7B8FB4C20BDE8104000F01BB800BFAE
:1016B000B83C002010B508F013F90BF0B1FA044B58
:1016C000002147F2C5101980BDE81040FFF7A2BB0A
:1016D000B83C0020024B1888003818BF0120704722
:1016E000B83C0020542873B5044663D83D4BDB78E2
:1016F00003F02003DBB2002B72D13F2801D811F098
:1017000027FE394D35F81460002E69D1E10001F54E
:10171000DA416846D5310822FFF797FB3348214666
:1017200011F001F850B1F3B2072B07D03F2C05D8C8
:101730000122B240D243D2B22D4B27E01DF8063031
:101740000122542B08D0562B03D0532B284B1AD1EF
:1017500000E0284BB24007E0B240254BD2B2195D01
:1017600042EA01011955234B195D0A431A55FFF747
:10177000D3FE98B1204B1B7883B13F2C0ED81E337B
:1017800025F814300AE0B240D243D2B2195D02EA21
:1017900001011955174B195D0A401A550136082EDB
:1017A000BCD1134B1A5D134B1B5D134318D125F8A5
:1017B000143015E0C10001F5DA416846D531082240
:1017C000FFF743FB00231DF803202D2A05D001213C
:1017D0009940074A105D014311550133082BF2D19E
:1017E0007CBD00BF403200200A1A0020F0250020F6
:1017F000D61E0020311D00205C1700201FB501F00F
:1018000015F910B901F026F948B10021FF23009322
:101810000B2004220B4601910291FFF783FBAD22BE
:101820000023D9B24D2909D0012A07D90D4800213A
:1018300019540D4819540D4820F813100133013282
:10184000552BD2B2EDD1074B002183F85510084B30
:1018500008481970084B0822197005B05DF804EBB0
:10186000EEF79CBDD61E0020311D00200A1A002074
:10187000951B0020741B0020081A002059B1064B4C
:101880000C2202FB0030437AC918837A4172083077
:101890000BB93C33837070473C260020072813B5F2
:1018A000044624D9124B1B5C022B20D10DF10701F9
:1018B0000DF1060208F002FA58B19DF80610012059
:1018C00010FA01F19DF807300A4AD05C0143D15467
:1018D0000DE0083CE4B2E308012104F0070411FA2A
:1018E00004F4054A0133D15C41EA0404D4541CBD1C
:1018F00068240020F5320020EC320020044B0C223A
:1019000002FB00330C3A5A729A72FFF7C7BF00BF4E
:101910003C26002010B50446FFF7F0FF034B0C22D5
:1019200002FB0434FF23637210BD00BF3C2600207D
:1019300070B5104D002410482146E6B210F0F3FEB9
:1019400098B96B7A8BB10D4AA318A25C93F88030DA
:10195000022A0AD0413BDAB2122A06D8084A5BB200
:101960009A4002D53046FFF7C9FF01340C35402CB0
:10197000E1D170BD3C260020CC1600206824002058
:101980000020008810B50A4B0C2203EBD00393F81B
:101990008011084B02FB00331C7A3CB900F00700B1
:1019A00051FA00F010F0010F18BF1A7210BD00BFFD
:1019B000682400203C260020044B0C2202FB00334C
:1019C0001A7AFF2A01D1FF3A1A7270473C2600208A
:1019D000104B1B7813F0010F02D10F4B187818B180
:1019E0000E4B03F540720CE00C4B03F54072197A74
:1019F0000C330139C9B2FD2998BF01209342F6D1B9
:101A00007047197A09B1FF2119720C339342F8D14A
:101A100000207047F21600205C1700203C260020B2
:101A200030B504461048007800F00200C0B2C8B1DA
:101A30000C2060430D4D285C904201D1994207D0A3
:101A4000984201D1914203D0052A0BD1052B09D12F
:101A50000C2303FB0455064821462B72BDE8304099
:101A600010F056BE30BD00BFC11800203C2600203B
:101A7000C21800201FB504462146144810F053FE3A
:101A8000002821D00122022300210093A3180293F1
:101A90005C200B460192FFF745FA21460B4810F0F7
:101AA00037FE21460A4810F033FE2146094810F05F
:101AB00024FE074BE40804F5CC40195DCA3004B09D
:101AC000BDE81040FFF7A6B904B010BD51150020C5
:101AD0006C150020CC16002010B50D4C00210822FA
:101AE0002046EEF75BFC43F6F120FFF79DF92071ED
:101AF00043F6F220FFF798F943F6F42160710222D1
:101B00002046FFF7A2F9A37943F00203A37110BDA9
:101B1000B41A00200A4B1B781D2B0A4B0BD89A795C
:101B200012F0010F03D05A880AB1013A5A809A790B
:101B30006FF3000202E09A7942F001029A71704755
:101B40002C3A0020B41A00202DE9F0436F4885B0EC
:101B500010F08EFDDFF8D0816D4E0024E5B22846EE
:101B600005F0FEFA18F8019F074618F8403C13B13B
:101B7000022B3ED10FE02846FFF7C0FE2146654804
:101B800010F0C6FD2146644810F0C2FD21466348AE
:101B900010F0BEFDDAE028464946F3F72DFE10B1FD
:101BA0002846FFF79FFD737AFF2B01D1FF3B73722D
:101BB000737A4B4501D2F37A9BB15448214610F019
:101BC0009CFDF37A002B40F0C180204605F02EFEEC
:101BD000052128460A460B46FFF722FF2846FFF755
:101BE0008DFEF37A002B40F0B1802846FFF742FFCC
:101BF000ACE090B92846FFF781FE2146434810F03B
